:1000000080EC0020A5AF00009112050079AF000040
:1000100079AF000079AF000079AF00000000000068
:1000200000000000000000000000000005A7000024
:1000300079AF00000000000071A6000079AF000059
:1000400095A80000DB2D050095A8000095A80000EC
:1000500095A8000095A8000095A8000095A80000AC
:10006000A32D050095A8000095A80000C12D05004E
:1000700095A8000095A8000095A8000095A800008C
:1000800095A8000095A8000095A8000095A800007C
:1000900095A8000095A8000095A8000095A800006C
:1000A00095A8000095A8000095A8000095A800005C
:1000B00095A8000095A8000095A8000095A800004C
:1000C00095A8000095A8000095A8000095A800003C
:1000D00095A8000095A8000095A8000095A800002C
:1000E00095A8000095A8000095A8000095A800001C
:1000F00095A8000095A8000095A8000095A800000C
:1001000081F0004102E000BF83F0004330B54FEAC8
:1001100041044FEA430594EA050F08BF90EA020F35
:100120001FBF54EA000C55EA020C7FEA645C7FEAC8
:10013000655C00F0E2804FEA5454D4EB5555B8BFEB
:100140006D420CDD2C4480EA020281EA030382EA5C
:10015000000083EA010180EA020281EA0303362DEE
:1001600088BF30BD11F0004F4FEA01314FF4801CC1
:100170004CEA113102D0404261EB410113F0004FD3
:100180004FEA03334CEA133302D0524263EB43038A
:1001900094EA050F00F0A780A4F10104D5F1200E28
:1001A0000DDB02FA0EFC22FA05F2801841F1000183
:1001B00003FA0EF2801843FA05F359410EE0A5F157
:1001C00020050EF1200E012A03FA0EFC28BF4CF088
:1001D000020C43FA05F3C01851EBE37101F000453E
:1001E00007D54FF0000EDCF1000C7EEB00006EEB4B
:1001F0000101B1F5801F1BD3B1F5001F0CD34908D5
:100200005FEA30004FEA3C0C04F101044FEA44522B
:1002100012F5800F80F09A80BCF1004F08BF5FEAB2
:10022000500C50F1000041EB045141EA050130BD92
:100230005FEA4C0C404141EB0101013C28BFB1F5A4
:10024000801FE9D291F0000F04BF01460020B1FAEF
:1002500081F308BF2033A3F10B03B3F120020CDAC2
:100260000C3208DD02F1140CC2F10C0201FA0CF0A0
:1002700021FA02F10CE002F11402D8BFC2F1200C05
:1002800001FA02F120FA0CFCDCBF41EA0C019040BB
:10029000E41AA2BF01EB0451294330BD6FEA040404
:1002A0001F3C1CDA0C340EDC04F11404C4F12002EF
:1002B00020FA04F001FA02F340EA030021FA04F301
:1002C00045EA030130BDC4F10C04C4F1200220FA58
:1002D00002F001FA04F340EA0300294630BD21FA96
:1002E00004F0294630BD94F0000F83F4801306BF5C
:1002F00081F480110134013D4EE77FEA645C18BF50
:100300007FEA655C29D094EA050F08BF90EA020FE6
:1003100005D054EA000C04BF1946104630BD91EADE
:10032000030F1EBF0021002030BD5FEA545C05D1E1
:100330004000494128BF41F0004130BD14F5800420
:100340003CBF01F5801130BD01F0004545F0FE4194
:1003500041F470014FF0000030BD7FEA645C1ABFC9
:10036000194610467FEA655C1CBF0B46024650EA00
:10037000013406BF52EA033591EA030F41F400212C
:1003800030BD00BF90F0000F04BF0021704730B5B2
:100390004FF4806404F132044FF000054FF0000187
:1003A00050E700BF90F0000F04BF0021704730B548
:1003B0004FF4806404F1320410F0004548BF40421D
:1003C0004FF000013EE700BF42004FEAE2014FEA72
:1003D00031014FEA02701FBF12F07F4393F07F4F4D
:1003E00081F06051704732F07F4208BF704793F050
:1003F0007F4F04BF41F40021704730B54FF4607463
:1004000001F0004521F000411CE700BF50EA010265
:1004100008BF704730B54FF000050AE050EA01020E
:1004200008BF704730B511F0004502D5404261EB7E
:1004300041014FF4806404F132045FEA915C3FF4BF
:10044000D8AE4FF003025FEADC0C18BF03325FEA5C
:10045000DC0C18BF033202EBDC02C2F1200300FA0D
:1004600003FC20FA02F001FA03FE40EA0E0021FA32
:1004700002F11444BDE600BF70B54FF0FF0C4CF420
:10048000E06C1CEA11541DBF1CEA135594EA0C0FD2
:1004900095EA0C0F00F0DEF82C4481EA030621EA0D
:1004A0004C5123EA4C5350EA013518BF52EA033548
:1004B00041F4801143F4801338D0A0FB02CE4FF0FA
:1004C0000005E1FB02E506F00042E0FB03E54FF02A
:1004D0000006E1FB03569CF0000F18BF4EF0010E22
:1004E000A4F1FF04B6F5007F64F5407404D25FEA1E
:1004F0004E0E6D4146EB060642EAC62141EA5551D1
:100500004FEAC52040EA5E504FEACE2EB4F1FD0C12
:1005100088BFBCF5E06F1ED8BEF1004F08BF5FEA90
:10052000500E50F1000041EB045170BD06F0004642
:1005300046EA010140EA020081EA0301B4EB5C04EF
:10054000C2BFD4EB0C0541EA045170BD41F48011E7
:100550004FF0000E013C00F3AB8014F1360FDEBF0C
:10056000002001F0004170BDC4F10004203C35DAE8
:100570000C341BDC04F11404C4F1200500FA05F36B
:1005800020FA04F001FA05F240EA020001F000420C
:1005900021F0004110EBD37021FA04F642EB060182
:1005A0005EEA430E08BF20EAD37070BDC4F10C04AC
:1005B000C4F1200500FA04F320FA05F001FA04F270
:1005C00040EA020001F0004110EBD37041F100015C
:1005D0005EEA430E08BF20EAD37070BDC4F1200567
:1005E00000FA05F24EEA020E20FA04F301FA05F2CF
:1005F00043EA020321FA04F001F0004121FA04F277
:1006000020EA020000EBD3705EEA430E08BF20EA46
:10061000D37070BD94F0000F0FD101F00046400080
:1006200041EB010111F4801F08BF013CF7D041EA02
:10063000060195F0000F18BF704703F00046520006
:1006400043EB030313F4801F08BF013DF7D043EAD7
:100650000603704794EA0C0F0CEA135518BF95EA8D
:100660000C0F0CD050EA410618BF52EA4306D1D114
:1006700081EA030101F000414FF0000070BD50EA33
:10068000410606BF1046194652EA430619D094EABD
:100690000C0F02D150EA013613D195EA0C0F05D1A7
:1006A00052EA03361CBF104619460AD181EA0301FB
:1006B00001F0004141F0FE4141F470014FF00000B3
:1006C00070BD41F0FE4141F4780170BD70B54FF04E
:1006D000FF0C4CF4E06C1CEA11541DBF1CEA1355CE
:1006E00094EA0C0F95EA0C0F00F0A7F8A4EB0504B0
:1006F00081EA030E52EA03354FEA013100F08880A7
:100700004FEA03334FF0805545EA131343EA12636F
:100710004FEA022245EA111545EA10654FEA002624
:100720000EF000419D4208BF964244F1FD0404F5DD
:10073000407402D25B084FEA3202B61A65EB030539
:100740005B084FEA32024FF480104FF4002CB6EBF6
:10075000020E75EB030E22BFB61A754640EA0C0076
:100760005B084FEA3202B6EB020E75EB030E22BFB6
:10077000B61A754640EA5C005B084FEA3202B6EBF7
:10078000020E75EB030E22BFB61A754640EA9C00B6
:100790005B084FEA3202B6EB020E75EB030E22BF86
:1007A000B61A754640EADC0055EA060E18D04FEA44
:1007B000051545EA16754FEA06164FEAC30343EAE4
:1007C00052734FEAC2025FEA1C1CC0D111F4801FB1
:1007D0000BD141EA00014FF000004FF0004CB6E7AA
:1007E00011F4801F04BF01430020B4F1FD0C88BF49
:1007F000BCF5E06F3FF6AFAEB5EB030C04BFB6EB54
:10080000020C5FEA500C50F1000041EB045170BD46
:100810000EF0004E4EEA113114EB5C04C2BFD4EB73
:100820000C0541EA045170BD41F480114FF0000EF7
:10083000013C90E645EA060E8DE60CEA135594EA73
:100840000C0F08BF95EA0C0F3FF43BAF94EA0C0F76
:100850000AD150EA01347FF434AF95EA0C0F7FF4EB
:1008600025AF104619462CE795EA0C0F06D152EA3F
:1008700003353FF4FDAE1046194622E750EA410623
:1008800018BF52EA43067FF4C5AE50EA41047FF434
:100890000DAF52EA43057FF4EBAE12E77BB972B9B4
:1008A0000029BEBF00204FF0004106E008BF00282D
:1008B0001CBF6FF000414FF0FF3000F0B9B9ADF14F
:1008C000080C6DE904CE002909DB002B1ADB00F0CF
:1008D0004DF8DDF804E0DDE9022304B07047404242
:1008E00061EB4101002B1BDB00F040F8DDF804E078
:1008F000DDE9022304B0404261EB4101524263EB67
:1009000043037047524263EB430300F02FF8DDF8D6
:1009100004E0DDE9022304B0404261EB410170478D
:10092000524263EB430300F021F8DDF804E0DDE917
:10093000022304B0524263EB4303704753B94AB9F0
:10094000002908BF00281CBF4FF0FF314FF0FF30D7
:1009500000F06EB9ADF1080C6DE904CE00F006F8B8
:10096000DDF804E0DDE9022304B070472DE9F0472B
:10097000089D04468C46002B40F083808A4217462F
:1009800047D9B2FA82F242B1C2F1200024FA00F053
:100990009140974040EA010C94404FEA1748230CDD
:1009A000BCFBF8F61FFA87FE08FB16C143EA0143B9
:1009B00006FB0EF1994209D9FB1806F1FF3080F0D1
:1009C0001981994240F21681023E3B445B1AA4B25F
:1009D000B3FBF8F008FB103344EA034400FB0EFEBF
:1009E000A64509D93C1900F1FF3380F00581A645E1
:1009F00040F2028102383C4440EA0640A4EB0E0477
:100A000000261DB1D4400023C5E900433146BDE8AE
:100A1000F08702B9FFDEB2FA82F2002A50D1CB1B76
:100A20004FEA174E1FFA87F80126B3FBFEFC210C94
:100A30000EFB1C3341EA034108FB0CF38B4207D940
:100A400079180CF1FF3002D28B4200F2E980844623
:100A5000C91AA3B2B1FBFEF00EFB101143EA014428
:100A600008FB00F8A04507D93C1900F1FF3302D27A
:100A7000A04500F2D9801846A4EB080440EA0C40D7
:100A8000BFE78B4209D9002D00F0B1800026C5E9EF
:100A9000000130463146BDE8F087B3FA83F6002EF8
:100AA0004AD18B4202D3824200F2B880841A61EBB1
:100AB000030101208C46002DA8D0C5E9004CA5E714
:100AC000C2F1200320FA03F6974001FA02F04FEA40
:100AD000174ED9403043030CB1FBFEF61FFA87F8DE
:100AE0000EFB161143EA014306FB08F1994204FA92
:100AF00002F409D9FB1806F1FF3C80F08D80994281
:100B000040F28A80023E3B445B1A81B2B3FBFEF0A6
:100B10000EFB103341EA034100FB08F38B4207D977
:100B2000791800F1FF3C73D28B4271D902383944F5
:100B3000CB1A40EA064678E7C6F1200C03FA06F421
:100B400022FA0CF31C4320FA0CF701FA06F34FEAE1
:100B5000144E21FA0CF11F433B0CB1FBFEF91FFAB6
:100B600084F80EFB191143EA014109FB08FA8A4592
:100B700002FA06F200FA06F308D9611809F1FF300B
:100B800048D28A4546D9A9F102092144A1EB0A01BC
:100B9000BFB2B1FBFEF00EFB101147EA014700FBAC
:100BA00008F8B84507D9E71900F1FF312ED2B8454A
:100BB0002CD90238274440EA0940A7EB0807A0FBDC
:100BC00002894F45C64649461AD317D05DB1B3EBEB
:100BD0000E0267EB010707FA0CFCF2404CEA020236
:100BE000F740C5E9002700263146BDE8F0872E46CC
:100BF00028460BE70646E9E61846FDE64345E5D2FA
:100C0000B8EB020E69EB04010138DFE70846D2E7D2
:100C100060468DE78146B9E7664675E730464AE7A4
:100C2000ACF1020C394413E702383C4424E700BF1E
:100C3000704700BFF8B515460A4A1C4656682EB1E3
:100C400001B02A46B446BDE8F040604700208DF868
:100C50000000684603F04AFA9DF80000281A207048
:100C60000020F8BD00000020002819D003781349A7
:100C7000134A13B1012B0ED011E00379012B00D0E0
:100C80006BB943790BB1012B09D18368643B8B426B
:100C900005D2C0680EE00379012B02D00BB1002011
:100CA000704743790BB1012BF9D1C368643B8B4288
:100CB000F5D280689042F2D8012070473D8601004D
:100CC000FF1FA10710B5054C206810B18047002018
:100CD0002060BDE8104001F035BC00000800002095
:100CE0002DE9F0410E46050004D000F045F8074616
:100CF00000240AE06FF01500BDE8F081204600F006
:100D000041F8807838B1641CE4B2BC42F6D300BF2D
:100D10006FF00B00F0E72746FF2CF9D0204600F0DB
:100D200031F8044603F085FB27712146074801F09E
:100D3000E1FBE070202805D00120A560A07037708D
:100D40000020D9E76FF02200D6E7000093410000B1
:100D500010B5820702D06FF00D0010BD054A11706A
:100D6000506028B101EBC1018A00002103F097FD1A
:100D7000002010BD0C0000200148007870470000E2
:100D80000C00002005490A78904201D300207047EA
:100D9000496800EBC00001EB800070470C000020A8
:100DA00070B50546202A27D019481A4C00EB831C41
:100DB0000CEB420004EB8303202922D00CEB410111
:100DC00040784C784870204601460CEB4100914237
:100DD00005704078F8D193F82220202A1ABF0CEB36
:100DE0004202547083F8214020220CEB410C8CF815
:100DF000012083F8221070BD40F27E21702002F0A5
:100E0000ADFD93F82040407883F82000DBE7000038
:100E1000800C0020000D00202DE9FF4F85B0154605
:100E20000C4601F027FD284420F07F400290216805
:100E3000081A0002C11700EB11600012002800F32D
:100E4000D580AC48089FAC4E00EB8700039090F82B
:100E500020502020E9460DF104088DF8000006F529
:100E6000407A202D18BF0AEB871B25D005EB4500E3
:100E700006EBC0002268C168511A0902CA1701EBCB
:100E800012610830091217D4618971B1418961B9C1
:100E900000F0B2FD01F0EEFC2168081A0002C11753
:100EA00000EB11600012332806DB0BEB450089F8DC
:100EB00000504578202DD9D199F8000088F800001D
:100EC000A146202D1CBF8D4800EB871B00F00E8132
:100ED00005EB450106EBC10AD9F80420DAF8081041
:100EE0004846891A0902CA1701EB12610AF108077C
:100EF000091215D47989002900F0F8804189002968
:100F000040F0F48000F078FD01F0B4FC3968081A74
:100F10000002C11700EB11600012332880F2E68056
:100F200088F800509AF8141099F80C00814206D9FC
:100F30000BEB45004578202DCAD100F0D7B89DF8BD
:100F4000040000EB400006EBC005688AEF6800284B
:100F500043D16089E8B3A86803F0FFFA698A2A7C64
:100F6000674B1144491C4218984204D940F2096168
:100F7000702002F0F3FC6348814204DD40F20A6114
:100F8000702002F0EBFC6048814204DA40F20B6111
:100F9000702002F0E3FC5D489042DCBF02F5F702EE
:100FA000A2F1F85205DD002ABCBFA2F5F70202F15A
:100FB000F852104601F05EFC20F07F41781A0002E2
:100FC000C21700EB126000123328B8BF01F13300E2
:100FD00000E002E0B8BF20F07F470298381A000214
:100FE000C11700EB11600012002803DD09B00020DA
:100FF000BDE8F08FD4E90010401A384427F07F4153
:1010000020F07F40C4E900100398DDF820806F468F
:1010100090F8205020200DF1040A8DF80000202DBA
:101020001CBF364800EB881925D000BF05EB4500F2
:1010300006EBC0002268C168511A0902CA1701EB09
:1010400012610830091216D4618971B1418961B900
:1010500000F0D2FC01F00EFC2168081A0002C11752
:1010600000EB11600012332805DB09EB45003D70F1
:101070004578202DDAD138788AF800002746202DCF
:101080001CBF1E4800EB881B30D005EB450106EB6A
:10109000C1097968D9F808203846511A0902CA17D7
:1010A00001EB126109F10808091212D4B8F80A100C
:1010B000E1B14189D1B900F09FFC01F0DBFBD8F828
:1010C0000010081A0002C11700EB1160001233284B
:1010D0000CDA8AF8005099F81400397B88427FF6C0
:1010E0002EAF0BEB45004578202DCED109B0012065
:1010F000BDE8F08F000D002080090020800C00204A
:10110000FF7F841E0020A10700E05EF80080841E9F
:101110002DE9F05F04463C480E4600EB86003B4F4D
:1011200090F82050202098469246107007F540799C
:10113000202D18BF09EB861B28D000BF05EB45000A
:1011400007EBC00000F10801C0682268101A000215
:10115000C21700EB1260001218D4608978B1488978
:1011600068B9084600F048FC01F084FB2168081AC1
:101170000002C11700EB11600012332806DB0BEBF5
:1011800045008AF800504578202DD7D19AF8000004
:1011900088F80000202D18BF09EB861A30D005EB27
:1011A000450107EBC1096168D9F808202046511AAA
:1011B0000902CA1701EB126109F10806091210D4DD
:1011C0007189E9B14189D9B900F016FC01F052FBEF
:1011D0003168081A0002C11700EB116000123328B1
:1011E0000EDA88F8005099F81400217B884202D862
:1011F0000020BDE8F09F0AEB45004578202DCED1B8
:101200000120BDE8F09F0000000D002080090020B3
:101210002DE9F74F98B016460D464FF000084FF0F5
:10122000010B01F0A9FD0446012D18BF022D05D0C8
:1012300040F694114FF0700002F090FBF849012045
:101240000860F8498968086000208DF84E000C900D
:10125000401E0E90F44806EB460100EBC101083138
:101260000FAF0FC987E80F000FA800F0C5FB0D9066
:10127000ED48BDF84690B0F89C03ADF84C00B9F1CC
:10128000000F14BF4FF0010A4FF0000A0F9814909E
:10129000BAF1000F09D0E54890F82C0028B902F007
:1012A000E5FA002808BF012700D00027E048002108
:1012B000159100780E46012818BF03283FD1DC485D
:1012C000B0F80280A8EB09001590C84537D90D9BEE
:1012D000DFF860E36FEA080C03A917AA03EB0C0020
:1012E000734504D940F20961702002F037FBD24BFC
:1012F0009C4504DD40F20A61702002F02FFBCF4BC9
:101300009C4504DA40F20B61702002F027FBCC4BC5
:101310008342DCBF00F5F700A0F1F85005DD00289E
:10132000BCBFA0F5F70000F1F85001F0BFFA039838
:101330000F9920F07F400390081A20F07F41002F82
:1013400018BF322604D19DF84C00002818BF022691
:10135000B4F1807F08D00F98001B0002C21700EB89
:1013600012600012012802DA042218980BE047B13B
:10137000AE4890F82D0020B19DF84C00061C18BF17
:10138000022620460122B9F1000F02D0159B1E2B28
:1013900002DA9DF84C3013B14FF0000B521EA44BF3
:1013A0009DF84DE032441B7815930F9B5B1A23F098
:1013B0007F4CACEB00031B02DE1703EB16631B1222
:1013C000934218DB002918BFCDF83CC00F9E05974B
:1013D000002701F0C9FB301A0002C11700EB1160B1
:1013E00000123E283FDA012D20D0701E059920F012
:1013F0007F4019B32DE081B1BEF1000F04BF159BF2
:10140000032B0AD027B99DF84C10002918BF921E53
:1014100000218DF84C108846C7E707BB9DF84C307B
:10142000EBB100238DF84C30921EBEE7B4F1807F03
:1014300020D140F60D11702002F090FAB4F1807FB7
:1014400007D0211A0902CA1701EB126109120429F7
:1014500003DD044601F08EFB0CE000290ADD1BB021
:101460000020BDE8F08F701E20F07F44204601F080
:1014700081FB5746B4F1807F24D00F98714A001B3E
:1014800020F07F411098001B20F07F408B4598BFD3
:10149000B1F5800FE3D28242E1D3204603F05DF83C
:1014A00064490D9A4B1C161AB6EB930F24BFA0EBA0
:1014B000020CBCEB930F10D3B14208D2081A1044AF
:1014C000461C0AE040F62D21702002F047FA6145E3
:1014D0002CD2891A0844401C46425448807F50B39D
:1014E000284645464FF0000BD846012805D002207B
:1014F00001F098FD012001F095FDA94527D2A6EB4A
:1015000005014FF001034FF003024FF0020001F01C
:10151000B5FC002808BF4FF00108B9F1000F30D02A
:101520000123A6EB0901032218461EE040F60C3108
:10153000702002F013FAC14534BF40464846584473
:10154000B042CDDB4FF42461702002F007FA10D9CD
:101550000123A6EB09010322184601F08FFC28B3F2
:101560007DB1711B01230322022001F087FCE8B149
:1015700007E055EA090004D040F67711702002F028
:10158000EDF9012303223146002001F077FC68B118
:101590000125B8F1000F03D014980F908DF84CB0CE
:1015A000DFF8A480BAF1000F0ED109E0022001F0AB
:1015B00039FD012001F036FD1BB00020BDE8F08FA1
:1015C0001A4890F82D0000B14FB3DFF860A09AF8E8
:1015D0002C0018B102F018F88AF82CB0D7B3A4F197
:1015E000320020F07F414FF40020C8F800000023B3
:1015F0000322052001F042FC68B34FF0804405202F
:1016000001F0F6FD1149C1F81005C1F81445104963
:10161000E0120860054C94F82D00E8B330E01BE0C0
:10162000080500401400002080090020000D002063
:1016300016000020FF7F841E0020A10700E05EF856
:101640000080841EFFFF3F0008F5014098F0014034
:1016500004F5014005E025E0DFF8B4A09AF82C007D
:10166000C8B12B4C94F82D0050B14FF40020C8F8AD
:101670000000052001F0D6FC02F02EF884F82DB011
:10168000A6EB0900A0F11901002915DC40F6712133
:10169000702002F063F900E009E001F0D1FF8AF860
:1016A0002C509BE740F23E31702002F057F902F0D7
:1016B00005F884F82D50E3E703220123104601F0DA
:1016C000DDFBF8B113488068C0F800B01248C0F8DC
:1016D00000B00DF13008114898E8FE10C0F88013F2
:1016E000C0F88423C0F88833C0F88C43C0F8905306
:1016F000C0F89463C0F89873C0F89CC31BB0012075
:10170000BDE8F08F40F67921702002F027F9000043
:10171000000D002014000020080500408009002072
:101720002DE9F043064683B008789073CF7A57735B
:10173000887A10730889144650810D460A785F49EB
:1017400099464FEA810C4B42ACF101085AB1C043B3
:10175000D5F8048004F1080288423DDD40F20A61B8
:10176000702002F0FBF8EE686D686FEA000904F182
:10177000080206EB0900464504D940F209617020D1
:1017800002F0ECF88945E9DC994528DB8445DCBFAB
:1017900000F5F700A0F1F85005DD0028BCBFA0F56A
:1017A000F70000F1F850214601F080F8206820F0A1
:1017B0007F417019401C2160002F08BF7A3003D090
:1017C000012F08BF48302DD101F054F820F07F40A0
:1017D000606003B0BDE8F0830146984204DA40F24D
:1017E0000B61702002F0BAF88445DCBFA1F1F4501F
:1017F000A0F5902005DD0028BCBF01F1F45000F5F4
:101800009020214601F052F82068002F20F07F41FF
:1018100008F10100216008BF7A3008D0012F08BF0D
:10182000483004D040F2B161702002F097F801F026
:1018300021F820F07F416160608901AA694601F0CA
:1018400035F81F4890F82F10202923D00069401D3B
:1018500020F07F40D4E90021891A2060084420F05C
:101860007F4060604B4632462146E868FFF7D4FA75
:1018700000281CBF03B0BDE8F083D4E90010401A73
:10188000304426F07F4120F07F40C4E9001003B0CF
:10189000BDE8F083608906F1090720B101F0E6FF99
:1018A000002808BF3237074841780098814284BF3A
:1018B000081A074427F07F40CCE700000020A1076A
:1018C000000D00201600002010B5154C94F82F00D4
:1018D000202818BF10BD94F82E2004EB820090F849
:1018E0002010202917D0DFF83CC00CEB821303EB4B
:1018F00041035B7880F82030012380F8233084F89E
:101900002B3084F82F10022000F0B0F8002084F86B
:101910002A00A07710BD40F28B31702002F01EF833
:10192000000D0020800C00202DE9F05FDFF8B8806A
:1019300098F82E5008EB850090F82140202C08BF25
:10194000BDE8F09FDFF8A4B0DFF8A4A0AAF54079C5
:101950000AEB8517072617F8140001280ED0042873
:1019600008BF02260AD005280CBF0326062805D08A
:1019700040F6D9014FF0700001F0F0FFBBF1000F0D
:1019800018BFAFF30080EFF3108072B607EB44018D
:101990004A7808EB850181F8212091F82220A242A3
:1019A00004BF202281F82220B8B12A462146012016
:1019B00000F05CF804EB440109EBC10059F8312058
:1019C00040683146904798F82E5008EB850090F813
:1019D0002140202CBCD1BDE8F09F0648002818BF4C
:1019E000AFF3008062B6E0E7000D002000000000C9
:1019F000800C00200000000010B50446006802F0D2
:101A0000ACFD02466089217A144B0844411C5018F1
:101A10009A4204D940F20961702001F09FFF104AF8
:101A2000914204DD40F20A61702001F097FF0D4AF7
:101A3000914204DA40F20B61702001F08FFF0A49F5
:101A40008142DEBF00F5F700A0F1F85010BD00287C
:101A5000BCBFA0F5F70000F1F85010BDFF7F841E59
:101A60000020A10700E05EF80080841EDFF854C06B
:101A700010B500230CEB821C07281ED2DFE800F013
:101A8000050505050404040001230CF81100002BD2
:101A900008BF10BD0C4800EB820292F822002028FB
:101AA0000EBF82F821100CEB4000417020200CEB9F
:101AB0004103587082F8221010BD4FF41571702048
:101AC00001F04CFF800C0020000D00202DE9F34FA9
:101AD00083B05C48049900EB8100019090F82040AD
:101AE00003982546012818BF022805D04FF42B6122
:101AF0004FF0700001F032FF0027202D4AD05148EE
:101B000000910026807F002808BF022601F02CF8F3
:101B1000DFF838A104EB44010AEBC101DFF828919A
:101B20008A68C968121A091A22F07F4221F07F419F
:101B3000964298BFB2F5800F01D2894528D2444A17
:101B4000009902EB811B22460BEB42014C78202CC2
:101B500016D004EB44010AEBC10CDCF80880DCF879
:101B60000CC0A8EB000828F07F48ACEB000121F086
:101B70007F41464598BFB8F5800FE4D28945E2D34E
:101B8000202A05D020210420009BFFF709F90446F4
:101B9000AC4215D12F48002818BFAFF3008000F0E9
:101BA000E3FF284C94F8301020290DD0E168821C06
:101BB000511A0902CA1701EB12610912002903DD4B
:101BC00005B00020BDE8F08F202D0DD02A460399E6
:101BD000FFF71EFB58B3019880F8237084F830504B
:101BE00005B00120BDE8F08F94F82C0018B101F089
:101BF0000BFD84F82C7094F82D0050B116494FF469
:101C000000200860052001F00DFA01F065FD84F860
:101C10002D70042001F006FA01F072FA202084F8F9
:101C200030000E48806807600D480760D8E72A46F4
:101C300020210420049BFFF7B3F805B00020BDE885
:101C4000F08F0000000D0020FFFF3F008009002002
:101C5000800C00200000000008F501401400002066
:101C6000080500402DE9F04F5B4E814685B096F89F
:101C70002F008A4620284DD096F82F0006F10C043C
:101C800000EB4000A6F5607808EBC00720208DF837
:101C9000000096F82E0003AA06EB800001A990F838
:101CA0002050306902903068484400F0FFFDF86829
:101CB00001994A4A0844A9F1650191422FD8B968AF
:101CC000411A21F07F41B1F5800F28D220F07F40EA
:101CD0006060304684F80CA090F82E00EA46202D73
:101CE0001CBF3F4901EB801B3CD005EB450008EBD6
:101CF000C0076068BA682146101A0002C21700EBDC
:101D0000126007F1080600121BD4708950B348898D
:101D100048B127E040F67B31702001F01FFE05B08E
:101D20000120BDE8F08F2046FFF766FE00F0A2FD1F
:101D30003168081A0002C11700EB11600012332845
:101D400010DA8AF80050397D207B814205D802984C
:101D5000606005B00220BDE8F08F0BEB45004578D0
:101D6000202DC2D1052001F05DF91B4C4FF0FF3052
:101D7000A06094F82E309DF800202021202A13BF67
:101D8000052004EB830090F82000FFF709F894F891
:101D90002E20134901EB821194F82F2001EB420110
:101DA0004870206848442060012084F82B00607E41
:101DB000012805D12069401E20F07F4000F078FF07
:101DC0009DF80000202803D00648407801F096FED8
:101DD00005B00020BDE8F08F000D00209B1FA1077B
:101DE000800C00201400002070B5234A92F82F10B8
:101DF000202939D092F82F10A2F5607301EB410130
:101E000003EBC10C92F82E1092F82E4002EB8101E8
:101E100091F82010A2F1800505EB8414202928D028
:101E200001EB410503EBC5052D7D854284BF04EB25
:101E300041014978F2D801EB410103EBC101DCF823
:101E40000C0089681468081A0002C11700EB1160C1
:101E5000001207D402F081FB04F16501884224BF1F
:101E6000001B70BD002070BD40F64D31702001F0A8
:101E700075FD4FF0FF3070BD000D00200246144B81
:101E800010B508449A4204D940F20961702001F06B
:101E900065FD104A914204DD40F20A61702001F0B4
:101EA0005DFD0D4A914204DA40F20B61702001F0B1
:101EB00055FD0A498142DEBF00F5F700A0F1F85058
:101EC00010BD0028BCBFA0F5F70000F1F85010BD10
:101ED000FF7F841E0020A10700E05EF80080841EC2
:101EE000074991F83020824204BF4868704700EBF0
:101EF0004000044901EBC0000830FFF77DBD000041
:101F0000000D0020800900200E4910B591F82F0027
:101F1000202812D091F82F00A1F5607200EB40004C
:101F200002EBC00091F82F10406801EB410152F81C
:101F30003120BDE810400421104740F6BC0170205C
:101F400001F00CFD000D0020F8B56D4D6D49012626
:101F500005F56074082873D2DFE800F004679DAFD0
:101F6000CD44B4B994F82C0018B901F069FB84F899
:101F70002C60E08A10B101F079FC88B1FFF7A4FC75
:101F800084F82960A168B1F1FF3F05D00123032245
:101F9000052000F073FF40B1607E012810D109E0F8
:101FA0004FF40761702001F0D9FC40F675017020F4
:101FB00001F0D4FC2069401E20F07F4000F078FE44
:101FC00094F82F0094F82F1000EB400005EBC000B0
:101FD000406801EB410155F8312001B00121BDE815
:101FE000F0401047FFF770FC4FF0FF30A06094F80E
:101FF00029008DF800009DF8000088B194F82F00AA
:1020000094F82F1000EB400005EBC000406801EB96
:10201000410155F8312001B00621BDE8F0401047DC
:1020200040F68601702001F099FCFFF74DFC84F822
:10203000286001F01BFC20B194F82C0030B109E0BD
:1020400059E040F69601702001F088FC01F0F8FAA2
:1020500084F82C6094F82D0058B12B494FF40020DF
:102060000860052000F0DEFF01F036FB002084F858
:102070002D0094F82F0094F82F1000EB400005EB92
:10208000C000406801EB410155F8312001B000214A
:10209000BDE8F040104701F07DF8E08A10B101F092
:1020A000E5FB28B119480078032808BF6677F8BD1A
:1020B00040F6A101702001F051FC154806608868C7
:1020C0000660F8BD0878BDE8F84001F017BDFFF7DD
:1020D000FBFB94F82F0094F82F1000EB400005EB69
:1020E000C000406801EB410155F8312001B00521E5
:1020F000BDE8F040104740F6B401702001F02EFC1E
:10210000800900201400002008F50140160000207E
:10211000080500402DE9F34F8246DC488BB000688B
:10212000DB4DC005C00D0ED0103840B20028B8BF3E
:1021300000F00F0000F1E020ACBF90F8000490F830
:10214000140D40090DD00C984FF0000B00780028BA
:1021500018BF012818D040F24F714FF0700001F005
:10216000FDFB95F82F004FF0010B202807D00C98AD
:10217000007848B140F24B71702001F0EFFB4FF452
:10218000E961702001F0EAFBC24C24B1002140F269
:102190005270AFF30080C0490AEB4A0001EBC00067
:1021A0004FF00108009024B1002140F25A70AFF3C3
:1021B0000080B8F1000F09D095F82E604FF00009AB
:1021C00085F82B90BBF1000F07D032E0B348002810
:1021D00018BFAFF3008062B6EEE73746012020EA71
:1021E0000706AF48402200EB871100EB861002F093
:1021F000DCFA24B1002140F2CD50AFF3008005EBB2
:10220000870105EB8600096A016224B1002140F2D2
:10221000D150AFF3008024B1002140F26470AFF3DD
:10222000008095F82B008DF804009DF8040000282C
:10223000B9D124B1002140F26E70AFF3008000F0FC
:1022400093FC8046334606AA0C99FFF769FA24B13D
:10225000002140F27570AFF30080914906A801EBB0
:10226000861717F81A10012918BF02293CD10699C0
:10227000079BA1EB08018B4A21F07F41A3EB0803E8
:1022800023F07F43022971D3B1F5800F6ED29A42B9
:102290006CD34FF0010901AB05AA3146FEF738FFB8
:1022A00000286BD09DF814109DF8042033468A4214
:1022B00068D00520FEF774FD07EB4A0148709DF8D1
:1022C0001400202803BF05EB860080F820A080F8CA
:1022D000239007EB400018BF80F801A0324651461A
:1022E0005FF00300FFF7C2FB05EB860090F82300C8
:1022F0008DF804009DF8047024B1002140F27C7038
:10230000AFF300806848002818BFAFF30080EFF3F8
:10231000108872B624B1002140F28270AFF30080C1
:1023200095F82B008DF804009DF8040000287FF438
:102330003AAF24B1002140F28A70AFF300800DF172
:10234000180E00989EE80E1000F10800B9F1000F79
:1023500080E80E1044D024B1002140F29770AFF312
:102360000080BBF1000F2CD116E0FFE7324651464A
:102370000420FFF77BFB4FF00109B5E732465146D9
:102380000420AFE7202919BF07EB4100407805EB97
:10239000860090F820008FE79FB195F82F00202845
:1023A0000FD124B1002140F29C70AFF30080314680
:1023B0000220FFF78BFB20B90C980078F0B30128BE
:1023C0004CD024B1002140F2B970AFF30080BBF1D2
:1023D000000F18BF01204AD085F82B004FF00109EB
:1023E00024B1002140F2CA70AFF30080B8F1000FB1
:1023F00045D024B1002140F2CE70AFF30080B9F196
:10240000000F11D095F82E0005EB800090F8210008
:10241000202809D024B1002140F2D570AFF300800C
:102420002248407801F06AFB24B1002140F2DA70C2
:10243000AFF300800DB04846BDE8F08FFFE724B150
:10244000002140F2A470AFF3008095F82E20514691
:102450000420FFF70BFB4FF00109C1E7002C3FF40C
:10246000A2AE002140F2AF70AFF300809BE695F87A
:102470002E10012020EA010185F82E10ACE7074854
:10248000002818BFAFF3008062B6B2E704ED00E0A9
:10249000000D002000000000800900200000000066
:1024A000800C0020FFFF3F0000000000140000200F
:1024B00010B5202811D20E4991F82E30A1F18002DA
:1024C00002EB831C1CF810303BB191F82E3002EB6C
:1024D000831212F81020012A01D0002010BD91F8BB
:1024E0002E2001460020FFF7C1FA012010BD000098
:1024F000000D002070B50D46064601F0A5F90F4805
:1025000090F82E200024803800EB821010F8141070
:1025100029B1611CCCB2202CF8D3202070BD084812
:1025200004EB440140F8316000EBC10021464560F6
:102530000120FFF79BFA204670BD0000000D00202F
:10254000800900202DE9F04F83B000F00DFB054617
:1025500000F0D6FD674CA068B0F1FF3F1CBF4FF004
:10256000FF30A060A07FDFF890B1A8B9D4E90301E3
:10257000081A0002C11700EB116000124FF40C7131
:1025800002F018F821690844281A0002C11700EB6C
:1025900011600012C00F13D0607E28B394F8290098
:1025A0008DF800009DF80000F0B100F0EBFB00BFDB
:1025B00094F82A00F0B140F24741702001F0CEF9C2
:1025C00094F82F0094F82F1000EB40000BEBC000A4
:1025D000406801EB41015BF83120082190474FF43E
:1025E0008661702001F0BAF9E81C20F07F4000F00D
:1025F000C1FADDE74FF0010A84F82AA094F82F0011
:10260000202824D094F82F80202084F82F0084F8EC
:102610003000002684F8286084F829603748266056
:102620000078022816BF032801200020207794F8A4
:102630002E7004EB870999F82000202831D000EB98
:1026400040000BEBC000817D012905D029E040F25C
:102650004A41702001F082F9AB4600F10805408A3A
:1026600001AA694600F022F994F82F00202804D02E
:102670002069401D20F07F400BE068890BF1090BB9
:1026800028B101F0F3F8002808BF0BF1320B2BF052
:102690007F40D5E90021891A2860084420F07F4056
:1026A000686039460120FFF711FA0028F9D0144874
:1026B00000EB871010F81800022804D13A46414672
:1026C0000620FFF7D3F984F82BA099F821002028E1
:1026D00003D00C48407801F011FA207F002804BF95
:1026E00003B0BDE8F08F00F055FD2677667703B0A4
:1026F000BDE8F08F000D00208009002016000020AA
:10270000800C00201400002010B5324C82B094F8E8
:102710002F10202908D0A168B1F1FF3F09D040F661
:10272000E921702001F01AF940F6E821702001F04B
:1027300015F962680146284B50189A4204D940F2B4
:102740000961702001F00AF9244A914204DD40F247
:102750000A61702001F002F9214A914204DA40F244
:102760000B61702001F0FAF81E498142DCBF00F5D0
:10277000F700A0F1F85005DD0028BCBFA0F5F70078
:1027800000F1F85001AA694600F090F89DF80400A5
:102790000F288CBF012000200099084420F07F41C1
:1027A000A16094F829008DF800009DF80000002831
:1027B00004BF02B010BD01230322052000F05EFB20
:1027C00000281CBF02B010BD40F6F121702001F0BE
:1027D000C5F80000000D0020FF7F841E0020A10727
:1027E00000E05EF80080841E70B51E4C202184F845
:1027F000201084F8211084F82210002084F823008F
:1028000084F82E0084F82F10421EA2602060A0776A
:1028100084F8280084F829002077607784F8301045
:10282000114984F82C0084F82D0008704870488005
:10283000A4F182011022887001F8040F521EFAD10F
:102840000A4D012684F82A60FF202870084801F00C
:1028500037F9687001F092F9A86000F0E3FC84F8A1
:10286000316070BD000D0020160000201400002013
:1028700029190000410B48F2376251430A0C094BF9
:10288000510202FB03020848504300F586306E30C7
:10289000400D5B4210FB03F3B2EB532F88BF491C82
:1028A00008447047F7C2FFFF6F0C0100430B48F26A
:1028B000376C03FB0CF330B41B0CDFF844C05C0234
:1028C00003FB0C030F4858434FEA505C04EB0C0029
:1028D00043F609541CFB04F404F5807C43F60855C8
:1028E000A3EB5C2C2C440CF0FF0CB3EB542F84BFF7
:1028F0004FF0000C401C086082F800C030BC7047EC
:10290000F7C2FFFF6F0C01002DE9F041364CD4F8FF
:1029100004034FF4006610F4803F4FF0E0274FF0BF
:10292000000519D031480068B0B1C4F84051C7F86B
:1029300080622F480068D4F80415401A20F07F40C8
:10294000022802D3B0F5800F06D34FF48030C4F8CC
:1029500008030420FFF7F8FAD4F8040310F4003F4A
:1029600019D024480068B0B1C4F84451C7F8806257
:1029700021480068D4F80415401A20F07F4002284E
:1029800002D3B0F5800F06D34FF40030C4F808032B
:102990000520FFF7D9FAD4F8040310F4802F08BFFC
:1029A000BDE8F08115480068002808BFBDE8F08147
:1029B000C4F84851C7F8806211480068D4F804157B
:1029C000401A20F07F40022804D3B0F5800F38BFB2
:1029D000BDE8F0814FF48020C4F80803BDE8F04161
:1029E0000620FFF7B1BA000000B0004040B100403F
:1029F00040B5004044B1004044B5004048B10040FB
:102A000048B500402DE9F041384D2878042868D0B9
:102A1000E81C0122017859B1012908BF6A7002D06F
:102A20006978002958D002210170407800F0FAFA44
:102A30002F4CD4F804034FF0000810F4002F4FF48B
:102A400080774FF0E0260AD02A48006838B103208A
:102A500000F0E8FAC6F880720320FFF775FAD4F8A0
:102A6000040310F4802F0AD02348006838B10220F4
:102A700000F0D8FAC6F880720220FFF765FAD4F8A1
:102A8000040310F4003F0AD01C48006838B101204C
:102A900000F0C8FAC6F880720120FFF755FAD4F8A2
:102AA000040310F4803F08BFBDE8F08114480068BB
:102AB000002808BFBDE8F081002000F0B3FAC6F896
:102AC000807204202870C5F80880C4F80082BDE830
:102AD000F0410020FFF738BA40F26A316C2000F074
:102AE0003DFFBDE8F0410720FFF72EBA200000208F
:102AF000008000404C8100404881004044810040FB
:102B000040810040012211024FF0E0230020C3F871
:102B1000801103F5C073BFF34F8FBFF36F8FC3F8FE
:102B200000110E4941F8042F431EC1F80433C1F8C7
:102B30003C05C1F83C010A4BC3F84005C1F840010F
:102B40001B1DC3F84005C1F844011B1DC3F8400517
:102B5000C1F84801CA6003494870704700800040CE
:102B600004800040200000200148006870470000F9
:102B700004B500402DE9F047474E0546F71E327870
:102B8000F968012A04BFA942BDE8F0874FF0404030
:102B9000424B186042486FF48023C0F8083300F1BC
:102BA00004034FF00004002A61D06FF4A02CC0F899
:102BB00048C3C3F84045C0F844413A4B1B684FF046
:102BC000E0294FF00108002B04BF4FF40063C9F85F
:102BD00080324FF48033C0F80833C0F84833C0F86F
:102BE0004041D0F80435EB1A23F07F43022B4BD33E
:102BF000B3F5800F48D2C0F840554FF48033C0F889
:102C0000443332B1D0F804258A1A22F07F42022AD6
:102C1000F8D3C7F808803C70FFF774FF2248D0F85B
:102C2000041564F30101C0F80415D0F80825022149
:102C300061F30102C0F80825D0F81025042161F3E2
:102C40000302C0F81025C0F80C80B968C0F8001263
:102C50008015C9F88002C9F800011449C005086050
:102C60000420FD60707086F80080BDE8F0876FF486
:102C7000802CC0F848C3C0F84045C0F84041C3F8B4
:102C80004045C0F8444198E70021C0F840154FF492
:102C9000FA716C2000F062FE2300002008F501406C
:102CA00000B0004048B100400080004004F5014001
:102CB00070B52C4CE268824214BF01210021DFF87C
:102CC000A8C09CF80050022D02D0002937D002E0A5
:102CD000002908BF70BD617881B3244B4FF080415B
:102CE00019608B132249C1F80833C1F84833002317
:102CF000C1F84031D1F80435C31A23F07F43022BC9
:102D000027D3B3F5800F24D2C1F840054FF48033A8
:102D1000C1F844333DB100BFD1F80435D31A23F0D4
:102D20007F43022BF8D3134B02214A071A60E0605D
:102D300004208CF801008CF8001070BD04E040F213
:102D400002216C2000F00AFE40F206216C2000F007
:102D500005FE0020C1F8400540F212216C2000F071
:102D6000FDFD0000200000202300002008F50140A8
:102D700000B0004004F501400148C0687047000001
:102D8000200000202DE9F04136496FF48020C1F881
:102D90000803354D0B1D0022287868B16FF4A02C74
:102DA000C1F848C3C3F84025C1F844212F4B1B6824
:102DB0004FF0010C9BB90CE06FF4802CC1F848C3B4
:102DC000C1F84025C1F84021C3F84025C1F844218D
:102DD000ECE74FF0E0244FF40063C4F8803202289F
:102DE00004D040F21E216C2000F0B8FDD1F804059B
:102DF0001F4CC01C20F07F40E3681E4E98420CD050
:102E0000D1F80475DF1B27F07F47042F05D3B7F5F2
:102E1000800F02D2FFF7AEFE1FE0D1F80405181AAA
:102E200020F07F40022815D3B0F5800F12D212494E
:102E30004FF080400860C4F808C02270C6F804C093
:102E4000C6F80CC04000091F08600420687085F8AF
:102E500000C002E0C4F808C02270A068C6F80002F2
:102E6000BDE8F08100B000402300002048B10040E0
:102E7000200000200080004008F501402DE9F047C7
:102E8000DFF890C1002601279CF800409CF801C0A3
:102E90004FF4A07507287BD2DFE800F00404040497
:102EA0006C6C6C00DFF87081D8F80C90B9F1807F01
:102EB00004BF98F80180B8F1000F02D0022C05D0B1
:102EC0002CE040F251216C2000F048FDACF10408E8
:102ED00008F0FF0805EB880505F1804808F5304843
:102EE0000025012C02D0022C0BD014E0BCF1040F01
:102EF00024BFD8F80090B9F1000F08BF4FF000458B
:102F000009E0BCF1040F24BFD8F80090B9F1000F1C
:102F100008BF45F0804515F0804FE1D13F4C00F1EE
:102F2000100C07FA0CFCC4F808C304EB8005C2B10E
:102F30004FF0400808EB800808F0FF08A044C8F8EC
:102F4000007004EB8000D0F84005A1EB000020F0F9
:102F50007F40824298BFB0F5800F28BFC5F840651A
:102F600050D2C5F84015012B08BFC4F804C3012096
:102F7000BDE8F08734B1844504D14FF41D716C2055
:102F800000F0ECFCA0F1040C0CF0FF04012B00E0BD
:102F90003BE00CBF4FF001084FF00008032C04D3B6
:102FA00040F24D116C2000F0D9FCDFF874C004F140
:102FB000100307FA03F3CCF80833CCF8483305EBD9
:102FC00084044CF80460001FC0B20CEB80006AB1AE
:102FD000DCF804450C1B24F07F44A24298BFB4F5F2
:102FE000800F24BF0021C0F840150BD2C0F8401557
:102FF000B8F1000F18BFCCF80433CCF844330120EB
:10300000BDE8F0870020BDE8F08740F279216C2010
:1030100000F0A4FC230000202000002000800040DD
:1030200000B000402DE9F84300264FF4A0774FF0A0
:103030000108072851D2DFE800F00404040419193C
:10304000190000F1100108FA01F22649C1F808231D
:1030500001EB80030022C3F8402507EB80028E506D
:10306000214951F820000090BDE8F8831F4D011F51
:10307000CCB2297879B16A7882420CD11C4A4FF0DF
:1030800040401060012908BFFFF73CFD2E70194930
:103090004FF08070C86004F1100008FA00F1164883
:1030A000C0F80813C0F84813A1000144D1F8401536
:1030B000D0F80425891A21F07F41022907D300EBBB
:1030C00084020021C2F8401507EB840146500B48EA
:1030D00050F824000090BDE8F88340F2F1216C2004
:1030E00000F03CFC008000404081004023000020B4
:1030F00008F501402000002000B0004040B1004031
:1031000020496FF48020C1F808031F480A1D037886
:1031100000205BB16FF4A023C1F84833C2F840052A
:10312000C1F844011949096899B90CE06FF480238A
:10313000C1F84833C1F84005C1F84001C2F8400564
:10314000C1F84401EEE74FF0E0224FF40061C2F80D
:1031500080120F494FF0FF32C1F80823C1F8400533
:10316000C1F840010A1DC2F84005C1F84401121D12
:10317000C2F84005C1F84801121DC2F84005C1F867
:103180004C01704700B000402300002048B10040CF
:1031900000800040084890F902000028B8BF70473E
:1031A00000F01F01012202FA01F14009800000F144
:1031B000E020C0F8001270472000002010B507285A
:1031C0000DD2DFE800F004040404060606000649F8
:1031D00002E0001F0549C0B201EB800010BD40F2C3
:1031E0009D216C2000F0BAFB4081004040B10040BE
:1031F00010B507280DD2DFE800F004040404060629
:103200000600064902E0001F0549C0B201EB80003C
:1032100010BD40F29D216C2000F0A0FB40810040D9
:1032200040B1004010B51C48002404210470C01EA9
:1032300001708905C160FFF765FC4FF0E0234FF492
:1032400000624FF0010CC3F88021BFF34F8FBFF332
:103250006F8FC3F880221148C0F804C0C0F808C0BE
:10326000D0F804150029FBD1491EC0F80813C0F896
:103270004813C0F84045C0F840410949C1F84045ED
:10328000C0F84441091DC1F84045C0F84841C3F8A1
:103290000021C0F800C010BD2300002000B0004095
:1032A00004B000402DE9F041164C607A002827D088
:1032B0004FF480718D05284601F0A0F980464FF447
:1032C0008271284601F09AF900260746B8F1000FEE
:1032D00009D00120C5F80803207920B12671E069E2
:1032E00008B18047E66137B1C5F804610220C5F82E
:1032F000080300F067FA4046BDE8F04100F05AB814
:10330000BDE8F0813000002010B501F021FA30B99D
:1033100001F035FA18B901F03EFA002802D002494E
:103320000220086010BD0000340C004070B500F0B1
:1033300087F900F09BFA094C4FF0804530B1FFF758
:10334000E3FF012028610420A07204E00320A072A2
:103350000120C5F804030020E07170BD300000209A
:1033600070B5134CA079F0B1012803D0E179401E6B
:10337000814218DA00F07AFA054600F05FFBA17985
:10338000012902D9E179491CE1710DB1616900E0BF
:103390002169411A022902DA11F1020F07DC0DB18D
:1033A000606100E02061BDE87040FFF7BFBF70BD05
:1033B000300000202DE9F04706464FF080454FF4DD
:1033C0008671284601F01AF980464FF48871284624
:1033D00001F014F9274C8246277804F1080001F027
:1033E00081F910B14FF4D57116E04FF0010946B1E3
:1033F000A07A032805D10420A072FFF785FFC5F845
:1034000010900026B8F1000F18D0C5F80C61A07A12
:10341000042804D04FF4DE716D2000F09FFA01F013
:1034200097F928B901F0ABF910B901F0B4F908B176
:10343000114806600220A07200F0E6F8BAF1000F11
:1034400008D0C5F81061A07A022801D1FFF788FFE3
:10345000C5F814903FB12670A07A022801D1FFF779
:1034600065FF00F0D1F8BDE8F0470248083001F0F0
:1034700050B9000030000020340C00402DE9F04726
:103480005C4C4FF000080646C4F8188043788278F8
:103490000078E07263710127A271BD0784F807808C
:1034A000052824D2DFE800F00F03051F2100A761E3
:1034B00009E000F0C5F80121284601F0A4F8002831
:1034C000F9D00220A06101F0CAF8B0B100F0E8F92B
:1034D000217E01F0030188420FD1B07950B1022062
:1034E000C5F804036AE04448ECE74448EAE740F2E0
:1034F0002D3149E000F0A8F960E0EF604FF4827AE6
:10350000C5F80481A069C5F8180501F00DF940B9A6
:1035100001F014F928B901F028F910B901F02FF9D8
:1035200038B14FF080513648D1F84412C1F34231DE
:10353000016001F0F9F840B901F000F928B901F093
:1035400014F910B901F01BF910B12D4810300760C3
:10355000AF600220C5F80403B07978BBD5F8040346
:1035600010F0020F0ED0DFF89C90D9F80010C9437C
:1035700041F30017D9F8001041F01001C9F800100C
:103580007F1C07E040F2EE216D2000F0E7F900BF5C
:1035900000F00AFB5146284601F030F80028F7D029
:1035A00000F052F92FB9D9F8001021F01001C9F834
:1035B00000100220C5F80803C5F80481A07970B195
:1035C000307860B900F052F9064600F037FA6FF033
:1035D000004216B1C4E9042001E0C4E9040201215B
:1035E000284601F010F808B100F03AF984F80A8092
:1035F000BDE8F08730000020010002000100030058
:103600003C05004010ED00E010B5EFF3108472B6F9
:103610000A48417829B14178491E4170417829B161
:1036200008E040F20D116D2000F098F9807808B99B
:1036300000F02AF9002C00D162B610BD3000002045
:1036400010B5EFF3108472B606484178491C4170FA
:103650004078012801D100F0EDFF002C00D162B6C6
:1036600010BD000030000020054810B5C17821B120
:1036700000210171C170FFF7C7FF002010BD0000DD
:103680003000002070B50C4CE17861B90125E5707F
:10369000E061FFF7D5FF00F0E9F830B1E06910B163
:1036A00080470020E061002070BD4FF08040257110
:1036B000C0F80453F7E7000030000020EFF310805B
:1036C00072B604498A78521C8A70002800D162B60A
:1036D000704700003000002010B5EFF3108472B680
:1036E0000A48817829B18178491E8170417829B1D1
:1036F00008E040F225116D2000F030F9807808B91B
:1037000000F0C2F8002C00D162B610BD30000020DD
:103710002DE9F04104006FF015003CD02178042918
:1037200039D80029617838D0002934D1A17800290E
:1037300031D1002000F02DFF002000F01DFF4FF0E0
:1037400080484FF0FF31C8F808130026C8F8006120
:10375000C8F80461C8F80C61C8F81061144F7E7095
:10376000A088B88100F05DFF012508B1FD707D7073
:103770000121404600F047FF08B100F071F82046F3
:10378000FFF77CFE7D72002000F0F6FE4FF0E02196
:103790003046C1F80051BDE8F0810029FBD0202956
:1037A000F9D8A1782129F6D80129C2D1F3E7000080
:1037B000300000200248807A002800D001207047A5
:1037C00030000020F8B51F4DE87A00280FD1287E80
:1037D00000F0030000F033FF002808D0EFF3108161
:1037E00072B6FFF7E7FF18B1002900D162B6F8BD45
:1037F0000126AE7201B962B618204FF08044C4F8B9
:103800000803A6614FF42070ADF80000BDF8000079
:10381000411EADF80010F9D20027C4F80C71C4F8AD
:1038200010710848083000F070FF2F70FFF77EFD20
:103830006661687900F07F00C4F838051820C4F884
:103840000403F8BD3000002010B5044C207E00F0C9
:10385000030000F0F4FE0028F8D010BD3000002076
:1038600001490120087070476C0000204FF0804033
:10387000D0F8000118B903480078002800D00120D2
:10388000704700006C0000204FF080400121416033
:103890000021C0F800110148017070476C00002041
:1038A0000248006800F00300704700001C0400405C
:1038B00010B531B1012907D040F2023105A000F066
:1038C00021F8D0F8140401E0D0F8080400F0010059
:1038D00010BD00006E72665F636C6F636B2E6800D4
:1038E000BFF34F8F05480168054A01F4E0611143B9
:1038F0000160BFF34F8F00BFFDE700000CED00E05B
:103900000400FA0572B6034A526802B19047FFF705
:10391000E7FF000050000020064810B500210160BC
:1039200001210160084600F0B1FEBDE81040012011
:1039300000F09FBEFC1F0040074810B50121416008
:10394000891EC0F808130C2000F0A0FEBDE810404E
:103950000C2000F08EBE000000C000400EB572B614
:103960000F4A5568D5B1002203466E460A2403E08B
:10397000B0FBF4F0521CD2B20028F9D1B05409E0E7
:10398000B3FBF4F004FB1030B3FBF4F3521ED2B2DD
:103990003030B054002AF3D13046A847FFF7A0FFDB
:1039A0005000002070B5174C06460D46607810B1E7
:1039B0004FF0FF3070BD06B9134E62602570FFF7FF
:1039C000ABFFFFF7B9FF3046FFF7A2FE0600F1D1CB
:1039D000FEF70AFFFFF7F6FE00F030FD284600F084
:1039E00048FE0120002D09DB05F01F0100FA01F15E
:1039F0006A09920002F1E022C2F8001160703046BC
:103A000070BD000050000020AE4600000148407824
:103A10007047000050000020074890F9000000287F
:103A200009DB00F01F02012191404009800000F1F4
:103A3000E020C0F800127047500000202DE9F0414E
:103A400001264FF0E02231034FF000084046C2F853
:103A50008011BFF34F8FBFF36F8F164CC4F8000176
:103A60000C2000F032FE144D2868C04340F30017CC
:103A7000286840F010002860C4F8046326607F1CAA
:103A800002E000BF00F090F8D4F800010028F9D05F
:103A90001FB9286820F01000286008480568666093
:103AA000C4F80863C4F800810C2000F00EFE28461C
:103AB000BDE8F08100C0004010ED00E008C5004006
:103AC00010B5024605200C4904E000BF01EBC0031D
:103AD0001B7933B1401EC0B2F8D248216920FFF7EC
:103AE0003DFF41F8302001EBC00100224A718A718C
:103AF00001220A7110BD0000340D002010B5052808
:103B000001D3582106E00A4901EBC00001790129DF
:103B100003D059216920FFF721FF41798279491C9F
:103B2000C9B28A4200D04171BDE81040FFF774BFAE
:103B3000340D002070B505250E4E0F4C16E021788F
:103B400006EBC1000279012A08D1427983799A42B1
:103B500004D04279827156F8310080472078401CA9
:103B6000C0B22070052801D3002020706D1EEDB278
:103B7000E5D270BD340D00206D00002000B500F0CE
:103B8000D3FD40B900F0DAFD28B900F0EEFD10B920
:103B900000F0F5FD08B1024800BD024800BD00007C
:103BA0000C05004000E7014010B500F0E8FD30B31F
:103BB000EFF31080C8B1002172B6124802680368A2
:103BC000C2F3001243F0100303604FF0E023D3F878
:103BD0000042D3F804321C4300D040BF20BF00BFD6
:103BE00000BF00BF00BF12B105E00121E4E7026899
:103BF00022F010020260002900D062B610BD20BF82
:103C000010BD000010ED00E001490968896808470F
:103C10005800002001490968096908475800002038
:103C200001480068406800475800002001490968C1
:103C30000968084758000020734900006B490000DC
:103C40005F4900006F49000067490000094810B54E
:103C50008178042908D010290AD0202908D040F200
:103C6000BF116B20FFF77AFE1021817023F050F80E
:103C700010BD00005C0000200B4810B5017831B188
:103C8000EFF3108472B68178102905D008E040F275
:103C90000D316B20FFF762FE08218170FEF752FCA8
:103CA000002C00D162B610BD5C00002070B5124C33
:103CB000207858B1EFF3108572B6607948B10228C8
:103CC00009D040F2D6216B20FFF748FE40F2C32115
:103CD000F9E7012003E0A1780020042901D06071F8
:103CE00002E0607123F008F805B962B6E078BDE83B
:103CF0007040FFF703BF00005C0000200E4810B5C5
:103D0000017859B1EFF3108172B642794AB1012AB4
:103D100009D040F2FE216B20FFF720FE40F2EE2199
:103D2000F9E7022200E00022427101B962B6C078D0
:103D3000BDE81040FFF7E2BE5C00002010B5134C58
:103D4000207810B140F27F211DE00020607001203A
:103D5000A0700F484FF4C851016005210181B721BF
:103D600041810C4941600C48FFF7AAFEE070002138
:103D70000A48FEF7BFFB2071202802D001202070E6
:103D800010BD40F28E216B20FFF7E8FD5C000020A3
:103D90006C0D0020FF1FA107C93E0000FD3D000083
:103DA00012488178042901D0002070478079B8B189
:103DB0000F48D0F804050E49091DD1F84015401CE4
:103DC000081A0002C11700EB11600012002800DC85
:103DD00000200849A0FB0110420442EAD13070479C
:103DE000054801684089081A704700005C000020FF
:103DF00000B0004040420F006C0D002070B52F4E07
:103E0000D6F8040500252E4C082931D2DFE801F050
:103E100030043A3A211C4B400121022000F0FCF80A
:103E2000607858B10420A07026480068A060A57191
:103E3000607902283ED022F05FFF3BE02020A07096
:103E4000BDE87040FEF77EBB40F207216B20FFF714
:103E500085FD607800280BD0A078042809D04FF0A9
:103E6000E0210220C1F88001BFF34F8FBFF36F8FB5
:103E700070BD00F071F810B1D6F84401B0B915F07A
:103E80008DFC70BD0121022004E00120A07070BDF6
:103E90000121282000F0C0F860780028F5D0BDE8A6
:103EA000704000F095B800F057F818B1BDE87040C8
:103EB000FFF7CCBEBDE8704000F056B800B000403F
:103EC0005C0000206C0D002070B5EFF3108472B61A
:103ED000204D002069796871C1B3012906D00229FB
:103EE00018D084F310884FF4D07128E084F3108840
:103EF000687810B140F24D1121E00021142000F04B
:103F00008BF801206870A878012821D1BDE87040A5
:103F100000F05EB8697849B16870A878082815D0B3
:103F200007DC022812D0042807D10BE04FF4AF7150
:103F300005E0102806D0202808D04FF4BD716B2072
:103F4000FFF70CFD2020A870FEF7FCFA84F3108820
:103F500070BD00005C00002002488079012800D07C
:103F6000002070475C00002070B50420FDF73CFF86
:103F7000154D2968814200D8084606460421FDF700
:103F800071FE124C012130B1012818D04FF4A071FC
:103F90006B20FFF7E3FC2868B042A06806D1FEF76B
:103FA000B3FB2868A1680844A06070BD3044A060DD
:103FB000A1716989401ABDE87040FEF7A5BBA171E7
:103FC0006889A168081AF6E76C0D00205C000020E3
:103FD0000F4810B50021016001228160027001814B
:103FE0000421817200F110010A6842604968C160D1
:103FF00008480221817006490079FEF78BF80028F5
:1040000004D14FF482716B20FFF7A8FC10BD0000B3
:104010005C0D00205C0000200B4A10B5927812B1B4
:10402000531E1A4201D0DE2109E021B10240900660
:1040300008D1E32103E08243900603D1E7216B20FE
:10404000FFF78CFC10BD00005C000020D34900008D
:10405000EF490000DD490000E9490000D7490000B0
:10406000D1490000CF490000F5490000E3490000B4
:10407000C9490000C1490000C5490000BB49000012
:1040800001480068006B004768000020014A126880
:10409000526A1047680000200149096849690847C9
:1040A00068000020014800680068004768000020A0
:1040B000014800680069004768000020014A126852
:1040C000926810476800002001480068C0680047F7
:1040D00068000020014A12685268104768000020FA
:1040E00001480078704700006E00002070472DE9FD
:1040F000F0410D0004464FF002064FF0010708D0D2
:104100002878D0B1012807D0022814D003283BD149
:1041100016E080F820700EE06868C82803D30421F8
:10412000FDF7A0FD08B1002607E02046696800F011
:104130002AF9012601E0FCF7C5FD3046BDE8F08113
:1041400020780028F7D16868FCF78EFDE0B1696837
:10415000087828B1A078052807D040F2791110E03E
:10416000204600F018F96770E5E7204600F02BF9CB
:10417000E07804F10C0100F00AF80028DBD140F2ED
:104180007B116A20FFF7EAFB84F82070D3E7FDF784
:10419000C1BF2DE9F0410D4604000BD02679002760
:1041A0000220092D7BD2DFE805F008102E2E5B647B
:1041B0007C97860040F29311E2E0A07804286FD04B
:1041C0000328FCD04FF4CF71DAE0A078042804D0A3
:1041D000032802D04FF4D171D2E00520A07084F8FA
:1041E0002070207880BB0021204600F0CCF8207B96
:1041F000012804D0A069E0610021A26841E0E078D4
:10420000FDF76EFEF7E7A178042904D0032902D058
:104210004FF4E071B4E0227822B12146304600F03C
:10422000EEF8A4E0042900D00120A070A268022DBD
:104230000BD006213046904700286BD0007800282C
:1042400068D04FF4ED719BE031E005213046904796
:10425000002871D0007800286ED040F2D5118FE090
:10426000A078052802D040F2E11189E00221A2687D
:1042700007E0A078052802D040F2E71180E0A268AC
:1042800001213046904701462046FFF730FF0228C3
:104290006DD0F0B3012864D040F2272170E05DE0DA
:1042A00067E0A078052802D040F2ED1168E0BDE893
:1042B000F041FCF707BDA078052802D04FF4F97152
:1042C0005EE0A2680A213046904701462046FFF78B
:1042D0000EFF40F2F51153E0A178052906D062786F
:1042E0000AB1032902D040F2F91149E0217829B13D
:1042F00021463046BDE8F04100F081B894F8201026
:1043000089B184F82070A070A268082130469047D7
:1043100001E029E02BE000280ED0007800280BD027
:1043200040F205212CE0617859B1E07804F10C01EC
:10433000FFF72DFF10B16770BDE8F08140F2092151
:104340001EE0A070A2680721304690470028F3D0F5
:1043500000780028F0D040F2112111E040F216213F
:104360000EE00421A2688CE70321A26889E7002DF2
:10437000E2D100F0EFF800680028DDD040F23121F2
:104380006A20FFF7EBFA0246037B006908441061DC
:104390005938FEF7B9B9012202730022C2750A79B1
:1043A0006AB1002282824A795AB1042282758A68EF
:1043B0006A320261C96881610321817070472B22D2
:1043C000F0E70322F2E710B5044600202073E07501
:1043D000087980B10020A082487970B10420A075CE
:1043E000C8686A3020618968E069FDF747FDA0610F
:1043F0000420A07010BD2B20EDE70320EFE770B57F
:1044000005460C46C878FEF753F878B1204600F010
:1044100010F8A268092128469047002808D00078A3
:10442000002805D0DB216A20FFF798FAD721FAE7A8
:1044300070BD0021817001704170704770B5FCF74C
:104440009BFC0546002406E02046FCF79BFCFFF79A
:10445000F0FF641CE4B2AC42F6D370BD2DE9F0412C
:104460000D46FCF78FFC040007D0A0786FF0220601
:10447000012806D0022810D103E06FF00100BDE84A
:10448000F0816FF0150755B12846FCF7EDFB30B110
:10449000287830B1A078022808D03046EFE73846B7
:1044A000EDE729462046FFF776FF03E02946204640
:1044B000FFF789FFE07804F10C01FFF768FE08B10F
:1044C0000020DCE74FF42B716A20FFF747FA10B5A4
:1044D0000446FCF757FC010004D008786FF0220274
:1044E00068B902E06FF0010010BD887838B1022889
:1044F00007D0012805D001200870002010BD10460B
:1045000010BD2046FFF77BFFF7E72DE9F0410E468F
:104510000746FCF731FC054600240AE02046FCF77C
:1045200031FC807818B14FF0FF30BDE8F081641C99
:10453000E4B2AC42F2D3082E02D96FF01500F4E7D2
:1045400017B13146384601E000210846BDE8F04188
:10455000FCF7FEBB0020FEF731BE410A43F60952CC
:104560005143C0F3080010FB02F000F5807001EB2E
:1045700050207047FDF7C8BC002809DB00F01F027F
:10458000012191404009800000F1E020C0F8801234
:10459000704700280DDB00F01F0201219140400907
:1045A000800000F1E020C0F88011BFF34F8FBFF30F
:1045B0006F8F704770B50246002000291DD0A2FB06
:1045C0000101400A40EAC150490A401C41F1000182
:1045D00040F2A172831841F100015B1C41F100041B
:1045E0000021D3F1FF33A14103D271216D20FFF7E8
:1045F000B5F900F5F460B0FBF2F070BD405800284A
:1046000000D001207047D0F80C24D0F80C0402F040
:104610000102C00303D58A4201D101207047002066
:10462000704710B501218807FFF742F9002800D034
:10463000012010BD4FF080400121016070474FF014
:104640008041D1F81824D1F8181402F00302C903EC
:1046500003D5824201D1012070470020704710B578
:1046600000214FF08040FFF723F9002800D00120FF
:1046700010BD002809DB00F01F0201219140400914
:10468000800000F1E020C0F88012704700280DDBA8
:1046900000F01F02012191404009800000F1E0205C
:1046A000C0F88011BFF34F8FBFF36F8F70470010BA
:1046B0000200FA0000002357622423318F5774EE62
:1046C000D12F88C09445F7A2F936002809DB00F005
:1046D0001F02012191404009800000F1E020C0F854
:1046E00080127047EFF3108172B60278012A01D070
:1046F000012200E000220123037001B962B60AB171
:10470000002070476FF022007047002101700846BA
:104710007047EFF3108172B60022027001B962B6E1
:1047200000207047FFF706BA4FF08050D0F83001F4
:104730000F2801D000207047012070474FF08050B3
:10474000D0F830010A2801D00020704701207047BE
:1047500000B5FFF7F3FF20B14FF08050D0F83401DF
:1047600008B1002000BD012000BD4FF08050D0F8FE
:1047700030010E2801D000207047012070474FF013
:104780008050D0F83001062803D0401C01D0002012
:104790007047012070474FF08050D0F83001082852
:1047A00001D00020704701207047F0B480EA010C6E
:1047B00003461CF0030F3CD113F0030F0BD0002A6B
:1047C00004BFF0BC704711F801CB03F801CB521EB7
:1047D00013F0030FF3D1032A4FD9B2F1004F4CD29B
:1047E000C2F1000C4FEAEC740CEB947C4FEAAC0C79
:1047F000CCF1000CBCF1000F1BDD0D1F1C1F1CF0C9
:10480000010F03D055F8046F44F8046F5FEA6C069B
:1048100007D06F68676055F8087F44F8087F761EF8
:10482000F7D101EB8C0103EB8C03CCF1000C02EB14
:104830008C02002A04BFF0BC7047B2F1004F26D2B0
:10484000002ADCBFF0BC7047491E5B1E12F0010F4E
:1048500003D011F801CF03F801CF521004BFF0BC10
:10486000704791F801C083F801C011F802CF03F836
:1048700002CF521EF5D1F0BC7047042AD9D351F8AB
:1048800004CB121F43F804CB042AF8D2D1E711F865
:1048900001CB03F801CB521EF9D1F0BC704770B4C4
:1048A000034601F0FF0C10F0030F09D0002A04BFEB
:1048B00070BC704703F801CB521E13F0030FF5D103
:1048C000C9B241EA012141EA0145032A39D9B2F1CD
:1048D000004F36D25142CC1701EB947189104E42F1
:1048E000002E11DD191F16F0010F18BF41F8045FEB
:1048F000741004D04D6041F8085F641EFAD1714213
:1049000003EB860302EB8102002A04BF70BC7047F0
:10491000B2F1004F1DD2002ADCBF70BC7047591E97
:1049200012F0010F18BF01F801CF521004BF70BC84
:10493000704781F801C001F802CF521EF9D170BC56
:104940007047042AE0D3121F43F8045B042AFAD20A
:10495000DAE703F801CB521EFBD170BC7047072188
:104960000170002070470020704700207047002031
:10497000704708B1002070476FF01500704700B510
:104980000346FFF70DFA984201D9012000BD00202F
:1049900000BD08B50B380A460F2801D9372106E0BB
:1049A000C1B26B460420FCF745F918B140216420E0
:1049B000FEF7D4FF9DF9000008BD4FF0FF307047AF
:1049C00000207047002070474FF0FF30704770475D
:1049D0007047002070474FF0FF3070474FF0FF30B6
:1049E00070470021017070474FF0FF3070474FF063
:1049F000FF307047002070472DE9F04D164690B00B
:104A000005460F46002209A930464CF0BEFC099B22
:104A10001B78A3B1DFF82081002458F8041B30462E
:104A20004CF087FD60B10134392CF6D12846404A5C
:104A3000334601214BF0FBFD6FF0850028E0044672
:104A4000BB680AAA1B69A1B23846984700281FDB39
:104A50000B98FBF7A7FC34A3D3E90023FBF736FE42
:104A600006460A980F46FBF79DFC02460B46304669
:104A70003946FBF74BFB382C82468B460BDDCDE9E4
:104A800000AB2C4A2346082128464BF0D0FD0020DD
:104A900010B0BDE8F08D284B53F8248024F00403B7
:104AA000032B0CD00B2C0AD0CDE902AB234ACDF856
:104AB00000802346082128464BF0B9FDE7E70F9810
:104AC000FBF770FC18A3D3E90023FBF7FFFD0646B4
:104AD0000E980F46FBF766FC02460B4630463946F9
:104AE000FBF714FBCDE906010D98FBF75BFC0EA369
:104AF000D3E90023FBF7EAFD06460C980F46FBF7C7
:104B000051FC02460B4630463946FBF7FFFACDE929
:104B100002ABCDE904010A4ACDF800802346082102
:104B200028464BF084FDB2E70000000080842E414F
:104B30003AD70500CBD6050080010020EAD6050053
:104B400006D705000A4B10B5196801310029196014
:104B500001F001010446B8BF494203200AF066FF94
:104B600021460448BDE8104007220BF0CDBE00BF2F
:104B700060250020454B000001400B0703D502488B
:104B800000210BF09FBE7047B94B000010B50446E2
:104B900028B10146BDE8104006480BF093BEFF2146
:104BA00004480BF0EFFE21460320BDE810400AF058
:104BB0003DBF00BF454B00001FB52149214A0B688E
:104BC000528803F007030C465ABB022B08D91E4932
:104BD0001E48611A8908890141F003014BF03FF931
:104BE000402018F031FA4342C8B12268520714D06D
:104BF000154A0093A41A184618F03CF9A408144B5F
:104C00000293A4018B2344F0010401900393114803
:104C10002346042269464BF080F90BF035FF04B0BF
:104C200010BD022B08D9084B0B48C91A8908890105
:104C300041F003014BF013F918F01AFAEFE700BF47
:104C4000E806002014590020E80600204CB70500B3
:104C500060B7050090B70500A7B7050070B586B02E
:104C6000002301A90446019353F027FC0646204681
:104C700053F038F80221054620464EF059F9032E2C
:104C800025D1244A136803F00703ADB9022B0AD9D2
:104C9000214B2248D21A019B92089201197942F0C5
:104CA00003024BF0EBF8002031F04CF814B1204631
:104CB00033F0EEFA06B070BD002BF4D0164B184856
:104CC000D21A9208920142F001022946E9E72046F1
:104CD0000BF044F842420028E8D00E4B196849070F
:104CE00014D00D4D02925D1B104618F0C3F8AD08AC
:104CF0000C4B0493AD01D52345F0010503900593BA
:104D000009482B46042202A94BF007F90BF0BCFE20
:104D1000CCE700BFE8060020E8060020BCB705008D
:104D2000DAB7050060B7050090B7050010B5284C4C
:104D3000236803F00703022B08D926492648611A85
:104D40008908890141F003014BF089F823480AF0F2
:104D5000A9FD014658B123685A0708D01D4A2048CA
:104D6000A21A9208920142F001024BF087F80AF071
:104D70003FFD014658B123685B0708D0154A194822
:104D8000A21A9208920142F001024BF077F81648FD
:104D900022F006FC154B40F203421A80402000220C
:104DA0005A801AF081FA124BC0F80730236803F0DA
:104DB0000703022B0AD907490E48611A890889019D
:104DC000BDE8104041F003014BF049B810BD00BFF1
:104DD000E8060020E8060020FFB70500794B000038
:104DE00021B805003FB80500FE030020145900203B
:104DF0008D4B00005AB80500436803F00303022BF3
:104E000070B504460E46816010D0032B04D0012BF0
:104E10000FD10025284601E00568002000236360CB
:104E200010B1314621F0D2FA284670BD0068002545
:104E3000F4E70549054845224AF0CEFB02484521E2
:104E40004AF0A4FE0025E8E77FB80500A2B80500F7
:104E50000B6801330B60014B1B681847AC00002046
:104E6000014B1860704700BFAC00002007B50B462F
:104E7000002102460191034801A900F081FC03B022
:104E80005DF804FB514E000030B585B0CDE901015D
:104E90000446002501A90548039500F071FCDDE9F1
:104EA00002309842B8BF255405B030BDB3F50400B8
:104EB0002DE9F04F2DED028BB0F81C9083B019F066
:104EC000080F044601921FD001290CBF49F01009B8
:104ED00049F02009A0F81C9004F114001EF04EF8CF
:104EE00040B99C499C48AC224AF076FB9948AC21D9
:104EF0004AF04CFE019B83F31188BFF36F8F03B020
:104F0000BDEC028BBDE8F08F944FDFF84C82DFF8E8
:104F100044A209F00709022906D120464AF091FB74
:104F20000028D9D0012869D1D4F818B0A38BBBF1DF
:104F3000000F1CDA00262568009623F00703C4E959
:104F4000006643F00103A383A38B03F007024A45E5
:104F500008EE102A03D0A268002A40F001811DB992
:104F6000009A002A00F041814FF00009FAE003F0B6
:104F70000702511F012923D8002123F00703062A25
:104F800025689BB2C4E900110CD18D422A4638BF76
:104F90000A462AB1E18B12680131E183002AF8D177
:104FA00043F00203A38320464AF04BFB002800F0A5
:104FB000CC80A38B43F02003A38300230093C3E79B
:104FC000042A0FD123F007039AB2A28320464AF0A5
:104FD00038FB002800F0BB8042F02002A2830025AD
:104FE0000095B1E73946404640F21B124AF0F4FA08
:104FF00040F21B1138464AF0C9FDF0E7032832D1D0
:10500000B9F1000F0AD0394640464FF4AB724AF06E
:10501000E3FA4FF4AB7138464AF0B8FD236853B950
:105020003946404640F257124AF0D6FA40F257113C
:1050300038464AF0ABFD23691B68009353B93946E3
:1050400040464FF4AD724AF0C7FA4FF4AD7138469E
:105050004AF09CFDA38B23F0070343F00603A383D0
:105060000025AB4670E704282FD1B9F1020F0AD012
:105070003946404640F25D124AF0AEFA40F25D1108
:1050800038464AF083FDE38B53B1394640464FF42E
:10509000AF724AF0A1FA4FF4AF7138464AF076FD8C
:1050A00023695B68009353B93946404640F2611268
:1050B0004AF092FA40F2611138464AF067FDA38B3C
:1050C00023F0070343F00403C9E705282FD1B9F102
:1050D000010F0AD0394640464FF4B2724AF07CFACA
:1050E0004FF4B27138464AF051FD236853B939463E
:1050F000404640F265124AF06FFA40F265113846B8
:105100004AF044FD23699B68009353B939464046F1
:105110004FF4B4724AF060FA4FF4B47138464AF072
:1051200035FDA38B23F0070343F0050397E740F217
:105130006B12394640464AF04FFA002540F26B1197
:1051400038464AF023FD00958BE70090FCE60546C3
:1051500046E700BFDCB80500A2B80500BAB80500F4
:105160004FF0010943F00803A38304F11403184628
:1051700008EE903A1DF002FF40B951464046AC227D
:105180004AF02AFAAC2150464AF000FD019B83F315
:105190001188BFF36F8FB9F1000F35D1002D49D1C0
:1051A000009B13B12C49204698474FF04003EFF382
:1051B000118B83F31288BFF36F8F18EE900ACDF82E
:1051C00004B01DF0CDFE40B95146404681224AF060
:1051D00003FA812150464AF0D9FC18EE900A1DF0DE
:1051E000DDFEA38B23F00803A383A38BDA062AD565
:1051F00023F01003A3830121B4F81C9009F00709E0
:1052000000297FF488AE67E6A1680029C6D00B6844
:10521000002B38BF002399464B6818EE102A1E4613
:1052200020465B46B047B9F1000FB7D0D9F800303F
:105230004946EDE7294618EE102A5B4620462D68C0
:105240004AF01BFAAAE713F020011EBF23F0200347
:10525000A3830221D0E700BF5D520000F8B50446E9
:105260000D4600F114064FF04003EFF3118783F36E
:105270001288BFF36F8F30461DF072FE40B90A49A5
:105280000A4881224AF0A8F9074881214AF07EFCA9
:1052900030461DF083FEA5613A4620460121BDE857
:1052A000F840FFF705BE00BFDCB80500A2B8050056
:1052B0002DE9F04704460F464AF0F5F9051E54DB88
:1052C00004F114094FF04003EFF3118A83F31288BD
:1052D000BFF36F8F48461DF043FE40B93349344851
:1052E00081224AF079F9314881214AF04FFC484641
:1052F0001DF054FEE38BA28B4FF6FF718B4202F040
:1053000007064AD0022E1FD10133E38335464FF002
:10531000010848461DF032FE40B924492448AC2219
:105320004AF05AF92148AC214AF030FC8AF311883E
:10533000BFF36F8FB8F1000F17D000233246394604
:1053400020464AF09AF910E0930701D0062E0FD1BB
:1053500000233B606368EBB9C4E900773546F6B9D2
:10536000524602212046FFF7A3FD2846BDE8F087FC
:10537000052E17D0012E0AD00E490D4840F2C91251
:105380004AF02AF90B4840F2C9114AF0FFFB6FF0CE
:10539000040504E01F606760E0E76FF00A054FF066
:1053A0000008B6E76FF08505F9E700BFDCB8050037
:1053B000A2B80500BAB8050070B5044600F114059E
:1053C0004FF04003EFF3118683F31288BFF36F8F22
:1053D00028461DF0C5FD40B92249234881224AF0E4
:1053E000FBF8204881214AF0D1FB28461DF0D6FD6C
:1053F000A38B03F00703022B17D0012B0CBF6FF018
:1054000004046FF0850428461DF0B8FD40B9154925
:105410001548AC224AF0E0F81248AC214AF0B6FB3D
:1054200086F31188BFF36F8F17E0E38B53B90F49F1
:105430000D484FF4F8724AF0CFF80C484FF4F87169
:105440004AF0A4FBE38B013B9BB2E3833BB92046CC
:1054500032460221FFF72CFD0224204670BD0224B3
:10546000D1E700BFDCB80500A2B80500BAB8050056
:105470002DE9F0410E460546002848D0002946D0C7
:1054800000F114074FF04003EFF3118883F3128803
:10549000BFF36F8F38461DF063FD40B91D491E48AC
:1054A00081224AF099F81B4881214AF06FFB384667
:1054B0001DF074FD31462846AC8B4AF0A7F818B3AE
:1054C00004F00704231F022B0AD91449124840F2A2
:1054D0002E224AF081F8114840F22E214AF056FB64
:1054E00038461DF04BFD40B90A490B48AC224AF042
:1054F00073F80848AC214AF049FB88F31188BFF3E0
:105500006F8F2046BDE8F0816FF07704E8E76FF019
:105510001504F6E7DCB80500A2B80500BAB8050026
:1055200070B579B305680C1F641BE60824F0070406
:105530002C44A378DB0708D413491448A3224AF06B
:105540004BF81148A3214AF021FB314628464AF086
:10555000D6F8304435F83030C01A864208D00A49AF
:105560000A48AB224AF038F80748AB214AF00EFB54
:10557000638823F00103638031462846BDE870400C
:105580004AF07CB970BD00BF02B90500A2B80500A1
:105590004B422DE9F04703EA010731EA03030668AD
:1055A00014461BD0042F3D46B94628BF0425CF1B07
:1055B00007F1FF3A1AEA070F0AD03249324840F29F
:1055C00027124AF009F82F4840F227114AF0DEFA74
:1055D0007CB94FF000094846BDE8F087042904D89B
:1055E000BDE8F04711464AF07BB94FF000090425A9
:1055F000DEE7B368B3EBD40FEBD904F10B01394408
:10560000491BC90830464AF0D2F880460028E0D04D
:1056100009F1040505EBC005354455447F422F4090
:10562000A7EB09094C44A9F1040307349B1B24F0A0
:105630000704A41BB0EBD30F4FEAD3074FEAE404EF
:1056400008D201463A4630464AF0FEF84146304616
:105650004AF05AF8394630464AF051F83844844204
:1056600008D23946304622464AF0EEF82146304606
:105670004AF04AF806EBC706738843F001037380CB
:10568000A9E700BF02B90500A2B80500B2F5802F56
:105690002DE9F04180460E4615465ED3364937481F
:1056A00040F2A51249F098FF40F2A51132484AF0A5
:1056B0006DFA043DF41D354424F0070425F0070578
:1056C0002D1B172D4FEAD5070AD82B492B4840F23E
:1056D000B51249F081FF284840F2B5114AF056FA58
:1056E000C8F80040B7FA87F8C8F124084FEA8808DC
:1056F00008F107060023F608E360731CBB42A760AD
:105700000AD91D491D4840F2C51249F065FF1A48E3
:1057100040F2C5114AF03AFA04F11002A044002305
:10572000904525D1720042F00102628004EBC6016F
:10573000BA1B500023804880611924F8366004EBBE
:10574000C7074B8062537B8843F001037B8031465F
:105750002046BDE8F04149F0D7BF042AA9D8064940
:1057600006484FF4D67249F037FF4FF4D6719DE7E3
:1057700042F8043BD4E700BF02B90500A2B8050017
:105780002DE9F04FA5B08846039091461C460025B0
:1057900099F8000010B9284600F015BE09F1010380
:1057A0002528099307D04146039B98470028C0F25B
:1057B0000A86013545E21822002116A84BF006FFA3
:1057C00099F80130252B79D0002209981646964683
:1057D00017469446014610F8013B2B2B00F09E80A3
:1057E00000F29580202B00F09B80232B00F09B8003
:1057F000BCF1000F05D09DF8600040F004008DF86A
:1058000060002FB19DF8600040F008008DF8600046
:10581000BEF1000F05D09DF8600040F010008DF83B
:1058200060002EB19DF8600040F020008DF860000F
:105830002AB19DF8602042F040028DF860209DF86A
:10584000602002F04400442803D16FF386128DF8E3
:1058500060209DF860202A2B42F080028DF86020A5
:105860007CD19DF8612042F001024B1C8DF8612033
:105870001A782E2A9DF861200CBF0121002161F3C6
:1058800041028DF8612075D15A782A2A6BD00133F4
:1058900000210A26184610F8012BA2F13007092F23
:1058A00040F2AA809DF860201A91C2F3400040EABD
:1058B000D17161F341028DF860205BE009F10202D1
:1058C00009928DF863309DF86130DE0740F16F81F9
:1058D00054F8042B0892002A08DA9DF8602042F060
:1058E00004028DF86020089A52420892580740F14D
:1058F000668154F8047B002F80F265819DF8613049
:105900006FF341038DF861304FF0FF375BE12D2BD2
:105910000BD0302B7FF46CAF01225BE7012759E7F6
:105920004FF0010E56E7012654E74FF0010C51E706
:105930000CFB0202303A33461E4616F8010BA0F16A
:105940003007092FF4D9994292D09DF8601019922E
:10595000D20F62F341018DF8601089E70B460022F7
:105960004FF00A0CE8E79DF8612042F004028DF840
:1059700061200233194611F8012B6C2A5CD040D803
:10598000682A46D06A2A61D04C2A67D019460B464D
:1059900013F8012B0993782A8DF8632000F2DF8039
:1059A000572A68D8412A04D0A2F14503022B00F2FD
:1059B000D6809DF8623002F0DF020421A2F1410A94
:1059C00061F30203DAF100029DF861108DF8623094
:1059D00042EB0A0262F3C7110A068DF86110CBB2DE
:1059E00000F1E38003F07802182A40F0B5806FF3ED
:1059F000C6038DF861309CE006FB01213039034677
:105A000048E7742A26D07A2AC0D19DF86130062250
:105A10000DE05A78682A9DF8612006D1012161F3D2
:105A2000C6028DF86120991CB1E71346022262F389
:105A3000C6038DF86130AAE75A786C2A9DF8612078
:105A400001D10421EBE713460322F0E79DF8613012
:105A50000522ECE79DF861300722E8E7BDF86030E9
:105A600023F4F04323F0020343F4804343F00203A2
:105A7000ADF860308BE7A2F15803202B6FD801A15D
:105A800051F823F0375B00005F5B00005F5B0000B4
:105A90005F5B00005F5B00005F5B00005F5B00001E
:105AA0005F5B00005F5B0000B35900005F5B0000BC
:105AB000375B0000095B0000B3590000B3590000D8
:105AC000B35900005F5B0000095B00005F5B0000F2
:105AD0005F5B00005F5B00005F5B00006D5B0000D0
:105AE000375B00008D5B00005F5B00005F5B0000C8
:105AF0008D5B00005F5B0000375B00005F5B0000B8
:105B00005F5B0000375B00009DF86230012161F3AC
:105B100002038DF862309DF8613003F07803402B6A
:105B200002BF9DF8601041F001018DF86010632AFA
:105B300005D0002306E09DF862300221E7E7003B34
:105B400018BF01239DF86020C2F340010B4363F3AB
:105B500041028DF86020B6E613F0380FE9D09DF8C9
:105B6000603043F001038DF86030E2E79DF8623069
:105B7000032262F302038DF862309DF8613003F076
:105B80007803A3F140077B427B41DBE79DF862305D
:105B9000032262F302038DF862309DF8613013F046
:105BA000780F14BF01230023CCE70123CAE79DF936
:105BB0006020002AB4BF199A4FF0FF3295E699078A
:105BC0007FF5A2AE1A9F0023CDE919339DF862300C
:105BD00003F00703042B09D19DF861309A0705D41F
:105BE0009DF96130002BB4BF0D2706279DF8623068
:105BF0009DF8611003F00703012BC1F3C30136D1F7
:105C0000CB1E042B20D8DFE803F00307071F1F007B
:105C100054F8042BD31704E0073424F00704F4E805
:105C20000223CDE916239DF86060B30755D0099B88
:105C300003984A46414649F000FF0028C0F2C3835A
:105C40000544DDF82490A3E554F8042B01294FEA1C
:105C5000E273CDE9162305D19DF858301693002341
:105C60001793E0E70229DED1BDF95820D2E7022BD5
:105C700023D1CB1E042B13D8DFE803F0030A0A124A
:105C80001200226816920023201D17930446CAE7CB
:105C9000073424F00700F0E80223CDE91623F5E7E6
:105CA00054F8043B169301294FF000031793D3D007
:105CB0000229B8D1BDF85830D0E7042B07D10734FA
:105CC00024F00704F4E80223CDE91623ABE7032B05
:105CD00004BF54F8043B1693A5E79DF86390B9F10F
:105CE000780FAED8B9F1570F00F2A680B9F1250FA1
:105CF00000F0EC80B9F1240FA3D9B9F1410F03D022
:105D0000A9F14503022B9CD8DDE91623002A73F183
:105D10000001C0F2D381310700F1D28116F01006E4
:105D200018BF2026C3F30A5BC3F31303069207933D
:105D3000DDE90623CDE91223BBF1000F40F0C2815B
:105D4000DDE90632134314BF4FF0010C4FF0000C95
:105D50000799CB020699CA0243EA515358464BEAC7
:105D600002010C91C11719430D91DDE90C01B9F144
:105D7000460F08BF4FF066090143CDE9122300F03A
:105D80001482BCF1000F40F0D481129B0493139B4A
:105D900043F000430593DDE90423CDE912230023FA
:105DA000ABF2FE3B1A4605211BF1020FC0F2CA817D
:105DB0001BB1DDE90401CDE91201BBF1000FDDE902
:105DC000123100F3DA811399129BCBF104000BF12D
:105DD0001C0B01FA0BFBA0F1200CC34021FA0CFCB8
:105DE00043EA0B0343EA0C03C140CDE9123109F049
:105DF000DF03472B40F0E081D01C02DB974280F2AA
:105E0000D781A9F10209002F5FFA89F900DD013F6E
:105E10009DF86030990600F1CF81002FD4BF002398
:105E20000123B9F1660F0E9340F0C881BB1840F111
:105E3000C6814FF0000AC6E1A9F15803202B3FF6B6
:105E400000AF01A252F823F05D600000435C000047
:105E5000435C0000435C0000435C0000435C0000C6
:105E6000435C0000435C0000435C0000095D0000EF
:105E7000435C0000F95E0000FD5F0000095D00006A
:105E8000095D0000095D0000435C0000FD5F00004B
:105E9000435C0000435C0000435C0000435C000086
:105EA000936000005D60000061600000435C0000E2
:105EB000435C0000D35E0000435C00005D600000B6
:105EC000435C0000435C00005D60000041464846C2
:105ED0006AE4002FDDF858900ADB394648464BF05B
:105EE0001FFB09EB000A0026B9F1000F0CD1A8E650
:105EF00048464BF00EFBF4E7169B8DF874300026F5
:105F00000DF1750A0DF17409AAEB090206B101320F
:105F10009DF86200C30640F14B8202321999089B3A
:105F200040060A4444BF1A995218002B25DD9B1ADB
:105F30009DF860205107C2F3800B00F14B82570699
:105F400040F14482002E00F0438208934146039BB7
:105F5000304698470028C0F23682089B01355E46DD
:105F60003027089303EB050B089BABEB0305002BD5
:105F700003F1FF33089300F31F823EB1039B4146B8
:105F8000304698470028C0F21E8201359DF86220F5
:105F9000560640F17D829DF96120002AC0F21C82E4
:105FA000A5EB090599F80000A0F13002092A4F4637
:105FB00005EB090B09F1010940F23E829DF86220D0
:105FC000199E900608D406EB0B09002EA9EB060BD0
:105FD00006F1FF3600F3378238782E280BD1039B69
:105FE000414698470028C0F2EE81002E0BF1010BCC
:105FF00000F331820137ABEB070B37E230072BD4CC
:1060000016F0100618BF2026DDE91623002A73F1CA
:10601000000105DA524263EB4303CDE916232D2636
:106020000DF18D030093DDE916011DAB18AA49F0AF
:10603000B9FC8146002F0DF18D030BDB9DF860103C
:10604000A3EB09026FF3861197428DF8601001D916
:10605000BF1A19979A4647E72B26D5E70026DFE7B0
:106060001698002800F09E810DF18D03009318AA68
:106070001DAB002149F096FCBDF8623003F0EF0340
:1060800043F4F04343F010038146ADF8623000263C
:10609000D0E7169B07293FF6D4ADDFE801F00D04E9
:1060A000060D08080D0D1D70CBE51D80C9E52846BD
:1060B000E917C3E90001C4E51D60C2E52D2631E6FC
:1060C0002B262FE640F2FF739B452DD1DDE90623F9
:1060D0001343A9F1410918D1B9F1190F95BF44F63D
:1060E000496346F66963ADF87430ADF8743094BF17
:1060F000462366238DF876309DF860306FF3861363
:106100008DF860300DF1770AFCE6B9F1190F95BFF3
:1061100044F24E1346F26E13ADF87430ADF874309D
:1061200094BF4E236E23E5E74FF0000C10E60BF111
:10613000FF3B92185B41002A73F10001F7DACDE9C9
:10614000122322E6049B05985B0843EAC0734008CB
:10615000B0F1333FDC46CDE904300BF1010BF1D255
:10616000A3FB01ABCDE904AB059B4843C3180593E2
:106170000CF1020B013A012316E6023341F1000152
:1061800012A8CDE912310E9249F0D5FB0E9ADDE945
:1061900012010BF1FF3B013200184941002871F157
:1061A00000030BF1FF3BF7DA05E6002293460AE60F
:1061B000BF1A4FF066092BE6002332E67B1C102B3A
:1061C000A8BF10239A461021119100204FF00061C2
:1061D000CDE914010AF1FF3ABAF1FF3FDDE91410ED
:1061E0001FD1129BCB180A93139B40EB03030B9315
:1061F000DDE90AAB6FF070414FF0FF30594508BF41
:1062000050451AD350465946CDE91201B9F1660FEF
:1062100053D1002A20DC30238DF874300DF1750A3B
:106220002BE0490841EAC0714008CDE9141014A8D8
:106230000F9249F080FB0F9ACCE70A9B0F920B9AC2
:106240005B0843EAC273510812A8CDE9123149F044
:1062500072FB0F9A0132D9E70DF1740A11990029E6
:1062600009DD11A912A80F9249F085FB0F9A0AF8CF
:10627000010B013AF2D1199200229DF860108806B4
:1062800001D4002F3FDD53462E2103F8011B92B1AC
:10629000002F75DD5142B942A8BF39469DF8620012
:1062A00019910029A7EB0107D4BF0021012161F357
:1062B00045108DF862009A4620E011A912A80F92AD
:1062C00049F059FB0F9A9DF860308DF87400302822
:1062D00018BF02F1FF32990601D4002F52DD2E23A0
:1062E0008DF875300DF17603E5E711A912A80F922C
:1062F00049F041FB0F9A0AF8010B013F002F02DD24
:1063000011990029F1DC0E9B002B3ED11A9709F060
:10631000DF01452922D1002A5046BABF52422D2121
:106320002B21632A00F8029B8AF801100ADD6427FA
:1063300092FBF7F101F1300C0AF103008AF802C078
:1063400007FB11220A27824692FBF7F107FB112275
:1063500001F1300C30320AF802CB4270199A002A4F
:106360001EDC1A9A002AD4BF002201229DF8621076
:1063700062F3861100228DF862108AF80020C1E5D0
:106380009A46C0E70DF1750ABDE700211A91504603
:106390001AF8011D3029FAD02E2918BF8246B6E717
:1063A0000122E3E7DFF838A10646AAF10509ABE5CB
:1063B000070748BF0132B1E5039B4146384698477D
:1063C0000028BFF6D1AD25B0BDE8F08F2027C8E585
:1063D0003027C6E50893D0E5A5EB090B4E460BEB3D
:1063E000090519F8010B702820D11A9A02EB05094A
:1063F000A9EB0502002A43DC534632460398414686
:1064000049F01BFB0028DEDB089B284403440546BB
:106410009A46AAEB0503002B7FF713AC039B41467A
:10642000202098470028CEDB0135F2E7039B414648
:1064300098470028D2DAC6E7039B414698470028D0
:10644000BFF6B0ADBFE7039B414630209847002818
:10645000BFF6BBADB7E7039B414630209847013EEE
:10646000C0E5039B414698470028ACDB3E460BEB5A
:10647000070517F8010BA0F13002092AF1D9B4E79A
:10648000039B41463020984700289CDB0135AFE74D
:10649000D10601D4120706D5039B41463020984708
:1064A000002890DB01359DF86220D30607D59DF8C2
:1064B0006300039B41469847002884DB0135199E01
:1064C0002E44721B002A02DC53464A4696E7039B81
:1064D0004146302098470028FFF675AF0135F0E7B8
:1064E00028B905002DE9F34180460E4615460027E0
:1064F0002A4601A9404649F0CCFA314604460246F4
:1065000001984BF058F82D1B2744264401D0002C4D
:10651000EED13946404649F0D8FA40B1064907481D
:10652000E82249F059F80448E82149F02FFB3846A1
:1065300002B0BDE8F08100BF29B90500A2B805008E
:106540002DE9F34180460D4616460027324601A943
:10655000404649F0D4FA04462DB102460199284636
:106560004BF029F82544361B274401D0002CEDD1EF
:106570003946404649F0EEFA50B10749074840F223
:10658000351249F029F8044840F2351149F0FEFA75
:10659000384602B0BDE8F08129B90500A2B805006F
:1065A00008B54FF04002EFF3118382F31288BFF376
:1065B0006F8F04F0F5FE034849F00EF803F0F8FE83
:1065C000FCE700BF51B9050030B51049104889B04B
:1065D000002250F0BCF80F4D0F4900220023CDE9F6
:1065E000062300240E23CDE90334CDE901440B4BEF
:1065F00000944FF4407228461CF00EFE08492846CD
:106600001CF064FC204609B030BD00BF25660000C8
:1066100080140020B814002080C90020DD6A00002A
:106620000DBE050001481DF0A5BA00BF800800207E
:106630002029F8B505460C4608D913491348872286
:1066400048F0CAFF1048872149F0A0FA002003460D
:106650000246012715F8011B09B1A34200D3F8BD7A
:10666000252902D182F00102F4E7002AF2D041F09C
:106670002006613E192EEDD8732904BF07FA03F2F4
:10668000104301330022E5E77AB90500A2B80500FE
:106690000E4A08B5002313700D4A13600D4B0E4AC5
:1066A0001A604FF4004000F0EBFE00F0D9FB0B48FD
:1066B00049F0AFFB18230A490A484FF4BC724FF067
:1066C00011FFBDE8084000F099BA00BF5159002001
:1066D00068250020B000002057FE0400702500202F
:1066E0002007012078250020194B1A4A9B1A9F2B5E
:1066F00070B54FEA23160AD91749184840F24A22C2
:1067000048F06AFF144840F24A2149F03FFABFF3CB
:106710005B8F134B53E8005F6A1C43E8002100299C
:10672000F8D1BFF35B8F15B90A4CB54200DB70BDE1
:10673000237B53B123689B690BB12046984763685C
:1067400004221968204600F049FB01351034ECE7BB
:10675000A0A3050080A305007AB90500A2B8050032
:106760006C25002010B54FF04003EFF3118483F344
:106770001288BFF36F8F044849F05BFB84F31188E4
:10678000BFF36F8F10BD00BF7025002010B5044C03
:10679000227812B903481DF0EDF90123237010BDD2
:1067A00050590020800800200C4BBFF35B8F53E84A
:1067B000002F013243E800210029F8D1BFF35B8F9D
:1067C000BFF35B8F064B53E8002F013A43E80021EB
:1067D0000029F8D1BFF35B8F704700BF6825002008
:1067E000642500200020064BBFF35B8F024653E870
:1067F000000F43E800210029F9D1BFF35B8F7047F8
:1068000068250020F8B5FFF7EDFF0B4C0B4D2D1B55
:1068100007462D110026AE4200DBF8BD204649F0A8
:106820000EFB28B123681B6913B1394620469847EF
:1068300001361034EFE700BF80A30500A0A30500D8
:10684000174B984237B5044602D3164B984221D3D2
:1068500015480022002301A91CF08CFA0546E0B976
:106860000122019BBFF35B8F53E8001F43E8002028
:106870000028F9D1BFF35B8F0198214640F27112D5
:1068800004304AF025FE019C7E2384F8753184F89B
:1068900076510434204603B030BD044CFAE700BF03
:1068A000C8A005009029060078250020A7B905009A
:1068B00050B1064B984206D303F50D5398422CBFB6
:1068C0000020012070470020704700BF20070120F2
:1068D000464B1B782DE9F047054603B9A0B1FFF7F9
:1068E00041FF044618B195B1204649F0A8FB2DB9E7
:1068F0003F4B1B68002B01DDFFF784FF3D4849F04B
:1069000096FA051E18BF01252846BDE8F0873A4BC8
:10691000BFF35B8F53E8002F013A43E800210029C1
:10692000F8D1BFF35B8F354B1B78A3B9237ADB0714
:1069300011D449F097FB0646204649F05EFB01461C
:106940003046FFF775FEDFF8C890DFF8C8A0DFF823
:10695000C880064636B92A4E2A4B9B1B4FEA23189D
:10696000002740E0B6FA86F7C7F11F0739462046F0
:1069700049F046FB4845024602D3234B984213D3C5
:106980001046FFF795FF78B952450DD06189C1F3E4
:10699000891100F051F91D484146D82248F01CFEEB
:1069A000D821404649F0F2F8012303FA07F726EA16
:1069B0000706CFE7304649F042FA90B1A17A6289E2
:1069C00001F007090123C2F38912C1F3C201304665
:1069D00000F040F9814504D8336821465B683046B1
:1069E0009847013710364745E4DB7DE750590020D2
:1069F00068250020702500206425002051590020C2
:106A000080A30500A0A3050090290600A2B80500F8
:106A1000C8A00500A7B905007AB90500284B37B50D
:106A20001B68418104469847E0604FF04003EFF354
:106A3000118583F31288BFF36F8F2248214649F0F6
:106A4000ECF985F31188BFF36F8FBFF35B8F1E4B9B
:106A500053E8002F511C43E800100028F8D1BFF381
:106A60005B8F1A4B1B7883B14FF04003EFF3118417
:106A700083F31288BFF36F8F0020FFF729FF84F3A1
:106A80001188BFF36F8F03B030BD114B1B68002B13
:106A9000F9D052B900220023CDE900230D484FF46C
:106AA000004200231FF032F9EDE70A2AEBD1094832
:106AB0004FF059FE084803B0BDE830401DF05AB809
:106AC000B0000020702500206425002051590020CE
:106AD000982500208014002080080020164B174ABB
:106AE0009B1A002B10B50ADC1549164840F2F142FA
:106AF00048F072FD124840F2F14149F047F8FFF7C3
:106B0000F3FD1EF09DFC104B186030B10F4B1B685D
:106B1000092B02DD0E481DF02DF80D4C0020FFF76B
:106B2000D7FE0028FAD14FF0FF324FF0FF33204656
:106B30001DF05CF8F2E700BFA0A3050080A30500EC
:106B40007AB90500A2B80500982500206425002028
:106B500080080020F8B50F4F3D7875B90E4C0F4EE8
:106B6000FFF7C2FD361B3611B54207DB0020FFF7E9
:106B7000AFFE0028FAD101233B70F8BD204649F052
:106B80005EF918B1236820465B69984701351034D7
:106B9000EAE700BF5159002080A30500A0A305002B
:106BA00007B504380190BFF35B8F50E8003F5A1ED1
:106BB00040E800210029F8D1BFF35B8F012B03D1FE
:106BC000034801A91CF030F903B05DF804FB00BFD5
:106BD0007825002010B5044640B906490648DF2252
:106BE00048F0FAFC0348DF2148F0D0FF63681879C9
:106BF00010BD00BFC5B90500A2B805000B480C4B7D
:106C000030B51B1A0B4CDB0800210430994200D12F
:106C100030BD10F83120256802F0070225F0070585
:106C20002A4344F8042B0131F0E700BF98A2050085
:106C300080A30500E8060020044A054B9B1AB1EB2F
:106C4000D30F34BF52F831000020704798A20500DE
:106C500080A30500F8B51546144C154A121B42F3E3
:106C6000CF02AA4206461F4608DC12491248BC223F
:106C700048F0B2FC0F48BC2148F088FF7FB1002DDE
:106C800011DB0E4B304653F82540FFF7A3FF00B24F
:106C900000EB400024FA00F000F00700F8BD04EB20
:106CA000C5010879FAE70420F8E700BF98A20500BB
:106CB00080A30500F6B90500A2B80500E80600208B
:106CC0002DE9F04715469846314A324BD21A42F325
:106CD000CF02AA420446894608DC2F492F48572292
:106CE00048F07AFC2C48572148F050FFB4B92C4B9F
:106CF0002C4FFF1A3F1126469A46BC4202DB304613
:106D0000BDE8F0870AEB041043462A464946FFF7E0
:106D1000D7FF864238BF06460134EEE72A46494689
:106D200000232046FFF796FF404528BF4046064611
:106D30002046FFF74FFF1C4F00B2072300EB400037
:106D400003FA00F057F8253023EA000347F825300E
:106D50002046FFF73FFF00B257F8252006F0070155
:106D600000EB400301FA03F313430021032223FA4B
:106D700002F000F00700814202F1030238BF014631
:106D80001E2AF4D123F007030B4347F82530B6E75A
:106D900080A3050098A20500F6B90500A2B8050079
:106DA00080A30500A0A30500E8060020F8B5094C63
:106DB000094BE41A06460F46E4080025A54200D117
:106DC000F8BD00212AB23B463046FFF779FF013576
:106DD000F4E700BF80A3050098A20500F8B5104CA9
:106DE000041B2411013405460E461746E4B240B98F
:106DF0000C490D48D12248F0EFFB0A48D12148F058
:106E0000C5FE6B6839461C712846FFF7CFFF6B68DB
:106E100001221E605A71BDE8F840FFF7B7BC00BF01
:106E200080A30500C5B90500A2B8050010B5044649
:106E300050B90949094840F20F1248F0CDFB064805
:106E400040F20F1148F0A2FE6368002120465971FC
:106E5000BDE81040FFF7AABFC5B90500A2B80500FC
:106E60002023024902481A464FF03CBB602A012009
:106E70009C25002037B50023094D01930120FFF721
:106E800027FD0446FFF790FC0022002301A92846B5
:106E90001BF070FF08B1002CF0D1019803B030BD99
:106EA0009C25002007B500230193074800220023FA
:106EB00001A91BF05FFF10B1FFF7DCFF0190019803
:106EC00003B05DF804FB00BF9C250020F0B5037AF9
:106ED000457A85B02D090190D8071CD4DDB1002476
:106EE00026460198314649F08BF80746FFF7E0FC4B
:106EF00070B134B9019B29461869FFF799FB044624
:106F000048B124FA06F3D90702D53846FFF748FE00
:106F10000136AE42E5D3019B1A7A920704D55B692C
:106F2000084C0393039B2BB9064801A91BF07CFF77
:106F300005B0F0BD1D6803A920461BF075FF039541
:106F4000F0E700BF9C2500200E2A2DE9F84F81466E
:106F5000884615460AD92D492D4840F23B1248F083
:106F60003BFB2A4840F23B1148F010FEFFF79AFF26
:106F7000044630B301230027032D4360078109D95C
:106F800002220281A5F1020A00F1140B4761BAF155
:106F9000000F0EDC637AC4F8109065F30713032D1D
:106FA000637218D8AA00414604F114004AF003FBAA
:106FB00007E0FFF777FF064630B92046FFF786FF68
:106FC00034462046BDE8F88FCBF80000AAF1070A46
:106FD00007608346DBE74146082204F11800676931
:106FE0004AF0E9FA023D08F10808072D2E4628BFAD
:106FF00007264FEA86094146381D4A464AF0DBFA21
:10700000AD1B3F68C844F0D1DBE700BF23BA0500E1
:10701000A2B80500024BD868DB69C01A704700BFF0
:107020009C250020014BD869704700BF9C2500209B
:107030000EB403B503AB014653F8042B0448019387
:10704000FEF79EFB02B05DF804EB03B0704700BF93
:10705000B17200002DE9F04F87B01F4601F0010327
:1070600005929DF84090BDF948A0049306468846D5
:1070700001F0020B01F0080548F05AFF0246002813
:1070800044D039493046FFF7D3FF0446BBF1000F27
:1070900008D018F0440F3BD134493A463046FFF748
:1070A000C7FF0444049B53B1314B324953F82920A4
:1070B000314B3046002A08BF1A46FFF7B9FF3DB1F1
:1070C0002E4B2F4953F829203046FFF7B1FF0546D4
:1070D000BAF1000F16DB059B002B43D0012303FA06
:1070E00009F9284B284F19F0100F18BF1F465146B9
:1070F0009DF84400FFF7A0FD394602463046FFF7F1
:1071000097FF0544281907B0BDE8F08F0446BDE796
:107110001E4B18680028C4D01D4B4FF4616C1968D1
:10712000B7FBF1F7B7FBF0F100FB1177B1FBFCF215
:107130000CFB121C4FF47A714F434FF03C0EB7FB1F
:10714000F0F800FB18774F43BCFBFEF30EFB13C1B6
:10715000B7FBF0F00091CDE901800E493046FFF712
:1071600067FF9EE7084FC2E75DBA050061BA0500F8
:1071700028A5050018C105004FBA05003CA505006B
:1071800086BA050059BA050054BA0500BC2500208E
:10719000C02500206ABA050038B50C46E10705464F
:1071A00003D5084A0849FFF743FFE20608D4A306BF
:1071B00028464CBF05490649BDE83840FFF738BFAF
:1071C00038BD00BF4FBA050018C10500CEBF05008D
:1071D000AABB05002DE9F0471D46089B1746DA06B5
:1071E00004460E4605D499064CBF2A492A49FFF7A2
:1071F0001FFFDFF8AC904FF00008A8452ADBDFF84E
:10720000A480DFF8A490DFF898A00025BD422FD21B
:10721000725D49462046FFF70BFF0135102D20D146
:107220001E49DFF87C80DFF884902046FFF700FFDE
:107230000025AF4228D9725DA2F120035F2B28BF41
:107240002E2249462046FFF7F3FE0135102D14D1BA
:10725000BDE8F08749462046FFF7EAFE08F101083D
:10726000CBE76A07D2D151462046FFF7E1FECDE7D2
:1072700041462046FFF7DCFECFE76B07D9D14146F8
:107280002046FFF7D5FED4E741462046FFF7D0FE63
:10729000DBE700BFCEBF0500AABB050092BA050020
:1072A000300C06002E0C06008CBA0500C8C605007E
:1072B00038B54B681A68CB689A4205460C4602D12D
:1072C000084649F042F86368BFF35B8F53E8002F2C
:1072D000511C43E800100028F8D1BFF35B8FA3686E
:1072E0009D5463681A68E3689A4208D905490648BC
:1072F000742248F071F90348742148F047FC0020DB
:1073000038BD00BF94BA0500A2B805002DE9F047CA
:107310008B7A13F0070716468AB00A7A04460D46A0
:1073200020D04989C3F3C203C1F38911D243CDE907
:1073300000730291EB6802F001023146FFF78AFE0A
:1073400081462B7ADB4313F001080DD021462846F5
:1073500048F09EFE002F3BD03A4631462046FFF7CC
:107360001BFF35E0B946ECE7002F37D1E36853B98E
:1073700029492A484FF4E87248F02EF926484FF47C
:10738000E87148F003FC0026E368069306AA33463A
:10739000A168284648F068FE069A63681A604AB1F8
:1073A000A368134413F8018CA8F10A03D3F1000871
:1073B00048EB0308204648F0C8FF069B1E44002BFC
:1073C000E2D1B8F1000F03D015492046FFF730FE97
:1073D000204648F0BAFF0AB0BDE8F087284648F0DA
:1073E00041FE104902462046FFF722FE4FF0100AE8
:1073F00005AA434606A92846CDF814A048F034FE55
:10740000059A002AA8D04B46009606A92046FFF709
:10741000E1FE059B9844EBE794BA0500A2B805008D
:10742000C3BA050018C1050073B542F20F738B4251
:1074300028BF0B4605680F4A04460521684648F0F8
:10744000D8F863680C495B6806460B22284648F06A
:1074500012FE63683246694628465B6848F00BFEB8
:10746000636806495B681B22284648F004FE02B0A8
:1074700070BD00BF22DF050001BB0500E5BA0500B5
:10748000084A10B50123084C13600021A04204D81B
:1074900001B11360054B186010BD40085B0001216D
:1074A000F4E700BFC025002040420F00BC250020AB
:1074B00000230428CB604B6098BF044B044A98BF5C
:1074C00053F820308A600B60704700BF90A505001C
:1074D0006CA505000023084A0B60CB604B608A60F6
:1074E000064B074AD21AB0EB221F3EBF03EB001037
:1074F00083680B60704700BFE4A6050080A3050009
:10750000A0A3050038B50446FFF784FD0546FFF744
:1075100089FD094A03460821204649F088F82B4690
:107520002046064A082149F082F82046044A0821EC
:1075300049F07DF8002038BD0DBB05001EBB0500DD
:107540002FBB05002DE9F347114C124D124FDFF808
:107550004C80DFF84C902D1B82462D110026AE4248
:1075600003DB002002B0BDE8F0876268537912792E
:10757000002B14BF3B464346CDE900320821A368E7
:107580004A46504649F053F801361034E7E700BF49
:1075900080A30500A0A305007BBB050083BB0500FD
:1075A0008CBB050010B50023054ACB600C464B6030
:1075B0008A6001461846FFF73FFB206010BD00BF00
:1075C0006CA505002DE9F04F2A4B2B4EF61A85B01D
:1075D0000446F6080D4651B92849294840F21D12C3
:1075E00047F0FAFF254840F21D1148F0CFFA6B68CA
:1075F0005B7923B9234A0321204649F018F8224B2E
:10760000224ADFF890A0DFF890B00821204649F028
:107610000EF81F4A0821204649F009F84FF00008EB
:107620000FFA88F7B74208F1010803D3002005B02C
:10763000BDE8F08F3A46012300212846FFF70AFBF8
:1076400000233A46194681462846FFF703FB394690
:1076500003900020FFF7F0FA039A5AF822200192D3
:107660005AF82920009203465A460821204648F03D
:10767000DEFFD5E798A2050080A30500C5B9050087
:10768000A2B80500ADBB0500BFBB0500CBBB050024
:10769000E9BB05007CA5050026BC050010B5044625
:1076A00050B90749074840F20F1247F095FF0448C8
:1076B00040F20F1148F06AFA636800225A7110BD57
:1076C000C5B90500A2B8050038B50D46044650B945
:1076D000074908484FF4817247F07EFF04484FF491
:1076E000817148F053FA636801221D605A7138BDF8
:1076F000C5B90500A2B805002DE9F04F85B00746D1
:10770000019352F8043C184C184E029318469146C7
:107710008A4649F0FEFE361B024636114FF000083D
:10772000A346B045029B07DB114A0121384648F0C9
:107730007EFF6FF0070513E0A168039218460293DD
:1077400049F003FF1034054618B1039A08F1010807
:10775000E7E7019C4B4652460BEB08113846A04721
:10776000284605B0BDE8F08F80A30500A0A3050062
:107770003ABC050008B5024BFFF7BEFF002008BD6C
:10778000C5750000014BFFF7B7BF00BF65030500DB
:10779000014BFFF7B1BF00BF71030500014BFFF7BD
:1077A000ABBF00BFA5780000014BFFF7A5BF00BF2E
:1077B000F903050010B5C369DB681C792CB9044ACC
:1077C000012148F034FF204610BD0120FCE700BF36
:1077D0004FBC05002DE9F04F2C4E1F462C4BF61ADE
:1077E000151E85B04FEAD60614BF2B4633460293CA
:1077F0004B685B79804689461BB9264A032148F0CD
:1078000016FFDFF89CA00024029B9C4202DB05B01F
:10781000BDE8F08FBDB357F824B000239E4207D1D6
:1078200057F824301C4A0121404648F000FF23E06D
:10783000194600200393FFF7FFF94022594649F00B
:1078400084FE039BD0B91A4600210E9B12B2484613
:10785000FFF736FA0E9B834283460DD085B9214649
:107860002846FFF7E9F903465AF82B200092032136
:107870000A4A404648F0DBFE0134C5E70133CDE754
:1078800057F82430F0E72246DEE700BF80A305006A
:1078900098A2050073BC05009EBC050088BC0500CD
:1078A0007CA505002DE9F74FD3F804B0DFF850A010
:1078B0000646884691461D4600275AF8041B0422B6
:1078C000584649F042FE044670B10137052FF4D105
:1078D0006B680A4A0121304648F0A9FE6FF00704A0
:1078E000204603B0BDE8F08F009705F10803A9F129
:1078F000020241463046FFF76DFFF1E7B8BC0500D4
:107900007CA50500014B01221A70704762590020C6
:10791000024B034801221A7048F017BD635900203A
:1079200010A705000148FFF77FBD00BF10A70500A5
:1079300010B508460C4648F053FB054821460F2277
:10794000FFF7E4FC2046BDE8104048F078BB00BFDC
:1079500010A70500054B1B781BB141F288304EF093
:10796000C9BEA42000211DF01FBD00BF6359002027
:107970002DE9F84FDFF89490DFF894A080460F4689
:107980000424CB4699F80050CDB94FF0FF334FF0A7
:10799000FF3250461BF094FE3A464146284615F009
:1079A000F5F9064650461BF063FF174DFEB1012363
:1079B0002B709BF800306BB93846BDE8F88F3A461B
:1079C0004146002015F0E2F90646EEE75CB92C705E
:1079D0004FF0FF34002015F025FA0028ECD02B786A
:1079E000002BF3D1E8E7013CFFF7B4FFF2E72B7877
:1079F00013B1013C04D12C702B78002BC2D1DBE7F2
:107A0000FFF7A8FFF8E700BF625900206359002084
:107A1000F007002013B504461BF0C4FCC0F3072395
:107A20000193C0F307430093044A030E0821204644
:107A300048F0FDFD002002B010BD00BF83BE050070
:107A40002DE9304804464EF053FE4FF47A75A0FB02
:107A500005BC05FB01CC4FEADB3242EA4C43204631
:107A6000034A082148F0E3FD0020BDE8308800BF4C
:107A70009CBE050010B5044607F03CFC084A0346CE
:107A80000821204648F0D3FD064A2046082148F048
:107A9000CEFD054821461BF089FA002010BD00BF2D
:107AA000ABBE0500CABE0500117B000030B5014623
:107AB00087B0044612481BF079FA124A002312F8E4
:107AC000011BAA2903D10133B3F5066FF7D1C3F522
:107AD00006604FF4066100256422CDE90230019171
:107AE000094B009542432046B2FBF1F2CDE9041266
:107AF000064A082148F09BFD284607B030BD00BF6C
:107B0000F17B0000A0EE002080EE0020D4BE050036
:107B1000F0B587B0D0F8A07004460D464EF004FDD5
:107B200006461DF08DFC234B2349244A002E08BF36
:107B30001E46234BCDE90046844208BF0B4628462B
:107B4000082148F074FDD4E90A23CDE9022394F911
:107B50000E301C4A00930821237B284648F067FD1D
:107B600020461BF0C3F9626E00920346164A0821B4
:107B7000284648F05CFD05A920464EF0D9FC034696
:107B800030B1124A0821284648F051FD07B0F0BD37
:107B9000059A6423B91ACDE900214B430C4AB3FB83
:107BA000F7F30821CDE9027328463B4648F03FFD34
:107BB000ECE700BF1ABF0500F4D005001DBF0500AB
:107BC000300C060029BF050055BF05006CBF05003D
:107BD00099BF050010B504464BF0D9F8034A034697
:107BE0000821204648F023FD002010BDD0BF05002D
:107BF000F0B5D0F8A06089B004460D4607A94EF054
:107C000097FC034630B1104A0821284648F00FFD82
:107C100009B0F0BD20464EF087FC0C4F079A0028B3
:107C200008BF3846B11A6423CDE90221CDE9000628
:107C30004B43074AB3FBF6F30821CDE9046328461A
:107C4000234648F0F4FCE3E76CBF05001ABF0500CB
:107C5000E6BF05000346006810B50C46114608B1A2
:107C6000027822B9024A204603F052FB204610BD9A
:107C7000E8C0050010B50C68D1E90112FFF7EAFF72
:107C8000034A03460821204648F0D1FC002010BDDD
:107C9000EDC005002DE9F0478AB0054601A81AF0AD
:107CA000AFFD019B1B4ADFF87880DFF87890DFF8A2
:107CB00078A0182606FB00360821284648F0B7FCB5
:107CC000019CB44203D300200AB0BDE8F08705AFA1
:107CD000394614222046FFF7BDFF424603460821DD
:107CE000284648F0A4FC20464EF0D1FB0A4A002862
:107CF00014BF4B4653460821284648F098FC1423ED
:107D000020460649049302AACDE9025718344EF0E2
:107D1000C8FBD6E70CC105004FD70500757C0000F5
:107D200016C10500FDC0050003C105002DE9F043A3
:107D3000114BDFF8489053F82140013187B053F8D8
:107D4000218006460027A04503D8384607B0BDE885
:107D5000F08320464EF09BFB054658B1142201A942
:107D60002046FFF777FF4A4603460821304648F091
:107D70005EFC2F461834E6E720A805001BC105006D
:107D800010B5082104461E4A48F051FC0021204647
:107D9000FFF7CCFF20B91B4A0821204648F047FCDA
:107DA00008212046184A48F042FC01212046FFF7EE
:107DB000BDFF20B9134A0821204648F038FC0821AD
:107DC0002046124A48F033FC02212046FFF7AEFF5E
:107DD00020B90C4A0821204648F029FC08212046F9
:107DE0000B4A48F024FC03212046FFF79FFF20B9EF
:107DF000044A0821204648F01AFC002010BD00BFAC
:107E000021C1050030C1050038C1050047C105008A
:107E100055C105008B1E022B2DE9F041074688460F
:107E2000144633D860681022002149F0AEFAB8F148
:107E3000020F06461ED0A0680A22002149F0A5FACA
:107E4000C5B2214A2B460821384648F0F0FBB8F16C
:107E5000040F1ED0102D0FD0202D10D0082D10D1C2
:107E60003378DBB2194A0821384648F0E0FB00209D
:107E7000BDE8F0812025E4E733889BB2F2E7336860
:107E8000F0E7134A0821384648F0D1FB6FF015009F
:107E9000EEE7E0681022002149F077FA0D4A034628
:107EA00004460821384648F0C2FB102D06D0202D8C
:107EB00007D0082DE5D1E4B23470D8E7A4B23480FD
:107EC000D5E73460D3E700BFADC10500D8C10500D8
:107ED000C2C10500E9C1050070B50F4C0546237805
:107EE0000E4639B133B10D4A012148F0A0FB6FF0C5
:107EF0000F0070BD83F00103237033B1084A0821DD
:107F0000284648F094FB012323702846314648F068
:107F10009BFB0020EDE700BF66590020FDC1050076
:107F200038C205002DE9F74F06462E48DFF8CC9001
:107F3000DFF8CCA0DFF8CCB0002303600D462A4860
:107F40002A4903600B7014468846012D274654F8D1
:107F5000043F24D9184602224946019349F0F5FA14
:107F6000019B90B922689278003A18BF012213440D
:107F7000184602225146019349F0E7FA019B30B9B5
:107F8000012388F80030013DDFE70022EFE71846C3
:107F90004946019349F0CDFA019BB0B9043700225C
:107FA0001146786849F07BF9114B002211461860A0
:107FB000786849F074F90F4B0F4918603046FFF7A5
:107FC0008BFF002003B0BDE8F08F1A782D2AE6D190
:107FD0005A78002AE3D05A460821304648F027FB59
:107FE000D1E700BFDC250020E425002067590020F0
:107FF000D8250020E02500200980000062C205008D
:1080000065C2050068C2050073B53E4B1C78182C8C
:1080100002D10C78112C31D0013A0C465518A542EA
:1080200025D18A5C1A700A78374CA2F13003092BEB
:1080300004D922F02003413B052B04D8236833499F
:10804000CA54013323602368022B34D110222F48F5
:10805000002149F09AF92E4A136803F8010B1360C6
:108060002C4A1368013313600023236023E014F8C3
:10807000016B182ED3D12678112ED0D1254C264A4B
:1080800023680190082148F0D2FA01980021FFF7F7
:1080900023FF224B187870B9214A23681168042BFA
:1080A0000BDC08B11160236013F003010CD11268DE
:1080B00013681BBA136002B070BD086800BA41F8BB
:1080C000040B043B0120EAE75B4203F0030358BFC3
:1080D0005942022907D112681168C1F3072343EA04
:1080E00001239BB2E6E70329E5D110680268110479
:1080F000C2F3074301F47F010B4302F47F421343B1
:108100000360D8E768590020DC250020645900206E
:10811000D8250020E42500207DC2050067590020F5
:10812000E025002007B50A484EF0B1F960B1094AD0
:1081300007491268084804230093012300F098FEC1
:10814000002003B05DF804FB6FF01200F9E700BFF8
:1081500020A20500BCA80500A0A305002DE9F34757
:1081600082460D4683685B6C03B19847DAF80830A5
:108170005B6B002B31D1DFF8F880DFF8F890002737
:10818000E86801A9026947F084FCDAF8083006467D
:1081900000283AD09B690199002B33D00246504603
:1081A00098470446002CE868214618BF012747F08D
:1081B0008CFC40B1414648464E2247F00DFA4E2114
:1081C000404647F0E3FC0CB1A642D9D04FB12B6832
:1081D0000020D3E90121904703E05046984700284A
:1081E000C9D1DAF808305B6ADBB9A86801A902696D
:1081F00047F085FC0446D8B9504648F022F92B6870
:10820000DC602BE06FF05704CCE79B6933B10122AF
:108210000DF10301504698470446D4E76FF0570428
:10822000D1E7504698470028DFD102B0BDE8F0877B
:10823000DAF8083001995B69B3B1024650469847B5
:108240000146A86847F086FC40B1094909488922DF
:1082500047F0C2F90648892147F098FC2B680120B5
:10826000D3E901219047E0E76FF05701E9E700BF4C
:1082700024C30500A2B8050070B546680C463168F5
:10828000B0688B600025C1E900420822C0E90055B2
:108290002946104449F09AF9F0680822C0E90055CF
:1082A0002946104449F092F93368DD60A3682BB188
:1082B0009B6C1BB10549324620469847A3689B6AD0
:1082C0000BB120469847002070BD00BF5D810000C3
:1082D00010B581680446083101F080FCA168034AAA
:1082E00020460831BDE8104001F01ABC87C30500E4
:1082F00038B5044650B92049204840F2D64247F0EC
:108300006BF91D4840F2D64147F040FCA3680BB121
:10831000636853B91849194840F2D74247F05CF9ED
:10832000154840F2D74147F031FCA368D3F86432D6
:10833000DB071DD4E06948F078FD606803685B687E
:108340009847054620B9E06848F0B4FEA3681D715F
:10835000A3685B6B13B1294620469847A3680022A7
:10836000C3F80C231DF06CF8BDE8384002F08EBE57
:108370006FF00F05ECE700BF95C30500A2B805003C
:1083800037B504468068D0F864325A070D4605D5E3
:10839000002148F0FCF8E06848F05EFEE368DB6826
:1083A0006BB9002D37D0A068423048F0DDF8A368E3
:1083B00098B303F1420103F5A17049F07FF8A26878
:1083C000E0680DF106034232294648F048FE58B9EC
:1083D000A06800F5A171423049F070F8A068423001
:1083E00048F0C2F8ADF80600204648F006FCA36845
:1083F000D3F860329B0603D50949606948F0BAF8A2
:10840000204601F073F8A368BDF80620DA879A8742
:10841000204601F02DF803B030BD83F84201CEE7CD
:10842000B0A405008368022210B51A719B6B044644
:10843000CBB9826882F84230D3638368D3F8643260
:10844000DB040BD50321084B084A01F00BF9A068A7
:108450006FF4805100F5197048F05EF82046BDE8D1
:10846000104001F02DBA10BDBDC3050018C10500B4
:108470002DE9F04F00239FB0CDE905338368044612
:108480004233039348F0BFFB204648F042FB18B943
:108490009F49606948F06EF8A068142200210830F6
:1084A00049F094F8204648F0ACFAA168E0688A8F59
:1084B0004231002601F016FD204648F021FE4FF023
:1084C000FF38B146B24611AF02963546B346DDE9F4
:1084D0000532012A00F0D7800B2B40F2AF80069BBB
:1084E000022B40F0AF808B4B8B4A012114E0039AA2
:1084F0000223394606A848F012F906997A680392D1
:10850000034629B96FF0070528461FB0BDE8F08F74
:10851000012905D120B1814A204601F0A3F8F1E7F5
:10852000059B4BB3386801F07DFB98B166B1A56837
:108530000D9608350CAE0FCE0FC533682B60204664
:10854000FFF7C6FE0125DFE7754A0121204601F04D
:1085500089F8D7E7059B7BB13A682946204601F0A8
:108560003BFD022800F08F80032805D0059B0133D6
:10857000059301230293AAE7BAF1000F05D13968E8
:1085800007AA584648F0B9F90546043708F1FF38FC
:10859000002D41D0029B4BB1EB683BB1204648F027
:1085A00032FB204600F064FF5E4ACEE7EB68CBB1B9
:1085B000A368DDF81490AE4603F1080CBEE80F0086
:1085C000ACE80F00DEF80030CCF80030AB684BB9F7
:1085D0006B7CFE2B01BF95F8108009F1010308F1B7
:1085E000FF380593D5F804C0BCF1000F08D0AE46A3
:1085F000BEE80F000CAE0FC6DEF8003033606646F2
:10860000AB46B8F1000F03D1069B022B7FF45FAF9E
:10861000059B013305935AE7059B63B9A368DB69A2
:108620000BB1DB683BB9404B0093404A119B0121E1
:10863000204601F017F84FF0010AE2E7B8F1000F09
:108640007FF455AF029B4BB1204648F07EFDA268F7
:108650000C23423211A905A848F061F8059DA068D5
:108660001EAB03EB8503002243F8342C436973B936
:10867000002E3FF447AFC368B3423FF460AF0D969E
:1086800000F1080556E7059B0B2BDBD927E7037E96
:10869000A5EB0905B3B1427E4FF6FF71FF2A08BF73
:1086A0000A469D4202D313449D420BD98368204A57
:1086B0000121204600F0D6FF2046FFF709FE6FF0AB
:1086C000150521E74FF4006100F5197047F015FF1B
:1086D000A06800F53E7047F045FFA36811AA29463F
:1086E00002EB89025B69204698470546A0684FF077
:1086F000FF324FF0FF3300F53E7047F068FFA0688F
:108700006FF4006100F5197047F006FFFCE600BF4A
:10871000CEBF050076C405001DC1050001C40500DB
:1087200015C4050033C4050062C4050079C70500FF
:108730009AC405002DE9F04F2DED028B0446A9B037
:1087400050B9B849B84840F2A35246F045FFB54881
:1087500040F2A35147F01AFAA36853B9B149B2489D
:1087600040F2A45246F038FFAE4840F2A45147F020
:108770000DFAA068012100F5197047F0BEFEA3684C
:108780001B79022B17D100230993A36860689E6BA5
:1087900003681D6909ABD6B110221BA9A847099A25
:1087A0004AB11BA92046B047A3689B6B002BECD1B4
:1087B0002046FFF737FEA0686FF0010100F5197041
:1087C00047F0AAFE29B0BDEC028BBDE8F08F012274
:1087D0000DF12301A847099B002BECD09DF9232024
:1087E0009DF82330A068002ACFDB4279032A00F2EB
:1087F0003883DFE812F00400A602CF0236030D2B07
:108800001AD00A2B18D0B0F864226FF3CA02A0F86D
:108810006422092B4DD033D8002BB6D0082B00F0A2
:10882000F281A3F120025E2A00F2F981012147F0D2
:10883000AEFE9DF82310FCE0D0F86422C2F3C7021C
:108840002AB1D0F86422C2F3C7029342E1D1B0F852
:108850006422818F63F3CA02A0F8642261B947F0F1
:1088600096FEE06848F0F8FB7049606947F082FEC8
:108870002046FFF7D7FD88E72046FFF7F9FDF7E729
:108880001B2B13D07F2BCCD1D0F860329D077FF506
:108890007CAF012147F07BFEA368D3F86032190753
:1088A00000F1B981204648F047FA6EE70123437191
:1088B0006BE7D0F860329B077FF567AF012147F087
:1088C00066FEA068838FFF2B3FF45FAFC28F00F17D
:1088D000420100F5A17048F06EFEA268D38F1344E8
:1088E000002583F842511BA90C2302F5A1720BA8A5
:1088F00047F015FF0B990C293FF647AF28AB03EB68
:10890000810343F8345CA368DA8F134493F8413051
:10891000202B00F0A882093B042B40F2A4820129FD
:108920005BD800250A950A9B28AA02EB8303002640
:1089300053F834AC504647F017FEB04681460396D4
:10894000374616AA3946284600F024FD83460028FB
:1089500050D1012E76D10A9B28AA02EB830353F84B
:10896000340C47F001FEA26806460832284641460C
:1089700000F010FD054650B92A492B4840F26F120D
:1089800046F02AFE274840F26F1147F0FFF82868AA
:1089900047F0EAFD864206D02968821B92B2314434
:1089A000204648F0C7F9A068C38F034493F84230CB
:1089B000202B42D0093B042B3FD9D0F86032DF078F
:1089C00036D5002147F0F3FD2021204600F040FF7E
:1089D000A068012147F0EBFDD7E6013900200CAB80
:1089E000009301900AAB1BAA47F0A7FF0546002899
:1089F00099D1CAE6DBF800004A46514648F0A5FD89
:108A000068B9DBF8000048F084FD039B834238BF5F
:108A100003469BB2002E08BFB846039301360137C8
:108A20008FE700BF95C30500A2B80500CEBF0500C3
:108A30002021204600F00CFFA7E60121204648F047
:108A40007EF8A2E67FF6A1AE0A9B28AA02EB83037A
:108A5000C14653F834AC504647F086FDA3680496EF
:108A6000A3F830B008EE900ADFF824B3A2684946B4
:108A70000832284600F08EFC074650B9BC49BD4874
:108A80004FF4DC7246F0A8FDB9484FF4DC7147F0B2
:108A90007DF8386809F10109BAF1000F5FD13B6830
:108AA000002B66D1A2681386049B013B0493DDD1A1
:108AB000B149606947F05EFD204600F001FF0A9B66
:108AC00028AA02EB830308F1010953F8340C47F09C
:108AD0004BFD4146074611AA284600F05BFC804644
:108AE00050B9A349A3484FF4EA7246F075FDA04877
:108AF0004FF4EA7147F04AF8A068D8F80010FF2256
:108B000000F5A17048F0E4FCD8F800A04FF6FF781B
:108B100016AA4946284609F1010B00F03BFC002843
:108B200064D0A368006803F5A173002213F801CB99
:108B3000815C614505D121B101324FF6FF718A4256
:108B4000F4D10FB1BA4208DB904506F1FF36A8BF59
:108B50009046012E1FFA88F848D0D946D8E7002859
:108B60009DD018EE902A514648F0EFFC002896D090
:108B70007CE75846059347F0F7FC039BA16818442F
:108B800082B258464F8D079247F0EEFC059B069047
:108B9000184647F0E9FC079A0699101A83B2A068B4
:108BA000B0F830C07F1A97FBF2F292B2BCFBF2F140
:108BB00002FB11C20CF1010E92B208EE103AA0F8BD
:108BC00030E0059B62B900936C4A5B460621204663
:108BD00000F048FD18EE101A204600F033FC63E761
:108BE000674A0621204600F03DFDF3E7B8F1000F8B
:108BF0003FF4CBADA8EB070292B20AEB0701204687
:108C000048F098F8C1E5D0F860329E077FF5BDAD19
:108C1000012147F0BCFC204648F0A9F8B5E5D0F8A2
:108C2000602292077FF5B1AD013B162B3FF6ADAD4B
:108C300001A252F823F000BF358E0000958C000091
:108C40009D8C0000A5880000298E0000BD8C0000CE
:108C50008B8700008B8700008B8700008B870000CC
:108C6000C58C0000CD8C00008B870000F78C0000C5
:108C70008B870000018D00008B8700008B87000030
:108C80008B8700008B870000058D00008B8700001C
:108C9000338D0000204647F0BDFF76E5204647F0C3
:108CA000B2FF204647F035FF18B93349606947F0F5
:108CB00061FCA068012147F06AFCD9E5204647F035
:108CC000B1FF62E5204647F0B6FF5EE5D0F86032BE
:108CD0009F0603D52B49606947F04CFCA368D3F885
:108CE00060329E0603D52849606947F043FC204660
:108CF00000F0E6FD49E500212046FFF741FB44E591
:108D00000121F9E7204647F078FFA368002283F8A5
:108D10004220DA63A068012147F039FCA368D3F848
:108D200060329D067FF531AD1849606947F022FC3D
:108D30002BE5204600F0F0FCA068012147F027FC5D
:108D400023E55B2B01D10223B1E5D0F86022900727
:108D500006D5622B08D14FF0FF31204647F013FFB4
:108D6000A36800225A7110E5662BF9D10121F4E7BE
:108D700095C30500A2B80500CEBF0500B5C4050027
:108D800018C10500B5A40500BAA40500B0A40500EB
:108D90002F0C060000224271A268D2F860128907E7
:108DA0007FF5F3AC313B1B2B3FF6EFAC01A151F843
:108DB00023F000BF318E00003D8E0000518E000078
:108DC000258E00008B8700008B8700008B870000BA
:108DD0008B8700008B8700008B8700008B8700004B
:108DE0008B8700008B8700008B8700008B8700003B
:108DF0008B870000018D0000F78C0000BD8C000007
:108E0000958C00008B870000298E00008B87000066
:108E1000358E00008B8700008B8700008B87000059
:108E2000418E000003235371204647F0ECFEACE472
:108E300003235371204647F0E0FEA6E40323537159
:108E4000A068D0F8601201F0010181F00101C1E5D4
:108E500003235371A368D3F860329B077FF595AC69
:108E600020E5002323E500293FF45BADB6E500BF14
:108E70002DE9F043884689B015461F46044650B98F
:108E80004B494C484FF4A96246F0A6FB48484FF4C2
:108E9000A96146F07BFEA3681BB163680BB1236830
:108EA00053B94349434840F2495246F095FB404884
:108EB00040F2495146F06AFEA368D3F80C33002B08
:108EC00072D1237C013B012B0AD93949394840F240
:108ED0009F4246F081FB364840F29F4146F056FEE5
:108EE0000021A0684FF4447248F070FBA368226828
:108EF000E0681A6048F0EAF8A06800F53E704DF0AE
:108F00002CFB4FF42A794FF41A76A06830444DF0C8
:108F10008AFCA068002283190121484410361DF004
:108F200049F9B6F52A7F09F11409EED1A369A068C1
:108F3000002602211E6000F5197047F0DEFAA368D2
:108F40001D4A9A62186847F00FFBA3681B4A83F812
:108F50002C00606866F38205C3F8605203684146DE
:108F60001D682346A8470546D0B9A36801221A7197
:108F7000D4E90A0100220023CDE906230E2303933E
:108F8000109B0495CDE9017300940D4B4FF40062E2
:108F90001AF042F9A368616AC3F80C0319F096FF4E
:108FA000284609B0BDE8F0836FF07705F8E700BF09
:108FB00095C30500A2B80500180050001B06050067
:108FC0005190000010B5044650B91E491E4840F2A9
:108FD0007B5246F001FB1B4840F27B5146F0D6FD28
:108FE000A3681BB163680BB1236853B915491648D0
:108FF00040F27C5246F0F0FA124840F27C5146F0C2
:10900000C5FDA0680379012B19D14FF0FF324FF055
:10901000FF3300F53E7047F0DAFA0821204600F0F1
:10902000E3FA0A49606947F0A5FA2046FFF7FAF922
:10903000A06800F53E7047F095FA002010BD6FF073
:109040008500FBE795C30500A2B80500CDBF05006C
:109050002DE9F34104464068019203680D469B6880
:109060000021984700284DD125B1019AE069214699
:1090700047F0C2FE2046FFF7A5FF002842D1DFF8E7
:109080009880224F224EA06800F52A704FF0FF32E0
:109090004FF0FF3303211DF0C3F80546A0684FF0E1
:1090A000FF324FF0FF3300F53E707DB147F08FFA8D
:1090B0002046184A2B46012100F0D4FAA06800F59A
:1090C0003E7002B0BDE8F04147F04CBA47F07FFA7D
:1090D000606803685B6903B19847424620460221F5
:1090E00047F029FA3A462046002147F024FA204664
:1090F0003246012147F01FFAA06800F53E7047F0A4
:1091000031FAC0E702B0BDE8F08100BF358700004A
:10911000D3050500BBC40500F18200002DE9F04134
:109120000E4615461F46044650B9474947484FF476
:10913000B86246F051FA44484FF4B86146F026FD53
:109140004DF0ECF950B14049404840F2C15246F070
:1091500043FA3D4840F2C15146F018FDA36853B9A7
:1091600039493A4840F2C25246F036FA364840F29F
:10917000C25146F00BFDD4F80880D8F864321805C7
:1091800010D41CF05DF9D8F80C3383420AD12E4973
:109190002E4840F2C35246F01FFA2B4840F2C3510A
:1091A00046F0F4FC636953B92749284840F2C55298
:1091B00046F012FA244840F2C55146F0E7FC55B992
:1091C0002149224840F2C65246F006FA1E4840F2B3
:1091D000C65146F0DBFCA0680379022B07D0BDE83E
:1091E000F0414FF4805100F5197047F086B94FF007
:1091F000FF324FF0FF3300F53E7047F0E8F9A36807
:10920000D3F86422110504D49B6B13B9204647F0B0
:109210001BFD3B462A463146204647F031FDA368F8
:10922000D3F86422120504D49B6B13B9204600F0D6
:1092300047FB606947F00BFAA068BDE8F04100F514
:109240003E7047F08FB900BF95C30500A2B8050076
:1092500010B50D4A0446082147F0E9F920460B4AAB
:10926000082147F0E4F92046094A082147F0DFF9D0
:109270002046084A082147F0DAF92046064A00212C
:1092800000F04EFC002010BDD2C4050010C5050042
:109290006FC50500C3C505005DC605002DE9F04793
:1092A00016461F462A4ADFF8B480DFF8B490DFF88C
:1092B000B4A00B460821044647F0B9F90025AF4297
:1092C00031D9735D4A460821204647F0B0F901358F
:1092D000102D20D11F4ADFF88C80DFF88C900821F8
:1092E000204647F0A4F90025AF422AD9735DA3F1C7
:1092F00020025F2A28BF2E234A460821204647F035
:1093000096F90135102D14D12046134ABDE8F047D7
:10931000082147F08CB96A07D1D15246082120466E
:1093200047F085F9CBE742460821204647F07FF910
:10933000CDE76B07D8D142460821204647F077F9A0
:10934000D2E742460821204647F071F9D9E700BF2D
:1093500073C6050092BA05007AC605002E0C0600F9
:109360008CBA0500300C0600C8C6050010B50446CE
:1093700013460A4601460648FCF702FA23691B79A0
:1093800023B12046BDE8104047F061B910BD00BFD1
:109390006706050070B50D461446064650B91449D7
:1093A000144B5B1AB5EBD30F1BD201EBC5014C6814
:1093B000204670BD52B91049104840F2031246F0E1
:1093C0000BF90D4840F2031146F0E0FBB26842B1E0
:1093D000536812783AB12146284698472368002BF3
:1093E000E6D10024E4E714214D435C195B59F6E70C
:1093F000D0A3050068A4050096C60500A2B8050024
:109400008368D3F860329B0603D50249406947F070
:109410005DBB7047C0A405000A1E0DDC0ED04223C0
:109420008168D1F86012890608D5002A044940698C
:10943000B8BF524247F04ABB4123F1E7704700BF33
:10944000C4C605000A1E0DDC0ED044238168D1F885
:109450006012890608D5002A04494069B8BF524203
:1094600047F034BB4323F1E7704700BFC4C6050093
:1094700010B5044647F04DFB28B160690549BDE8C9
:10948000104047F023BB04F1080047F02CFB0028F4
:10949000F3D110BDCEBF05002DE9F04106460546CB
:1094A00056F8084F04F12000A28FE18F47F021F910
:1094B0003046B4F82480E78C47F015FB18B10A4910
:1094C000686947F003FBB84507D1218C638C2846B7
:1094D000C91ABDE8F041FFF7B5BFE18CA38C28465F
:1094E000C91AFFF799FFF0E7CEBF0500826802496D
:1094F0004069423247F0EABA18C105002DE9F04749
:109500000E4686B01446054600B151B93449354877
:109510004FF4CA7246F060F831484FF4CA7146F011
:1095200035FB2F4FDFF8BC904FF0000814B906B0A0
:10953000BDE8F087686803682246D3F80CA006EB04
:1095400008016B46D04750B1394648464FF4CF72B8
:1095500046F042F84FF4CF71384646F017FB009BB7
:10956000A3420AD93946484640F29F1246F034F8E1
:1095700040F29F11384646F009FB009A9044A41A25
:10958000002AD3D1AB6819790329CFD0022913D887
:1095900003F52673012101A81CF00CFE4FF0FF32E9
:1095A0004FF0FF33012101A81CF03AFEA86800F536
:1095B00026704DF03DF9B9E7D3F864229207FBD548
:1095C000BFF35B8F03F5197353E8002F22F00202FB
:1095D00043E800210029F7D1BFF35B8FA6E700BF66
:1095E000CBC60500A2B80500082918D8836893F8EF
:1095F0002E208A4213D083F82E1083680829D3F8CE
:10960000603206D09A060AD50A464069044947F0F6
:109610005DBA9B0603D50349406947F057BA7047C6
:10962000F7C60500C5A4050038B50D4609780446FF
:10963000FFF7DAFF6A78072A11D8A36893F82F108A
:1096400091420CD083F82F20A368D3F860329B0698
:1096500005D560690249BDE8384047F037BA38BDE2
:1096600000C705000CB473B5069E0D46044650B9FC
:109670002749284840F2FD1245F0AEFF244840F249
:10968000FD1146F083FAA36853B9214921484FF4EC
:10969000FF7245F0A1FF1E484FF4FF7146F076FAC5
:1096A000636953B91A491B4840F2FF1245F094FF11
:1096B000174840F2FF1146F069FA56B914491548A7
:1096C0004FF4007245F088FF11484FF4007146F0E6
:1096D0005DFAA368D3F864329B040DD44CF01EFFEE
:1096E00050B10B490B4840F2012245F075FF084884
:1096F00040F2012146F04AFA07AB3246294620469D
:10970000019347F0BDFA02B0BDE8704002B0704767
:10971000CBC60500A2B80500F8B583689A8F054648
:10972000002A4ED0D88F00284BD04130184403F186
:1097300042060346C41AB342A4B219460DD311F827
:109740000179202F3BD01946013B0878202804D00E
:1097500001349E42A4B21946F5D9631C4E1C121B5B
:109760001944304647F010FFA9688A8F121B92B245
:109770008A870A440023614282F8423009B22846AF
:1097800047F0DDF9AB68D3F860329A0603D50D498E
:10979000686947F09BF933460B4A08212846FFF7D2
:1097A00061FF2846FFF72CFEAB68D3F860329B06BA
:1097B00007D568690549BDE8F84047F087B90B4609
:1097C000B8E7F8BDCAA4050018C10500CEA405007D
:1097D0002DE9F04104460D4617460AB1FFF710FE89
:1097E000A368D3F86022D88F520700F142000344E7
:1097F00021D5184647F08DFEDFF850800646013E21
:1098000014D2204650F8083F9A8FDA8747F06BF958
:1098100028B107B11DB10B49606947F057F969429A
:10982000204609B2BDE8F04147F089B96069414678
:1098300047F04CF9E3E7044A08212046FFF712FFFE
:10984000DFE700BFCEBF050018C10500F4D005005A
:1098500013B583688DF80710D3F860220446D0074B
:1098600023D5D98F9A8F8A421FD0481CD8870B44A2
:109870009DF8072083F84220A368D3F86012890777
:1098800011D5D3F8603260690B4913F0040F18BF8B
:109890002A2247F01BF9204647F03BF918B1074947
:1098A000606947F013F902B010BD01220DF1070104
:1098B000204647F00DFAF6E7C8C60500CEBF050002
:1098C00083680A4A1B6810B504460221FFF7CAFEE6
:1098D000A368D3F860329B0707D52046FFF706FE42
:1098E0002046BDE81040FFF7D7BD10BD18C10500E8
:1098F0002DE9FF4743681C68A3680846D3F86062F7
:109900000D4646F06DFBE369DB681B79012BC6F35E
:10991000001605D0032B77D0284646F090FB70E068
:1099200000954CF0E5FE4FF47A730A46A0FB030164
:1099300003FB0211C30B43EA414301934FF400457B
:1099400040F2E7360027E3691969D3F80480B1468D
:10995000BA46E5FB019A4FF47A7200234846514615
:10996000F6F7ECFF02460B466946404619F046FD05
:1099700010F10B0F03D000283DD0233032D1E36922
:10998000D3F80480D3F810904CF0B2FE4FF47A7301
:109990000A46A0FB030103FB02114FEAD03A4AEA50
:1099A000414A02A9404619F04BFE0028CBD1039B47
:1099B000AAEB03039945C6D20023002202A9404620
:1099C00019F0AAFD029846F03AFBA369BFF35B8F3A
:1099D00053E8002F013243E800210029F8D1BFF3FA
:1099E0005B8FDEE70F4910487F2245F0F5FD0D48FB
:1099F0007F2146F0CBF8A06800F51E7000211CF016
:109A0000E5FC04B0BDE8F087204647F01DF9E369A6
:109A1000002E98680CBF0E220F222946FDF776FC17
:109A20007AE700BF09C70500A2B805002DE9F04795
:109A3000044690460E4600296ED00025735D202B0B
:109A400025D0093B042B22D9DFF8D090304647F0CF
:109A500060FDA368598D80B2401BA1EB08039842BA
:109A600006EB050A15D95046002710F8012B202ACD
:109A700006D0A2F1090CBCF1040F02D80A2A31D099
:109A80003B4608EB070291422BD90137EDE7013540
:109A9000D4E753460027B84217D013F8012B0A2AFF
:109AA00005EB07091BD1606946F0D1FD3A465146E6
:109AB0002046FFF723FD1949606947F037FA414610
:109AC000204609F10105FFF7BDFC6069711947F0F7
:109AD0002DFA60691149BDE8F04747F027BA013710
:109AE000D9E71F46606946F0B2FD3A465146204626
:109AF000FFF704FD3D44735D202B0BD0093B042B85
:109B000008D96069494647F011FA41462046FFF7F7
:109B100099FC9BE70135EEE7BDE8F087CEBF050075
:109B20002DE9F04F0E4600218DB0044617460D4634
:109B300007AA304601F10108FFF72CFCB8B99DB126
:109B400027B13A4608212046FFF78CFDDFF88080D8
:109B5000DFF880A0DFF880B000214B1C07AA304658
:109B60000493FFF717FC60B90DB0BDE8F08F0068F3
:109B700010B147F0CEFC80B2854238BF0546414661
:109B8000D6E70368D0F804901148059347F0C1FC6C
:109B9000059B07468BB11A787AB1CDE9013800955B
:109BA0004346524608212046FFF75CFDB9F1000FFD
:109BB00005D16069594647F0B9F90499CDE76A1CA7
:109BC00002EB470292B249462046FFF72FFFF4E727
:109BD00055C705003DC70500CEBF0500F7B50646D1
:109BE00008680D46B8B147F094FC84B20B4F384674
:109BF00047F08FFC2B680A4A00970444082130463E
:109C0000FFF730FDA4B269682246304603B0BDE8D4
:109C1000F040FFF70BBF0446E8E700BF51C705005F
:109C2000B6C4050010B50749044647F082FC38B1B8
:109C30000549204647F07DFCB0FA80F0400910BD90
:109C40000120FCE747C705004AC7050010B5836837
:109C5000D3F860329B06044603D50449406947F0B7
:109C600076F9A368024A9A62002010BDD2A40500CA
:109C70001800500008B58369034A1B68082146F0A4
:109C8000D6FC002008BD00BF58C705007FB50F4EA9
:109C900004460025A268E0680DF10E0302F5A172EA
:109CA000012147F0DCF9BDF80E00A36850B103F5BF
:109CB000A173009332462B460821204646F0B7FC9C
:109CC0000135E7E783F8420104B070BD68C70500BD
:109CD00010B58368D3F860329A06044603D5074965
:109CE000406947F034F9A368D3F860329B0603D586
:109CF0000349606947F02BF9002010BDD9A4050085
:109D0000DEA40500022907B50DD1536801930E4B5F
:109D1000009313680D4A012146F089FC6FF015008D
:109D200003B05DF804FB8368094AD3F8603213F08E
:109D3000020F4FF00801074B18BF1346064A46F0C2
:109D400076FC0020ECE700BF7FC7050076C7050062
:109D500094EB050072C7050094C70500F0B5012912
:109D600085B004460DD053680193574B0093136898
:109D7000564A012146F05BFC6FF01505284605B0F8
:109D8000F0BD8368D3F860329A0603D55049406924
:109D900047F0DDF86FF0F9012046FFF73DFBFA21AF
:109DA0002046FFF74FFBA06800254FF4807229463C
:109DB00000F5A1708DF80B5047F008FC454960692B
:109DC00047F0C5F8606946F042FC4FF47A76606867
:109DD000036801221F690DF10B0103ABB847039B18
:109DE00053B9013E4FF47A70B6B24CF083FC002EAA
:109DF000EDD16FF0850531E09DF80B30A2681B2B8B
:109E000057D092F842111B29E1D1522B51D1154460
:109E1000002385F8423192F843115B2951D102F5B4
:109E2000A2701F46022610F8011B01363B29B6B26C
:109E30002AD1B6F5807FDCD006F5A170104400234E
:109E400010F8015B55BBFA2B28BFFA23FA2F538574
:109E50003B4628BFFA2382F842511385A368D3F802
:109E600060329B0603D51C49606947F070F8002DED
:109E700084D0A368194A9A620321194A204646F001
:109E8000D6FB6FF0070579E707EB870301EB430388
:109E9000303BB6F5807F9FB2C5D1AAE703EB8303C1
:109EA000013605EB4305B6B2303DFF2EABB2C7D944
:109EB0009FE751190135ADB2092D81F8423186D99C
:109EC000002382F8423194E77FC7050076C705007A
:109ED000E4A4050092CB0500E8A40500180050009A
:109EE000A5C705002DE9F74F036802F10C056F4285
:109EF0001B6907F003073D449D4204468946164608
:109F00003FD80023C360002A3BD000F1040840681A
:109F100080452BD10193DFF8BCA020682A4601A917
:109F200045F0B7FD854283462ED920682A4601A90F
:109F300045F0AFFD854228D15946206845F0C5FD62
:109F40005F44BFB2AB46019D324649462E816F81C8
:109F500005F10C0047F02FFB62682068C5E9002876
:109F600059465560656045F0B0FD0AE00190002853
:109F7000D1D003899342CED10C3047F0F5FA0028B6
:109F8000C9D103B0BDE8F08FDDD02068002145F0D5
:109F90009CFD6368984515D1206845F06AFD40B97D
:109FA0000B485146BD2245F017FBBD21504645F0F8
:109FB000EDFD206800210822C0E90011104447F09F
:109FC00005FBAAE7204647F035F80028A5D1E3E7CE
:109FD000A2B8050097CB05002DE9F04F074689B0E0
:109FE0001546894621B90324204609B0BDE8F08F03
:109FF000104647F071F80028F5D04FF000084146B0
:10A00000022426E05C463EE029460AF5A17047F0AE
:10A0100035FA0646002850D047F07BFA04F1010CCF
:10A0200080B2421C314606EB0C0047F0ADFA2246E6
:10A030005946304647F0BFFA4FF020033355BAF87F
:10A04000400004440134AAF8404008F1010800240B
:10A0500001994B1C03AA48460193FFF79BF906465A
:10A06000F8B131680022284645F0CFFE0028EFD134
:10A07000D6F800B0D7F808A0BBF1000FC2D0584600
:10A0800047F047FA84B2BAF8402001322244B2F5D0
:10A09000807FB9DD0A4A2B4603213846FFF7E2FAF2
:10A0A0000124B8F1000F9FD0B8682A4600F14001A2
:10A0B00000F5A17046F0FAFB96E70224F1E700BF35
:10A0C000C7CB05000C4B1B6870B573B10B4A156804
:10A0D0000022AA4202DB6FF0010070BD1C4613F89B
:10A0E000106B864204D00132F3E76FF00C00F4E706
:10A0F0000C600020F1E700BF3401002084AB0500B4
:10A100002DE9F84305464FF04003EFF3118683F342
:10A110001288BFF36F8F1E4818F022FF40B91D4907
:10A120001D48812245F058FA1A48812145F02EFD3C
:10A13000174818F033FF194B1C68002C38BF002457
:10A140009CB1174FDFF85C804FF00C09D4E9013265
:10A15000002D08BF13462BB198F8142009FB02F21A
:10A16000B85C98472468002CF0D1094818F006FF25
:10A1700040B908490848AC2245F02EFA0548AC2100
:10A1800045F004FD86F31188BFF36F8FBDE8F883B7
:10A190002C290020DCB80500A2B8050030290020D9
:10A1A0003C290020BC55002000F01F0301229A40EA
:10A1B0000A4BBFF35B8F400903EB800050E8003F80
:10A1C00043EA020140E8001CBCF1000FF6D1BFF3E6
:10A1D0005B8F1A4214BF01200020704748290020DD
:10A1E00030B51D4B1D7DBFF35B8F05F01F030122B2
:10A1F0009A401A4B690985B0D04303EB810353E8B9
:10A20000001F01EA000443E8004CBCF1000FF6D146
:10A21000BFF35B8F114217D0114C0C2202FB054299
:10A2200007CA01AB83E807000E4A7AB193E807003A
:10A2300047F0F8F90020FFF763FF0C236B4300227F
:10A24000E118E250C1E9012205B030BD82F3118866
:10A25000BFF36F8FEEE700BFBC5500203829002008
:10A260003C290020251605002DE9F041374BDFF889
:10A27000F4801C7D88B007462046FFF795FF60B943
:10A280006E463A462146304646F0E7FF96E807001C
:10A290000C2505FB048585E807000C23634308EBC8
:10A2A000030218F80300650904F01F06C8B37B1CFD
:10A2B0000FD0D2F808E02648264A4FF4004C00217F
:10A2C0000023ECFB0E01F6F739FB0121381A1BF0D5
:10A2D00055FB1AF0C1F90120FFF712FFBFF35B8FA6
:10A2E0001D4B0122B24003EB850353E8001F1143CD
:10A2F00043E800100028F8D1BFF35B8F0C2303FB69
:10A30000048494E8070005AB83E80700134A1AB1F8
:10A3100093E8070047F073F9FFF762FF1AF050FE69
:10A3200001200F4ABFF35B8F0123B340DB4302EBF5
:10A33000850555E8002F1A4045E800210029F8D18D
:10A34000BFF35B8F08B0BDE8F08100BFBC550020B3
:10A350003F420F0040420F0038290020FF15050042
:10A36000482900203C29002070B504460D461646B9
:10A3700000F0E8F840B108490848542245F02CF9AB
:10A380000548542145F002FC054840F8346000EBD4
:10A39000C400456070BD00BF2CCC0500A2B805000C
:10A3A0003C050020014910220A60704710ED00E0D2
:10A3B00072B6404080F31188BFF36F8FBFF34F8FA9
:10A3C00030BF62B6BFF36F8F704700BF72B64940AF
:10A3D00081F3118820BF80F3118862B6704700BFF7
:10A3E0002DE9F04F81468BB00C4600296ED03B4ED4
:10A3F0003B4D3368751B5A074FEA95051DD0AF01D9
:10A4000047F00107ADF80070D1E90123354809682C
:10A4100045F064FD33685B070FD0ADF80070D4E9F8
:10A4200004233148E16845F059FD3368580704D0EA
:10A43000E1692E483A4645F021FD4FEA851ADFF8DA
:10A44000B8B0A04600274AF0010A3368590725D062
:10A45000D8ED087A0297FCEEE77A7B1CCDED037A03
:10A46000D8ED097A0493FCEEE77ABB1CCDED057AB2
:10A47000D8ED0A7A0693FCEEE77AFB1CCDED077A5D
:10A48000D8ED0B7A0893FCEEE77A082253460DEBE1
:10A4900002015846CDED097A45F03FFD0437102FF3
:10A4A00008F11008D1D133685A070FD0AD0145F03B
:10A4B0000105216E0E482A4645F0E0FC33685B0733
:10A4C00004D0A1690B482A4645F0D8FC21464846ED
:10A4D00018F0D6F90BB0BDE8F08F00BF28070020B8
:10A4E000E80600205BCC05008ACC0500B9CC05004D
:10A4F0000BCD05001ACD0500C8CC050043B2002BDA
:10A5000008DB012200F01F0002FA00F05B09024A9A
:10A5100042F82300704700BF00E100E043B2002B87
:10A520000DDB01225B0900F01F0002FA00F020336E
:10A53000034A42F82300BFF34F8FBFF36F8F70477A
:10A5400000E100E0054B420900F01F0053F8222013
:10A55000012303FA00F01040704700BF00E100E063
:10A5600038B5D30705461ED48C1C072C08D90F49D3
:10A570000F48592245F030F80C48592145F006FBA8
:10A580006BB2002BACBF03F160430A4B4FEA44149B
:10A59000B8BF05F00F05E4B2AABF03F561435C55EF
:10A5A00083F8004338BD0024EAE700BF48CD05002A
:10A5B000A2B8050014ED00E008B572B6044B9A6924
:10A5C0001AB100229A614BF0C1FF62B608BD00BF0C
:10A5D000BC55002030BFFFF7FDBF00BF144A08B5CF
:10A5E000144B22F07F029A60BFF34F8FBFF36F8F3F
:10A5F000D3F8882022F47002C3F88820D3F888208A
:10A6000042F4A002C3F888204FF04042C3F834223D
:10A61000BFF34F8FBFF36F8F0023E1EE103A18F0B6
:10A6200003FA1BF013F800F0B1FC18F007FA00BFB2
:10A630000000000000ED00E00A4A0B499368096839
:10A64000C3F8B0100949C3F8AC004B6843F080531D
:10A650004B60002383F31188BFF36F8F9368D3F8A7
:10A66000B0007047BC550020CCB6050000ED00E0FE
:10A6700022498A6882F8F5E04FF030001044EFF389
:10A68000098C80E8F01F1EF0100F03D102F1B40016
:10A6900080EC108A402080F31288BFF36F8F184F30
:10A6A0004FF00066CA698A603E6092F9F5E0D2F820
:10A6B000AC000023C2F8AC3080F311881EF0100FFC
:10A6C00003D00023E1EE103A03E002F1B40090EC75
:10A6D000108AEFF3148323F0040383F31488BFF389
:10A6E0006F8F04B5104600F0EFFCBDE8044002F1A6
:10A6F000300090E8F01F8CF309887047BC550020AB
:10A7000004ED00E01EF0040F0CBFEFF30880EFF340
:10A710000980816911F8021C0229FFD001B546F0B9
:10A72000A1FD01BD017B10B511F0020409D0D0F8E4
:10A730009C106031C0F89C10D0F8A0106039C0F8AF
:10A74000A01042F8203C029B42F81C3C039B42F8BC
:10A75000183C0D49049B42F8143C4FF0807342F8BA
:10A76000043C21F00101002342F8081C203AC0F803
:10A77000AC304FF47D430265C0F8F4301CB14FF6A5
:10A780000853C0F8F43010BDEBF6040030B5017B7F
:10A79000D0F8F4301B4A11F0020F03F0080503D182
:10A7A00090F8F540E40617D4546844F080445460AF
:10A7B0006DB943F00803C0F8F430D0F89C30603332
:10A7C000C0F89C30D0F8A030603BC0F8A03041F019
:10A7D00002010173802030BD516821F08041516039
:10A7E0006DB123F00803C0F8F430D0F89C30603B22
:10A7F000C0F89C30D0F8A0306033C0F8A0302020E2
:10A80000E9E700BF30EF00E00F4B0246986810B553
:10A81000C8B1D0F8F430D0F89C0013F0080F14BF82
:10A820008024202412F1160F04D0031B934206D873
:10A83000824204D281422CBF0021012100E000218C
:10A84000002908BF002010BDBC550020144608B5E3
:10A850000D460022E1EE102AEFF3148222F00402EA
:10A8600082F31488BFF36F8FBFF36F8F084A906035
:10A8700000F02AFC204685F30988002163B681F3A5
:10A880001188BFF36F8F0022002344F02EFF00BF1A
:10A89000BC55002001B572B60B4A906900281EBF56
:10A8A000002191614BF052FE62B6EFF30580A0F1FA
:10A8B00010004FEAC0000549014409C99847BDE8A6
:10A8C0000140034908470000BC5500203C0500201A
:10A8D000D5A80000044B9968D869884203D0034981
:10A8E0004FF080520A607047BC55002004ED00E034
:10A8F0002DE9F041574C236888465907074615460D
:10A9000008D055495548611A8908890141F001016B
:10A9100045F0A5FA524B9B6ADA060BD523685B0714
:10A9200008D04D494F48611A8908890141F0010159
:10A9300045F095FA4A4B9B6A1E070BD523685807CA
:10A9400008D045494848611A8908890141F0010148
:10A9500045F085FA424B9B6A990735D46FF015068E
:10A960003F4B9B6AD9070BD523685A0708D03A4951
:10A970003E48611A8908890141F0010145F06FFAEA
:10A98000374B9B6A9B060BD52368580708D0324982
:10A990003748611A8908890141F0010145F05FFAE1
:10A9A0002F4B9A6A12F0100F984634D19B6A990780
:10A9B00031D400242A4A936A43F0FF0393620023B0
:10A9C0002B702046BDE8F08123685A0708D0224941
:10A9D0002848611A8908890141F0010145F03FFAD0
:10A9E0001F4B5E6B9B6A1B06B8D52368580709D0BE
:10A9F000194A2148A21A9208920142F001023146F6
:10AA000045F03CFAB8F1000FAAD0154A936A23F03A
:10AA100080039362A4E7D8F804301A05C9D53946F3
:10AA20003046FFF7F1FE044618B180F3098802248E
:10AA3000C0E7D8F82830DB06BBD51049104840F2F3
:10AA4000491244F0C9FD0D4840F2491145F09EF805
:10AA5000B0E700BF28070020E80600207ECD0500F3
:10AA600000ED00E094CD0500C7CD050008CE05003F
:10AA700027CE0500DACD0500F2CD050056CE050043
:10AA8000A2B8050010B53B4C23685B0708D03A49D3
:10AA90003A48611A8908890141F0010145F0DFF95E
:10AAA000374B9B6A98010BD52368590708D0324968
:10AAB0003448611A8908890141F0010145F0CFF954
:10AAC0002F4B9B6ADA010BD523685B0708D02A4914
:10AAD0002D48611A8908890141F0010145F0BFF94B
:10AAE000274B9B6A18030BD52368590708D02249C6
:10AAF0002648611A8908890141F0010145F0AFF942
:10AB00001F4B9B6A5A030BD523685B0708D01A4971
:10AB10001F48611A8908890141F0010145F09FF938
:10AB2000174B9B6A98030BD52368590708D0124925
:10AB30001848611A8908890141F0010145F08FF92F
:10AB40000F4B9B6ADA030BD523685B0708D00A49D1
:10AB50001148611A8908890141F0010145F07FF926
:10AB6000074A936A6FEA03436FEA13439362002034
:10AB700010BD00BF28070020E806002090CE050089
:10AB800000ED00E0A8CE0500BBCE0500D5CE050047
:10AB9000F3CE050018CF050032CF050070B5464C46
:10ABA00023680D465907064608D044494448611AAF
:10ABB0008908890141F0010145F051F9414B9B6A37
:10ABC000DA040BD523685B0708D03C493E48611A7C
:10ABD0008908890141F0010145F041F9394B9B6A2F
:10ABE00018050BD52368590708D034493748611A2E
:10ABF0008908890141F0010145F031F9314B9B6A27
:10AC00009A0522D523685B0708D02C493048611A81
:10AC10008908890141F0010145F021F9294B996B1F
:10AC20009B6A180411D523685A0708D0234A29487B
:10AC3000A21A9208920142F0010245F01FF926B1D2
:10AC4000204A936A23F4004393621E4B9B6A5B0580
:10AC50000BD523685E0708D018491F48611A890878
:10AC6000890141F0010145F0FAF8164B9A6AD005C6
:10AC700013D52368590708D010491848641AA40846
:10AC8000A40144F0010145F0EAF80E4A936A00205D
:10AC900043F47F439362287070BD9B6A9A04F4D595
:10ACA00023685B07F1D005490D48641AA408A40184
:10ACB00044F00101E7E700BF28070020E806002074
:10ACC0005DCF050000ED00E073CF0500C7CD0500A6
:10ACD00084CF05009DCF0500B2CF0500CDCF050084
:10ACE00027CE05002DE9F0418E4B5D689CB0C5F381
:10ACF0000804002787F31188BFF36F8F02F07F43AA
:10AD0000B3F17F4F11D102F00C03082B1AD1864901
:10AD10000B6813F007032AD0844B8548C91A8908A9
:10AD2000890141F0010145F09AF88249824840F2D8
:10AD3000F23244F051FC7F4840F2F23144F026FFF9
:10AD4000002606E016074EBF0E4606460127002ED7
:10AD5000EBD000238DF80730E31E092B00F2C580ED
:10AD6000DFE803F007AEB296C3C3C3C3C3B61F4642
:10AD7000DBE76D4D2B685C0708D06C496F48691A9A
:10AD80008908890141F0010145F069F8654BDC6AE9
:10AD90004FF0000814F002048DF807800ED02B68E5
:10ADA000580701D1002418E060496548691A8908EC
:10ADB000890141F0010145F052F8F3E7DA6A002A0F
:10ADC00026DA2B685907EDD058495E48691A890878
:10ADD000890141F0010145F042F89DF80730A3B91F
:10ADE0006822314602A846F0E6FB099B002F00F0DE
:10ADF0009480C3F3080222B96FEA53236FEA432316
:10AE0000099302A92046FFF7EBFA1CB0BDE8F081D8
:10AE1000DB6A5A004BD52B685B0708D043494A4888
:10AE2000691A8908890141F0010145F018F8B369F0
:10AE300033F8022C4DF602739A420DD003F16043B1
:10AE400003F626631B78B3B10DF1070201213046EA
:10AE5000FFF74EFD0446C0E72B685C0709D0334A74
:10AE600031683A48AA1A9208920142F0010245F06C
:10AE700005F83468B1E7364B1B782BB10DF10701AB
:10AE80000120FFF78BFEE5E7324B1B889BB213B125
:10AE9000FFF7F8FDDEE72749274840F2C32244F0D8
:10AEA0009BFB40F2C321234844F070FE95E7214903
:10AEB000214840F2C72244F08FFB40F2C721F2E75D
:10AEC0000DF107020021C2E70DF107010020D8E7CC
:10AED00015490B6858073FF465AF144B1E48C91A53
:10AEE0008908890141F0010165E70F4B1A68520793
:10AEF0003FF458AF0D4A194819499B1A9B0815F49D
:10AF0000F87F4FEA831318BF014643F00103154849
:10AF1000A4F1100244F0C9FF44E723F4FF7323F0C7
:10AF200001036DE700ED00E028070020E80600209F
:10AF3000E5CF050056CE0500A2B8050010D00500EB
:10AF400027D0050048D0050056D0050075D0050073
:10AF500029ED00E02AED00E091D00500CAD00500FF
:10AF6000B5D00500E3D00500024A536943F0100351
:10AF70005361704700ED00E0EFF30880EFF30981C3
:10AF800001B57246FFF7AEFE01BD00BF04480023C5
:10AF90004021C2180133302B82F80013F9D17047D9
:10AFA00000E100E0002080F31488BFF36F8F4FF0C2
:10AFB00085F8002011490860BFF34F8F104880F3D7
:10AFC000088800F031F8402080F311880D484FF0D8
:10AFD000AA014FF4026246F0F9FA0A484FF40261FE
:10AFE000401880F30988EFF314800221084380F3AE
:10AFF0001488BFF36F8FFFF7F1FA000094ED00E0C3
:10B0000080EC002080EE0020064A11680023C1F386
:10B01000072118468B4200D17047936010610133BD
:10B02000F8E700BF90ED00E008B572B6002383F3A7
:10B030001388FFF7E9FF144B4FF0FF32C3F880206D
:10B04000C3F88420C3F88820C3F88C20C3F890206C
:10B05000C3F89420C3F89820C3F89C20C3F880213B
:10B06000C3F88421C3F88821C3F88C21C3F8902148
:10B07000C3F89421C3F89821C3F89C2162B6BFF3AA
:10B080004F8FBFF36F8F08BD00E100E0064B9B6858
:10B09000834207D1EFF3058323B1044A536843F099
:10B0A000805353601AF0E2B9BC55002000ED00E077
:10B0B000024B034A0348012100F092B8000002202D
:10B0C0000000002088AB050010B50446FFF75EFBCA
:10B0D000D4F89C20054B121AC3E90020044A9A6058
:10B0E000BDE810400121184600F098B84C29002016
:10B0F00000000B15F8B52C4F0E460021B14201DBC4
:10B100001046F8BD4468002C4BD0C3B104F1FF3C9D
:10B1100014EA0C0F0DD0254A1368580726D0244B8B
:10B120002448D21A9208920142F0010244F0A6FE8D
:10B130001CE01F2CEFD905681CEA050FEBD1202C71
:10B14000D5B2D0F808C0026813D9B4F1004F12D8B4
:10B15000013CB4FA84F4C4F11F046400072D4CEAE6
:10B16000040413D9114A13685B0706D16FF0150266
:10B17000C6E70824F2E73E24F0E70D4B0E48D21A4A
:10B180009208920142F001022946CFE722F01F0205
:10B190002A4342F0100244F00104BD60FA603C61B1
:10B1A0006A1C01310C30A9E790ED00E0180700207F
:10B1B000E8060020FAD005001DD10500034B05224A
:10B1C0005A60BFF34F8FBFF36F8F704790ED00E071
:10B1D000BFF35F8F014B00225A60704790ED00E093
:10B1E00010B50B4C01232278FFF784FF2070163036
:10B1F0000CD10849084840F2111244F0EDF9BDE8BD
:10B200001040044840F2111144F0C0BC10BD00BF12
:10B210008759002043D10500A2B8050008B50F4AA0
:10B2200000231278FFF766FF10F1160F08D00C4BC1
:10B230000022072800DD08BD98601A610130F8E798
:10B24000084909484FF4987244F0C6F9BDE808402F
:10B2500004484FF4987144F099BC00BF875900200E
:10B2600090ED00E043D10500A2B80500204910B5DB
:10B270000C68082C0DD91F491F484FF4A47244F0E4
:10B28000ABF91C484FF4A47144F080FC4FF0FF3040
:10B2900010BDFFF79DFF486818490022944200F155
:10B2A0000C0015D1164B1C70FFF788FF0B68C3F319
:10B2B0000723082B0AD00F490F484FF4D47244F0EB
:10B2C0008BF90C484FF4D47144F060FC0020DFE7A8
:10B2D0008A6050F80C3C23F01F03134343F0100323
:10B2E000CB6050F8043C43F001030B610132D5E719
:10B2F00094AB050043D10500A2B8050090ED00E035
:10B3000087590020014B1860704700BF38010020AA
:10B310000CB41FB509B90DF10300CDE9020107AB6B
:10B32000069A0648019302A9FAF72AFA029B00221C
:10B330001A7005B05DF804EB02B07047E515050022
:10B340000EB40FB505AB6FF0004153F8042B02901B
:10B3500003910648019302A9FAF712FA029B002210
:10B360001A7004B05DF804EB03B07047E5150500F2
:10B370004FF04003EFF3118283F31288BFF36F8F16
:10B3800006490123C1F840354FF08041C1F87835B6
:10B3900082F31188BFF36F8F0020704700E00140F7
:10B3A0004FF08043C0B2C3F81C05BFF34F8F05496F
:10B3B000054BCA6802F4E0621343CB60BFF34F8FC2
:10B3C00000BFFDE700ED00E00400FA0520B1034BEB
:10B3D000800143F001031847704700BF10A5050026
:10B3E0008379074A342101FB03231A6B93F8243035
:10B3F0001733801A23F00303B0FBF3F0704700BF4C
:10B40000B008002010B50A4A8379342404FB0323D2
:10B410000A68DB6A5C6823689A4294BF0A600B6022
:10B42000FFF7DEFFD4E9002302FB003010BD00BFB0
:10B43000B008002010B54379044643B10C490D48CB
:10B44000562244F0C9F80A48562144F09FFB23686D
:10B4500043B107490748572244F0BEF80448572132
:10B4600044F094FB0023A3812369A36010BD00BFB7
:10B470008DD10500A2B805002DE9F74F05460191D1
:10B480001046194616461F464BF038F981468A4643
:10B4900045B96B496B48F42244F09EF86848F421A2
:10B4A00044F074FB05F11C084FF04003EFF3118BDF
:10B4B00083F31288BFF36F8F404617F051FD40B9F8
:10B4C00061496048812244F087F85F48812144F057
:10B4D0005DFB404617F062FD6B8C002B77D02A8C09
:10B4E0009A424DD900220023284618F0E9FA044672
:10B4F000002845D0404617F041FD40B95249514817
:10B50000AC2244F069F85048AC2144F03FFB8BF387
:10B510001188BFF36F8FDDF80480B8F1000F00F0E1
:10B520008B8056EA070310D07B1C08BFB6F1FF3FA3
:10B530000BD01AF019FBB9EB00066AEB0107002EDD
:10B5400077F10003BCBF00260027A379DFF8FC9049
:10B550004FF0340A0AFB03933246DB6A1B6801A9E9
:10B560001D6820463B46A8470546206100284BD170
:10B57000A079214600FB0A904BF01AF82C463FE0D8
:10B580006C8C631E6B84404617F0F8FC40B92E4962
:10B590002C48AC2244F020F82B48AC2144F0F6FAB9
:10B5A0008BF31188BFF36F8F2B8C95F824201C1B15
:10B5B00002F117002B6B20F0030004FB003423483A
:10B5C000234BE2712D1AAD105D43A571A3E74046F0
:10B5D00017F0D4FC40B91C491A48AC2243F0FCFFD8
:10B5E0001948AC2144F0D2FA8BF31188BFF36F8F66
:10B5F00032463B46284618F063FA044600288AD1B2
:10B60000204603B0BDE8F08F019B98450AD90C494C
:10B610000C4840F2551243F0DFFF094840F2551143
:10B6200044F0B4FA002323600123A380019BE3814B
:10B630002046FFF7FFFEE3E7C4F81080F2E700BF03
:10B640008DD10500A2B80500DCB80500B0080020C7
:10B65000C54EECC42DE9F041054628B31C4E002729
:10B660004FF034082C462D682379013BDBB223715F
:10B67000C3B9216959B163799B0707D4A37908FB42
:10B6800003632046DB6A1B689B6898472761A079A3
:10B69000A76008FB006327609B6A93B12046984728
:10B6A000002DDFD1BDE8F0810A490B484FF4047248
:10B6B00043F092FFBDE8F04106484FF4047144F0B6
:10B6C00065BA214600FB08604AF072FFE8E700BF58
:10B6D000B00800208DD10500A2B8050010B50446C1
:10B6E00050B9084908484FF41F7243F075FF0548E8
:10B6F0004FF41F7144F04AFA20462468002CFBD115
:10B7000010BD00BF8DD10500A2B8050038B50D46AB
:10B71000044650B90F49104840F2872243F05CFFBD
:10B720000C4840F2872144F031FA55B909490A48DA
:10B730004FF4227243F050FF06484FF4227144F058
:10B7400025FA236823B12846FFF7C8FF2368036062
:10B75000256038BD8DD10500A2B8050083888B42D5
:10B7600070B5066804460D460AD20949094840F2F8
:10B77000834243F031FF064840F2834144F006FA29
:10B78000A38821685B1B2944A3802160304670BDDB
:10B790008DD10500A2B8050070B5036886880446FF
:10B7A0000D461E4445F04FFF88420AD2074908481B
:10B7B0004FF44A7243F010FF04484FF44A7144F0CA
:10B7C000E5F9A1880D44A580304670BD8DD10500F6
:10B7D000A2B8050038B50D46044650B90D490E48CB
:10B7E0004FF4F97243F0F8FE0A484FF4F97144F04F
:10B7F000CDF92368BFF35B8F012202FA05F10C3308
:10B8000053E8002F0A4343E800200028F8D1BFF393
:10B810005B8F38BDB9D10500A2B805002DE9F74FFF
:10B820000192002854D00026051D37464FF0280EFF
:10B8300048F2FE0A0EFB0704264A636A23F07F43A0
:10B8400023F47D0323F0FF0393422CD135F8043C0D
:10B85000022B28D1A388534525D001F1FF3905F1EA
:10B86000FF3B002319F8018F1BF8014FA04503F19E
:10B87000080C20D15FFA8CF3802BF3D1019A147855
:10B880009C4210D80EFB070494F82640620707D5A7
:10B890003F2B05D80C78FF2C05D14C78032C02D116
:10B8A000019A2E46137028351FB1304603B0BDE80B
:10B8B000F08F0127BEE788EA04045FFA8CFC2206B9
:10B8C000DCD40133DBB264009C45E4B2F7D1D5E7A8
:10B8D0000646EAE700010200014817F0C9BF00BFB1
:10B8E000C807002002460B46014817F0E9BE00BF1A
:10B8F000C80700202DE9F84F45F0A0FF4FF0FF31B9
:10B9000007464FF0FF30FFF7EDFF254B1B68002B7C
:10B9100041D0B3F1140A3ED01C6804B1143CDFF8E6
:10B9200080904FF0FF364FF002080AF1140B3946B1
:10B93000584646F0FDF80546A8B959468AF82580CC
:10B94000484645F015FF2A462946584646F0D0F8A5
:10B9500074B114F1140302D0636903B1143B3CB118
:10B96000A2461C46E1E7864228BF0646A245EFD123
:10B97000731C10D04FF4004440F2E73000214FF424
:10B980007A720023E4FB0601F4F7D8FF02460B4667
:10B99000044818F03DFDBDE8F84FFFF79DBF00BF1C
:10B9A00058290020A816002070B54FF0FF31054639
:10B9B0004FF0FF30FFF796FF1E4B1A6852B1136825
:10B9C000002B38BF00234FF0FF314FF47A7642B995
:10B9D0004B1C1BD1184818F021FDBDE87040FFF743
:10B9E0007BBFD069128C401B06FB0202002A0CDDD3
:10B9F000914228BF114633B11C68002C38BF002487
:10BA00001A462346E3E71C46FAE700214FF40040BC
:10BA100040F2E7340025E0FB01454FF47A72002341
:10BA200020462946F4F78AFF02460B46024818F0E2
:10BA3000EFFCD2E76829002008170020F8B545F090
:10BA4000FDFE4FF0FF3105464FF0FF30FFF74AFF94
:10BA50001C4A136833B92846FFF7A6FFBDE8F84033
:10BA6000FFF73ABF19680024002938BF00214FF4BE
:10BA70007A7EA446D869461B188C0EFB006000280D
:10BA80001F460FDC1868BCB9566810609E4200D192
:10BA9000506093F82200C3F800C06CF3000083F8F4
:10BAA000220027460029D6D0086800280B463C46CD
:10BAB000014638BF0021DDE720605068984208BF8A
:10BAC0005460E6E76829002070B505460E464FF041
:10BAD000FF304FF0FF31FFF705FF0721284645F003
:10BAE000BDFEC0B16B6873B126B90024FFF7F4FE48
:10BAF000204670BD3360F8E76B60C3F8F850002E45
:10BB0000F3D03360F2E7054BD3F8F840002CF3D0C4
:10BB10006FF00204EAE76FF08504E7E77029002080
:10BB20002DE9F04706460F464FF0FF304FF0FF314A
:10BB3000DFF88C80204DDFF88C90FFF7D3FEC246F3
:10BB400045450AD91D48494640F29C5243F044FD00
:10BB500040F29C51484644F019F8554501D3002461
:10BB600023E06C680CB90835EAE794F826309A07A8
:10BB700008D52388022B05D18022211D304645F0AF
:10BB800030FEB8B994F84E309B07ECD5238D022BCC
:10BB9000E9D1802204F12C01304645F022FE002834
:10BBA000E1D0282307B13D601C44FFF795FE2046F5
:10BBB000BDE8F0870023F5E718090020A2B80500CA
:10BBC00020090020E1D105002DE9FF4107460D467F
:10BBD00051B93749374840F2CA6243F0FDFC344856
:10BBE00040F2CA6143F0D2FF4FF0FF304FF0FF3117
:10BBF000FFF778FE7C6844B194F8263099070AD4A0
:10BC000094F84E309A070ED40024FFF765FE2046C4
:10BC100004B0BDE8F0812946201D45F007FE00284C
:10BC2000EED0002607E0294604F12C0045F0FEFD89
:10BC30000028E9D0012628217143631893F82630A3
:10BC4000DB070CD4DFF8748014312144404645F002
:10BC50008FFDD8F8003013B9174818F0DFFB282300
:10BC600003FB064494F826306FF3410384F8263032
:10BC700040F2FF2300930023ADF80430ADF8063006
:10BC8000ADF808304FF48073ADF80A30FF238DF81B
:10BC90000C306B7BEA7B8DF80D30AB7B43EA0223E3
:10BCA000ADF80E306946384645F003FE0124ACE796
:10BCB000E1D10500A2B80500A816002058290020EF
:10BCC000F7B545F0BBFD4FF0FF3107464FF0FF30B1
:10BCD000FFF708FE244B1C68002C3FD02568002D80
:10BCE00038BF00254FF0FF363946204645F020FF8B
:10BCF000E0B994F8253060F3410384F82530206AD8
:10BD000001A9FFF7E1FE002807DB94F82430019930
:10BD1000206A04F1100245F0FCFD1DB32B68002BD6
:10BD200038BF00232C4635B11D46DDE7864228BFCB
:10BD30000646AC42F1D1731C10D04FF4004440F2DF
:10BD4000E73000214FF47A720023E4FB0601F4F798
:10BD5000F5FD02460B46054818F05AFBFFF7BCFDFF
:10BD600003B0F0BD2B46DDE760290020D816002087
:10BD70002DE9F74F81460E464FF0FF304FF0FF316F
:10BD8000FFF7B0FD244DDFF898A0DFF898B05545D7
:10BD90000AD92248594640F2B97243F01DFC40F2DC
:10BDA000B971584643F0F2FE1D4B9D4201D3002469
:10BDB00026E02EB133681BB1AB4201D00835E6E76F
:10BDC0006C68002CFAD004F154010027182303FBFF
:10BDD00007F804EB080292F86420D20716D531F870
:10BDE000042C022A12D180224846019145F0F9FC28
:10BDF0000199182350B106B1356008F15008444448
:10BE0000FFF76AFD204603B0BDE8F08F0137032F2E
:10BE100001F11801DBD1D1E718090020A2B8050013
:10BE200020090020E1D105002DE9F7430D4600234C
:10BE300004464FF0FF314FF0FF308DF80730FFF729
:10BE400051FD2A8848F2FE039A422FD02B78FF2B0F
:10BE500002D16B78022B29D014B360680DF1070270
:10BE60002946FFF7DBFC044618E070680DF1070275
:10BE70002946FFF7D3FC0836002818BF0446BE4207
:10BE80000AD91F48414640F6782243F0A5FB40F608
:10BE90007821404643F07AFE4E45E6D32CBB21E0A4
:10BEA000184F194EDFF86480B946E8E71CB301214A
:10BEB000204645F077FDD6E70121284645F072FD82
:10BEC000044690B90835B5420AD90D48394640F6BE
:10BED000872243F081FB40F68721384643F056FE27
:10BEE0004545E9D300F05AF90446FFF7F5FC204632
:10BEF00003B0BDE8F083034E034D044FB046E2E7C4
:10BF0000A2B805002009002018090020E1D1050091
:10BF1000F8B505460E464FF0FF304FF0FF3117469B
:10BF2000FFF7E0FC0C4B1B681BB9BDE8F840FFF7BE
:10BF3000D3BC1C68002C38BF00245B683A463146ED
:10BF400028469847002CF0D02268002A38BF0022EB
:10BF500023461446F1E700BF6C2A0020F0B5002309
:10BF600085B0CDE9003305460C4600293BD01F4B78
:10BF70001B68ABB1496C94F8482089B1062A0FD8E8
:10BF80000DF10A0630468DF8092045F014FB9DF8A6
:10BF900009308DF8043094F8493000968DF805305A
:10BFA00000212846676945F059FCC8B1284645F08C
:10BFB000FAFB2146436828469847061E02DA2046C7
:10BFC00045F05BFF1FB13146384645F0F1FB009B61
:10BFD00023B1324669462846FFF79AFF012003E065
:10BFE0006FF07206EBE7084605B0F0BD6C2A002042
:10BFF00038B54FF0FF3105464FF0FF30FFF772FCC8
:10C000000021284645F02AFC20BB284645F0CBFB02
:10C01000044630B1846824B101212846A047041E9B
:10C0200014DB2B681B6953B90C490D4840F6B572F7
:10C0300043F0D2FA094840F6B57143F0A7FD28460F
:10C040000021FFF7C7FB284645F0BEFBFFF744FC85
:10C05000204638BD6FF07704F8E700BFE1D1050056
:10C06000A2B805002DE9F8434FF0FF314FF0FF3043
:10C07000FFF738FC274C284FDFF8CC8046F0BDF89E
:10C08000A1463E46BC420AD92448414641F2CF026D
:10C0900043F0A2FA41F2CF01404643F077FDB442AB
:10C0A00029D31F4B1F4AA3EB0903DB08964238BF75
:10C0B0000023E3B11C491D481D4C18F0B3F81D497D
:10C0C0001D4818F0AFF8402384F8F43047F230539D
:10C0D000C4F8E830204645F09FFC1849C4F8EC004D
:10C0E000174818F09FF8174B0022C3E90022BDE85B
:10C0F000F843FFF7F1BB23681B689D6845B12B68C7
:10C1000033B120460721FFF765FB2B68204698478F
:10C110000834B7E71809002020090020A2B805005C
:10C120002709002011090020F5B80000A8160020FA
:10C1300070290020C1BC0000D81600203DBA0000C4
:10C140000817002068290020E1D10500F8B50F4D3F
:10C150000F4C104E2F46AC420AD90F48314641F2DF
:10C16000011243F039FA41F20111304643F00EFD5D
:10C17000BC4200D3F8BD0321204645F06FFB10B947
:10C180002046FFF735FF0834E5E700BF200900200F
:10C1900018090020E1D10500A2B805000048704749
:10C1A000C0AB050002484FF0FF3201214AF00ABA45
:10C1B000742A002073B5044616461D464AF0AEF9AF
:10C1C00008B1002635462B46324601A9204616F016
:10C1D000D1FD0546D8B901466022019845F0F6F92F
:10C1E0000198FF2180F85B100A49446001228C42CB
:10C1F000826306D180F8562045F095FE019802B082
:10C2000070BD054A944208BF80F85650F4E70020FC
:10C21000F5E700BF7C0700205C07002002460B46C4
:10C220000148FFF7C7BF00BF7C0700202DE9F74F8B
:10C23000DDE90C6705468A463046394693464AF0A2
:10C240005DFA80468946BAF1000F09D1BBF1000FB3
:10C2500006D195F84F3013F00E0FC3F342005AD0B9
:10C260004AF05CF908B100260027284645F02FFE69
:10C2700095F84F30002851D113F00E0FC3F342024E
:10C280004ED0022A14BF00242824BBF1010F02D093
:10C29000BBF13A0F00D10434C3F34202AB69A244AC
:10C2A0000BB11B681B8B022A3CD1B3F5A06F38BFC2
:10C2B0004FF4A0631C1A3749374B6868374A544516
:10C2C00028BF544688420CBF92469A4656EA070356
:10C2D00010D0791C08BFB6F1FF3F0BD019F044FC19
:10C2E000B8EB000669EB0107002E77F10003BCBF35
:10C2F00000260027304639464AF000FA8B460021D6
:10C300008146884684B9B8F1000F19D028464146C5
:10C3100045F01DFE002003B0BDE8F08F0024BBE710
:10C320000446B9E75346C5E73B46324650460191BD
:10C3300045F084F90199034628B9B8F1000F25D1D9
:10C340006FF00B00E7E7B8F1000F00D1E1B10B602F
:10C35000DA89A24288BFDC81DA89A41A56EA070288
:10C3600010D07A1C08BFB6F1FF3F0BD0019319F033
:10C37000FBFBB9EB00066BEB0107012E77F1000325
:10C38000019BC0DB1946BDE78046E1E74046FFF769
:10C3900061F9D5E77C070020B0080020E408002000
:10C3A00030B585B0DDE908450093CDE90245134677
:10C3B0000A460146024845F0DBFD05B030BD00BF2E
:10C3C0007C07002030B585B0DDE908450093CDE954
:10C3D000024513460A460146024845F0C9FD05B02C
:10C3E00030BD00BF5C070020034B4FF4907202FB8E
:10C3F00000304AF0D2B800BF38170020024B07289F
:10C4000088BF0020185C704714D2050030B58BB08F
:10C41000154C20464AF0B4F84FF0FF324FF0FF338E
:10C42000CDE9062300254FF0FF33CDE90335009415
:10C4300004F12000CDE901550C4B0D494FF4BC62CD
:10C4400016F0EAFE044660B10A4A2B46082108A805
:10C4500043F0CFF808A9204616F038FD20464AF0F0
:10C4600065F80BB030BD00BF38170020DB21050098
:10C4700080D500200BD20500034B1A6802605A6871
:10C48000186002B9586070478C2A002073B50022EA
:10C4900004230E466946CDE90023054645F079FEA2
:10C4A000044610B9022002B070BD3A21284645F07A
:10C4B00096FB0028F6D10199284645F099FD0C4BD2
:10C4C0001B68002B38BF0023002BEBD0197A227891
:10C4D00091420BD15A7A6178914205D15B6822462C
:10C4E000314628469847DEE7002AF7D01B68EBE77D
:10C4F0008C2A00200148FFF7BFBF00BF3C0100208D
:10C500002DE9F04F2DED028B282387B00026CDE9D1
:10C51000046383690393836804460F463BB904A907
:10C52000204645F036FE054628B902209FE09A894C
:10C530001B681644F2E783884FEA032848EA132869
:10C540001FFA88F808F12808B045EEDC03DA414606
:10C55000204645F0C1FDAB6833B9EB6823B92B69C0
:10C5600013B96B69002BE0D02B7AFF2BDDD0297E2D
:10C57000FF2905F1180602D16B7E002BD5D0F7B943
:10C58000304645F08BFF0028CFD105F1080045F07B
:10C5900085FF0028C9D1FF2902D16B7E012BC4D0B1
:10C5A000FFF7FCFD0146304645F086FF38B12B7E93
:10C5B000FF2B04D16B7E052BB7D0082BB5D0AB7900
:10C5C00084F85B30282384F84C300021A368A4F859
:10C5D00054109B68DB7984F8523094F84F30022273
:10C5E00062F3430384F84F302B7EFF2B13D16B7E15
:10C5F000012B18D0022B04D18249304645F05CFF54
:10C6000088B903A93046FFF7B3FB00288DD0037D1E
:10C610009B0708D489E73046FFF782FA002884D0C8
:10C620002B7EFF2BE3D00599204645F0E1FCAE7947
:10C630002C2E26D020D83EB32B2E08BF4FF0040955
:10C6400018BF4FF000090623A4F858304FF0000B34
:10C650003A2E03D0112E01D0062E18D13A2EA4F86E
:10C6600054B07FF462AF29462046FFF70FFF07B0B2
:10C67000BDEC028BBDE8F08F3C2E08BF4FF00209E5
:10C68000DEE74FF00809DEE74FF00109DBE73B2E5C
:10C690003FF44BAF204645F030FD012200900DF1F4
:10C6A0000901204645F0BAFC00287FF43EAF9DF812
:10C6B00009302C2B1ED015D8F3B12B2B0CBF04271F
:10C6C000002719EA070F07D12C2B1DD018D81BB152
:10C6D000112B19D0062B17D0204645F00EFD012254
:10C6E000431E88E03C2B09D119F0020F0CBF022732
:10C6F0004027E6E70827E4E70127E2E70746E0E707
:10C70000A3F13B02012A7BD80EB13C2EE4D10023D9
:10C710000DF10B01012220468DF80B3045F07EFC17
:10C720001FFA88F60DF10B0100287FF4FEAE9DF88C
:10C730000B300133B6EBC30F4FEAC30AFFF4F5AE7B
:10C7400008EE101A0226204645F0D7FC012201907F
:10C750000DF10A01204645F061FC00287FF4E5AEAA
:10C760009DF80A20019BFAB99DF80A203AB3012AE4
:10C770009DF80B1026D0AAF1040081423FF7D5AEF8
:10C7800002F0C002802A35D0C02A2FD0002A7FF4C0
:10C79000CCAE204645F02CFC00287FF4C6AE9DF8B8
:10C7A0000B301E4402360BE018EE101A0122204610
:10C7B000019345F033FC019B0028D5D0B5E6013646
:10C7C000B6B205E00E4402362046B6B245F010FC83
:10C7D000B245B8D89DF800009DF80960A4F858004B
:10C7E000D34449EA07091FFA8BFB31E72A7EFF2A67
:10C7F0003FF49BAE02220421204645F084FD94E6DE
:10C800003A2B68E7F0AB05002DE9F04187683B68FB
:10C8100004460D46164643B9074908484B2242F0E4
:10C82000DBFE05484B2143F0B1F93B68324629460F
:10C830002046BDE8F04118471CD20500A2B805000B
:10C840001A4B2DE9F3411D6807460E4614469846DB
:10C850007DB9174815F0E2FF054640B9154916485D
:10C860003C2242F0B9FE13483C2143F08FF9C8F84E
:10C870000050B2B239462846FFF7C6FF002802DA58
:10C8800014B9A64203D8002002B0BDE8F081351BE0
:10C89000042D28BF042546F07AFA2A46019001A902
:10C8A000381944F088FE2C44EBE700BF942A00209E
:10C8B00049D205004DD20500A2B8050037B5104D8C
:10C8C0002C6874B90F4815F0A9FF044640B90E4909
:10C8D0000E481A2242F080FE0B481A2143F056F906
:10C8E0002C6004220DEB02012046FFF78DFF00288B
:10C8F00002DA46F04CFA0190019803B030BD00BF57
:10C90000942A002049D205004DD20500A2B80500A6
:10C910002DE9F0410E4C051BC5F347130C255D4373
:10C92000074605F148000E462044402145F065FECB
:10C93000011E08DB074B2C44C4E91036064B5B593B
:10C94000BDE8F041184738463346BDE8F041184786
:10C95000A82A00205D2605002CAC050038B5CCB215
:10C96000012C054608D908490848792242F034FECE
:10C970000548792143F00AF92B690C2104FB0134A5
:10C98000A06C00F0070038BD86D20500A2B80500F3
:10C99000F8B5CCB2012C0769054616460AD91849E4
:10C9A000184840F24D1242F017FE154840F24D1162
:10C9B00043F0ECF84FF04003EFF3118283F3128859
:10C9C000BFF36F8F0C2303FB0471896C11F0C0015E
:10C9D00001D08E4211D103FB047301219964002020
:10C9E00082F31188BFF36F8F30B969680C2303FBA2
:10C9F0000414636898470020F8BD4FF0FF30EFE75C
:10CA000086D20500A2B8050070B50D460649411A48
:10CA10000446491105484022FFF7BAFF2B4601465C
:10CA20002046BDE870401847A82A002090A10500C4
:10CA3000002270B5012104461046FDF791FD00204B
:10CA4000FDF75CFD0F4809F0ABF90F4B984215D18B
:10CA500046F0A8FB26690D49304642F033FE002817
:10CA60000BDB0125B5642469084904F1200042F07C
:10CA700029FE002801DB6565002070BD6FF0040011
:10CA8000FBE700BFCDCA00000000AD0B74AC050091
:10CA900073B50C2301460B484B43C418D4E910521C
:10CAA0000026483326641844019245F0C4FD35B190
:10CAB000019A05482B4602B0BDE87040184702B005
:10CAC00070BD00BFA82A002090A10500012808B56C
:10CAD00006D0032808D0A0B90F4B9B6C5B0719D177
:10CAE000BDE80840FFF7D4BF0C490D4840F25E2274
:10CAF00042F072FD40F25E21BDE80840074843F075
:10CB000045B80649064840F2622242F065FD40F20F
:10CB10006221F1E708BD00BFA82A002086D20500E7
:10CB2000A2B8050010B549F0E3FD4FF47A730C4646
:10CB3000A0FB030103FB0411054AC30B43EA414375
:10CB4000BDE81040C90B0120C2E9003109F0EEB880
:10CB50005818002008B54FF04003EFF3118183F31C
:10CB60001288BFF36F8F114A136843F0020013F06D
:10CB7000010310600CD04FF08042D2F80C34D2F890
:10CB80000C2413F0010303D0094845F054FD0123A0
:10CB900081F31188BFF36F8F23B1BDE808400020F7
:10CBA000FFF776BFBDE80840FFF7BCBF002B0020B1
:10CBB000F02A002010B549F09BFD4FF47A730C4623
:10CBC000A0FB030103FB0411054AC30B43EA4143E5
:10CBD000BDE81040C90B0120C2E9003109F0C8B816
:10CBE00060180020084BBFF35B8F53E8002F22F042
:10CBF000020143E800100028F7D1BFF35B8FD30791
:10CC000001D4FFF7D7BF7047002B00202DE9F74F65
:10CC10004FF080470446D7F8186406F480364FF08A
:10CC20004003EFF3118883F31288BFF36F8F49F04D
:10CC30005FFD4FF47A730A46A0FB030103FB021168
:10CC4000D7F80C94D7F80C34254BD3F800B0254B0B
:10CC5000C50BD3F800A045EA414588F31188BFF31E
:10CC60006F8F214ADFF89880204F2046082143F03B
:10CC7000DEFC19F0010FDFF88C901D4AB9F81E3068
:10CC80000093204614BF43463B46082143F0CFFCA7
:10CC9000A5EB0B03009320465B46164A0821A5EB43
:10CCA0000A0543F0C4FC53462046134A0095082168
:10CCB00043F0BDFC2046114A082143F0B8FCB9F806
:10CCC0003E30009320460A4A002E14BF43463B469E
:10CCD000082143F0ACFC002003B0BDE8F08F00BF9A
:10CCE0005818002060180020C8D20500C3D20500E3
:10CCF000D3D20500EDD205000FD3050030D30500D7
:10CD0000CFBF0500A82A00207FB500220123CDE96E
:10CD1000022304ABCDE90433094ACDF800D06B46B9
:10CD2000CDF804D045F0ACFC002805DB4FF4804280
:10CD30000023684616F05AFF07B05DF804FB00BFF9
:10CD40007B260500024BC0B203EB4010704700BFCA
:10CD5000A82A00202DE9F8434849BFF35B8F054618
:10CD6000012251E8003F41E800200028F9D1BFF33B
:10CD70005B8F9BB9424943484B60CB608A60F8F7B0
:10CD800097FA00280ADA404940484FF4087242F006
:10CD900023FC3D484FF4087142F0F8FEADB36B1E22
:10CDA000012B56D8012D07D14FF08043D3F81C3406
:10CDB00003F00303012B28D049F0B0FB044618B957
:10CDC000334B1B78002B51D14FF04003EFF311860A
:10CDD00083F31288BFF36F8F01242E4FDFF8B880E2
:10CDE000DFF8B8904FF08042D2F81834D2F8182407
:10CDF000D2030CD503F00303012B01D0012D06D182
:10CE00000CB386F31188BFF36F8FBDE8F883ACB124
:10CE10003046FDF7DBFA4FF08042D2F81835002B90
:10CE2000E0D139680029DDD03B603B680123C2F8BE
:10CE30001835C8F88031C9F80030D3E70021212027
:10CE400018F0B2FAE7E74FF080430222C3F8042358
:10CE5000DBE70D490D4840F2322242F0BDFBBDE850
:10CE6000F843094840F2322142F090BE4FF080432F
:10CE70000222C3F808230646AFE700BF042B0020B8
:10CE8000982A0020C82A002086D20500A2B80500F2
:10CE9000616800200401004000E100E0080000405B
:10CEA00038B543681B69D3F84035994205460C46AE
:10CEB0000AD3074907484FF49B7242F08DFB0448A0
:10CEC0004FF49B7142F062FE2B6900209C6038BDDC
:10CED0007ED30500A2B805002DE9F84F43681B6911
:10CEE000D3F840210446D2B1D3F80423D20316D597
:10CEF000026915680022C3F84021D3F8403155B9C2
:10CF0000324933484FF4A27242F066FB2F484FF487
:10CF1000A27142F03BFE236920465968A8470025CC
:10CF20004FF480382E464FF0010947E0E9B28B1CE0
:10CF3000DBB24FEA830C12690CF5A07C08FA03FA05
:10CF400052F80C0000283FD0D2F804031AEA000F70
:10CF500014BF4FF0010E4FF0000E2069C76809FAA8
:10CF600003FB0BEA070757EA0E0726D042F80C60CE
:10CF70006FEA0B0B0C3052F80C70BFF35B8F50E86C
:10CF8000007F07EA0B0740E8007CBCF1000FF6D1F8
:10CF9000BFF35B8F6068C2F808A3C06850F83570B3
:10CFA00040F8356000EBC50C3FB103F5A87320468F
:10CFB00052F82320DCF80430B84701356268537A10
:10CFC000AB42B3D8BDE8F88F8646C6E77ED30500EE
:10CFD000A2B805002DE9F74F0C464168D2F804A02D
:10CFE000CB680969D1F840158A4506460FFA84FBDB
:10CFF00003EBC40000F2B78053F83B10002940F067
:10D00000B580116843F83B10936843607368D2F8A9
:10D010000C801B693269D3F8403592689A4208D374
:10D02000544955488B2242F0D7FA52488B2142F09E
:10D03000ADFD08F001030093736802341F695FFAC5
:10D0400084F94FF4803303FA09F30193D7F840557C
:10D05000019AD7F804334C46A4001A4204F5A07490
:10D0600008D044494448982242F0B6FA41489821F1
:10D0700042F08CFDD6F804C0DCF81010012307EB59
:10D0800089004B64D1F844E5D0F84035C0F840E55C
:10D0900000233B513B59009B002B3FD033699A68DA
:10D0A000C8F34004AA1A5346C0F84035012048642A
:10D0B00028180542D1F8441503F1FF3343D15B1A18
:10D0C0002B409A424AD2009B002B0CBF00206FF0ED
:10D0D0003D00002C3DD03369BFF35B8F012202FA83
:10D0E00009F90C3353E8001F41EA090143E8001431
:10D0F000002CF7D1BFF35B8F73681B69190B43F3E7
:10D100000733002B07DB01F01F015B098A40403326
:10D110001A4941F8232003B0BDE8F08F6A08924510
:10D1200005F1010832BF012400242A4618EA050F40
:10D130000AEB0E0301D12B40B6E7A5EB0E0EF2452C
:10D1400088BF5B1BB0E78B4236BF451A5B1A5B1981
:10D15000B7E7DCF80C3043F83B40DCE7019BC7F84D
:10D1600004330020D7E76FF01500D4E76FF00F000D
:10D17000D1E700BF7ED30500A2B8050000E100E0C2
:10D1800008B5084B0848186049F081F938B10748DC
:10D19000FEF7B8F80548F7F763FE002008BD6FF00A
:10D1A0001200FBE7282B002020A20500B1D10000CF
:10D1B0000A2838B5074D044604D1286883680D2134
:10D1C0005B68984728688368E1B25B6898472046A7
:10D1D00038BD00BF282B0020034B044A0020C2F8B2
:10D1E000043583F8300070478859002000E0004083
:10D1F000024B002083F83000704700BF88590020A0
:10D20000012A70B50BD1CA8B940608D58A8B102AD7
:10D2100005D19DF81000012801D1012B0FD01F4925
:10D220000B68580708D01E4B1E48C91A8908890187
:10D2300041F0010142F013FE6FF0150070BD8D68E2
:10D240005DB916490B685A07F6D0154B1648C91A2E
:10D250008908890141F00101ECE7144890F8304059
:10D260007CB10E490B685B0708D00D4B1048C91AFA
:10D270008908890141F0010142F0F1FD6FF00F00D2
:10D28000DCE70C4E80F8303085424E600B7002D0E7
:10D29000294644F090F92046D0E700BFF806002068
:10D2A000E8060020DCD3050025D4050088590020BD
:10D2B00035D40500B9D200004A68102A10B50C46D2
:10D2C0000FD028490B68580708D0274B2748C91AA0
:10D2D0008908890141F0010142F0C1FD6FF015009C
:10D2E0003FE0CB680F2B0BDC1E490B685A07F5D0CB
:10D2F0001D4B1F48C91A8908890141F00101EBE75C
:10D3000009681C48814201D044F055F91A4A0021AD
:10D3100011601368194B19601968194901200860D8
:10D32000116811B919680029FAD01B687BB10D4941
:10D330000B685B0708D00C4B1248C91A8908890191
:10D3400041F0010142F08BFD6FF0040009E0A0689C
:10D350000D49884202D0102244F02DF96368236100
:10D36000002010BDF8060020E806002047D4050084
:10D3700069D405009859002000E1004004E1004014
:10D3800000E0004081D40500A859002070B505696F
:10D3900016460C4641B91E491E48242242F01CF98B
:10D3A0001B48242142F0F2FB636843B9184919482D
:10D3B000252242F011F91648252142F0E7FB6B685F
:10D3C0005BB100229C4213D123685AB9AA686B60F2
:10D3D000944200D1AB600023236076B9002070BD79
:10D3E0000B46EFE71360AB689C4208BFAA60F2E708
:10D3F00019681A460029F3D13EB16B682360A8680A
:10D400006C600028EAD1AC60E9E76FF01500E6E750
:10D41000A8D40500A2B805002DE9F843430903D0BC
:10D42000012B30D0BDE8F883184F3B695C68002CB5
:10D43000F8D02568DFF85C80DFF85C9000F01F0012
:10D440000126002D06FA00F638BF0025A3681E420B
:10D4500010D0636843B941464846452242F0BCF8C3
:10D460004521404642F092FBD4E901322146324048
:10D4700038469847002DD5D02B68002B38BF0023A5
:10D480002C461D46E2E7024FCFE700BFA8A10500EA
:10D49000C0A10500A8D40500A2B805007FB540686A
:10D4A000057B01F01F04B2F5005F44EA45144FF01C
:10D4B000000504D120460FF0ABFA002052E0B2F58F
:10D4C000804FCDE902554FD1B3F5003F0CBF042387
:10D4D00005238DF80830836823FA01F111F001016A
:10D4E00053D1B2F5A03F50D1660948D040F2FF3386
:10D4F000012E08BF194604F01F05E940CA070AD4E7
:10D500002A492B4840F2292242F066F8274840F287
:10D51000292142F03BFB66B1012E33D02349244838
:10D5200040F22E2242F058F8204840F22E2142F0DC
:10D530002DFB4FF0A04305F5E07553F82530DB07D0
:10D5400023D40DF10705294620460FF095F9194B14
:10D55000984219D128460FF0EBF9174B984213D097
:10D560006FF00B0004B070BDB3F5C02F05D0B3F55C
:10D57000003F0CBF02230123ABE70323A9E74FF0D1
:10D58000FF31B8E70D4BD6E703950023194602AAF1
:10D5900020460FF053F8084B984204D10121204651
:10D5A0000FF0CCF989E76FF00400DBE7D5D4050074
:10D5B000A2B805000400AD0B0000AD0B0003005045
:10D5C00010B50FF0A5F9044668B90FF079F9084BCA
:10D5D00098420AD1074821460FF048F92246052112
:10D5E0000620FCF7BDFF002010BD6FF00400FBE734
:10D5F0000000AD0B19D400002DE9F04347683B7BD8
:10D6000001F01F0585B00E4645EA43151446CAB918
:10D6100002A928460FF030F9044628460FF01AFAFE
:10D62000484B984204D06FF0040005B0BDE8F08389
:10D63000844205D19DF808000FF074F9A042F2D1A0
:10D640000020F2E74FF000090DF103013046CDE96B
:10D6500002990FF011F94B46804602AA4946284626
:10D660000EF0ECFF374B984202D06FF01500DCE76C
:10D67000804503D19DF803000FF054F9A3054ED562
:10D68000314B324A234093423AD00CD8062B14D067
:10D6900004D893B1022BE8D104230EE0B3F5801F28
:10D6A000E3D1012309E02A4A93422BD0B3F5A00F1E
:10D6B0002AD0B3F5800FD8D102238DF8043084F43A
:10D6C0008073C3F30023E0068DF8053054BFC4F324
:10D6D0004013032321058DF8063017D57B680121FF
:10D6E00001FA06F6C3F80865002201A928460FF0E2
:10D6F0004DF8144B984214BF6FF01500002094E7CA
:10D700000723DAE70523D8E70323D6E7620541BFFD
:10D710007B68012101FA06F6C3F80C65E4E7E3062D
:10D720004FF0000354BFC4F3401403241A4601A968
:10D7300028468DF804400EF081FF024B98423FF4DA
:10D740007FAF92E70000AD0B0600F000060010006E
:10D7500002004000014BB3F8A8067047800D00207E
:10D7600038B50B4DD5F8A04664B94FF47A704843EC
:10D77000C5F8A02645F09EFD38B9C5F8A0064FF0C3
:10D78000FF3038BD6FF07700FBE72046F9E700BFB8
:10D79000800D002008B545F062FD78B908490B6896
:10D7A0005B0708D0074B0848C91A8908890141F06E
:10D7B000010142F054FB6FF0040000E0002008BDBE
:10D7C0000C070020E806002016D5050008B545F036
:10D7D00049FD78B908490B685B0708D0074B084832
:10D7E000C91A8908890141F0010142F038FB6FF044
:10D7F000040000E0002008BD0C070020E80600201F
:10D8000031D50500F0B5144687B00A290DD8DFE8F8
:10D8100001F006163034380C0C0C0C0C3D0013785B
:10D8200043B1507820B1012802D06FF015001AE002
:10D8300045F04BFD207845F057FD002013E053796B
:10D84000117915683BB1284645F050FD0028F4D108
:10D850006FF00B0007E045B1284645F050FD002869
:10D86000EBD16FF0010007B0F0BD084645F04AFD6E
:10D87000E3E7107845F027FDDFE7107845F021FD5C
:10D88000DBE7214B1268C3F8A426D6E79768D38854
:10D89000ADF80C3004AEB74207F1080525D2AE4210
:10D8A0000AD21A491A4840F2172241F095FE174849
:10D8B00040F2172142F06AF92B46324613F8011D57
:10D8C00002F8011BBB42F9D1A38893B1012522685C
:10D8D0000095002103A845F0FAFCA3882268009572
:10D8E0002946304645F0F3FCA7E7DAD006AB9F4265
:10D8F000D6E71946012203A845F0F4FC012211469F
:10D90000304645F0EFFC98E7800D00204FD505002C
:10D91000A2B805002DE9F04315469A8906690C4620
:10D920001F469968931C85B0804686F80C36D2B2A3
:10D9300006F20D6043F03FFE06F2F459484616F039
:10D94000BFF9022C3AD013D9E31E012B46D9A04AC5
:10D9500013685D0709D09F4B9F48D21A9208920125
:10D9600042F00102214642F089FA6FF08505B1E0EC
:10D9700095F85E3004F00104C3F3800203A9C3F3F9
:10D98000C00306F20C608DF80C208DF80D308DF878
:10D990000E4008F0F7FF0446002C66D18C490B6856
:10D9A000580708D08B4B8D48C91A8908890141F066
:10D9B000010142F054FA6FF004058BE095F85E30F7
:10D9C00003A9C3F3800206F20C60C3F3C0038DF811
:10D9D0000C208DF80D3009F01BF8DCE755B98049B3
:10D9E000804840F22F2241F0F7FD7D4840F22F2180
:10D9F00042F0CCF8A4F1040C95F85E30DCF10004A0
:10DA000044EB0C04C3F38002C3F3C0038DF80C2075
:10DA10008DF80D308DF80E4045F00BFC4FF47A7206
:10DA20008DF80F000023D5E90C01F2F787FF03AB57
:10DA3000A0F57A714FF47A7206F20C6045F01FFC83
:10DA4000694BD3F8A4360446002BA5D060490B6877
:10DA500013F0060FA0D05F4B6448C91A89088901EA
:10DA600041F0020142F0FBF996E75F4BD3F8A43690
:10DA70001BB13A460021404698474FF0FF324FF025
:10DA8000FF33484616F0B2F896F8B03696F8B1264D
:10DA90009B0043EAC20395F85E2003F00C0322F0DA
:10DAA0000C02134385F85E3096F88C36052B82D82D
:10DAB00001A252F823F000BFDDDA0000D1DA000045
:10DAC000C3DB0000C9DB0000B7D90000C3DB0000E6
:10DAD0006FF00F05284605B0BDE8F083D6F89456E0
:10DAE000002DF7D02C78306800220023CDE90023E8
:10DAF00000231A462146FEF753FC074678B93449FD
:10DB00000B685A0708D0334B3948C91A890889016C
:10DB100041F0010142F0A3F96FF00B0547E0D6F8A0
:10DB200094162246013144F018FB00280FDA2849E8
:10DB30000B685B0708D0274B2E48C91A8908890152
:10DB400041F0010142F08BF96FF00B052CE096F8E3
:10DB50009C3687F85D3096F89D3687F85C30D6F8AD
:10DB60009816254AB1FBF2F30025C7E9083502FBF8
:10DB700013134FF47A7253433846BB6244F0D3F91F
:10DB80003068394603F076FDC8B111490B6803F0DF
:10DB90000703022B08D90F4B1848C91A89088901B5
:10DBA00041F0030142F05BF9384644F066F9D6F8DB
:10DBB000940608F007FF0023C6F894368AE7054666
:10DBC000F2E76FF0220585E76FF0680582E700BF96
:10DBD0000C070020E8060020E3D50500FCD5050071
:10DBE0007AD50500A2B80500800D0020B2D5050049
:10DBF0000ED6050028D6050040420F0045D6050088
:10DC00002DE9F74F3B4F3C4DDFF8F880DFF8F8A0E7
:10DC10007D1B0646AD084FF0FF334FF0FF3206F58F
:10DC2000976015F04DFF4368044643B9414650469E
:10DC3000BA2241F0D1FCBA21404641F0A7FF636807
:10DC400093F80090B9F1800F08D941465046C6229A
:10DC500041F0C2FCC621404641F098FF4FF0FF3230
:10DC60004FF0FF33CDE9002300231A4649463068C0
:10DC7000FEF7A8FB61684A460131834644F06DFA1D
:10DC8000814640BB237B8BF85D30637B8BF85C3037
:10DC9000A27B9BF85E3062F341038BF85E30A16893
:10DCA000164AB1FBF2F3CBE9083002FB13134FF431
:10DCB0007A7253433068CBF82830594643F022FD3E
:10DCC000002811DA3B685B0705D0A9010C4841F038
:10DCD000010142F0C4F8606808F074FE002363603C
:10DCE000584644F0CAF896E7606808F06BFEC4F83E
:10DCF000049090E70C070020E806002040420F0047
:10DD000069D605007AD50500A2B8050070B5466849
:10DD1000046988B0054604F5976048F031FC01229B
:10DD2000002104F2F45048F04DFC0122002104F5DA
:10DD3000BB6048F047FC08F0F7FD45F0EFFA82B20F
:10DD4000D301D10001F4816103F4807352020B43CB
:10DD500002F40062134343F42D731A4A43F00303A1
:10DD6000A2F8A83628463368984704F57075002253
:10DD70000023CDE9062300236FF00D02CDE9032334
:10DD8000CDE901330094104B4FF4487204F1800147
:10DD9000284615F041FA0D49284615F097F80C4928
:10DDA0000B6803F00703022B08D90A4B0A48C91A6B
:10DDB0008908890141F0030142F051F8002008B0C0
:10DDC00070BD00BF800D002001DC000085D605007D
:10DDD0000C070020E80600208DD605002DE9F04153
:10DDE0001F4F0646002418463D46D7F8D8348BB15D
:10DDF0000134102C07F11007F7D11A491A484FF4D3
:10DE0000707241F0E9FBBDE8F04116484FF47071C3
:10DE100041F0BCBE04F14D0805EB0813270105EBEA
:10DE200004149E6084F8E11484F8E024317845F00D
:10DE300012FAC4F8DC0473780C4813F020032F4462
:10DE400018BF95F8D43587F8E23405EB08110023A4
:10DE500085F8D4350431BDE8F04148F09EBB00BFE1
:10DE6000800D00207AD50500A2B8050038120020E8
:10DE7000124B07B5196802460968013A0868002183
:10DE8000072A19D8DFE802F0041216181818180427
:10DE90008DF8071083F8D415D3F8A4361BB10DF113
:10DEA00007020121984703B05DF804FB01228DF8B9
:10DEB0000720EFE70222FAE70322F8E7800D0020AF
:10DEC0004378034AC3F3001382F8D435704700BF88
:10DED000800D002010B5104C002284F88C260A78A2
:10DEE00084F8B0264A7884F8B1264A68C4F89426A3
:10DEF0000B465AB1497A84F89D16997A84F89C1693
:10DF00001178D86845F0A7F9C4F898060348BDE829
:10DF1000104015F02FBE00BF800D002074130020AC
:10DF2000064880F88C16137880F8B036537880F85D
:10DF3000B13600F2F45015F01DBE00BF800D002078
:10DF4000034B83F8F00503F5BB6015F013BE00BF6B
:10DF5000800D00200348002380F8F03500F5BB60F9
:10DF600015F008BE800D002070B5094CD4F8A056FD
:10DF700065B10023C4F8A03645F067F923681B6833
:10DF800001B218682B46BDE87040184770BD00BF4D
:10DF9000800D0020064BD3F8A02642B10021C3F823
:10DFA000A0161B681B6847F6FF711868104770477A
:10DFB000800D002000230A4A8A6030B5094C0B60AE
:10DFC000CB604B601A4654F8045B25B1824201D104
:10DFD0000D6030BD01320133392BF4D1F9E700BFB8
:10DFE00030AD05008001002010B50C46002142F044
:10DFF0003AFD00B1006820600023E3606360014BDC
:10E00000A36010BD30AD05002DE9F84304468846F5
:10E010005068164614F002FC054648B9204673685D
:10E020001D4A012142F003FB6FF01200BDE8F883A6
:10E0300083683921DB689847031E04DA174A0121F7
:10E04000204642F0F4FAB8F1020F20D1144F002616
:10E0500057F8042B1AB129462046F6F7CDFC0136B5
:10E06000392EF5D10020E1E756F827202946204631
:10E07000F6F7C2FC002806DA56F827304A46012196
:10E08000204642F0D4FA0137B845EDD8EAE7DFF888
:10E0900014900227F8E700BF56D705006BD705009C
:10E0A0008001002086D70500024B0B60012313601E
:10E0B000704700BF482B00200048704788AD05001E
:10E0C00037B50C46204619461546019344F01EFC10
:10E0D000019A80B90D4B1968490709D00C490D48C0
:10E0E0005B1A9B089B0143F00103214641F0DDFED2
:10E0F0006FF0150005E032B12146284643F05BFA87
:10E10000002003B030BD1046FBE700BF040700202D
:10E11000E8060020A0DA0500F0B587B00E461546E7
:10E1200045F044FD29460746304644F0EFFB90B3E6
:10E13000B6FBF7F307FB136323B9B5FBF7F407FB53
:10E1400014548CB1284B1A6851070AD0274A284822
:10E150009B1A9B089B0143F001032A46314641F07C
:10E16000A4FE6FF015043BE0AF4239D84FF0FF3307
:10E170004FF0FF321F4815F039FD45F016F802AB9D
:10E180000146B0B91022184643F020FACDE90365E4
:10E1900044F0CFFB20E0144B1A685207E1D0134A39
:10E1A00015489B1A9B089B0143F001032A46314600
:10E1B000D5E710222146184643F008FA01228DF8CF
:10E1C00014200E4ACDE900200D48CDE9036507F083
:10E1D00065FE684607F068FE0446064815F0CAFC6E
:10E1E000204607B0F0BD00BF04070020E80600206D
:10E1F000BDDA0500502B0020A0DA05003329050008
:10E20000645E010010B5012211460748074C48F032
:10E21000D9F907F03BFE45F0CDFC206045F0C6FC87
:10E220006060002010BD00BF502B0020482B002054
:10E2300038B5037B04460BB144F0B9FF0125A36850
:10E24000032B06D8124AD2F80034DB07FBD5002096
:10E2500038BD2368606819680EF02EFD63680433CA
:10E260006360236804332360A368043BA360237BBB
:10E270000135002BE3D0284607F0E0FE0028DED071
:10E28000034AD2F80034D907FBD50120E0E700BFEC
:10E2900000E0014070B50D4686B019462846164686
:10E2A0001C4644F033FB88B9264B1A6850070AD045
:10E2B000254A26489B1A9B089B0143F001032246EE
:10E2C000294641F0F2FD6FF0150431E045EA040300
:10E2D00099070DD01B4B1A685207F4D01A4A1C48F4
:10E2E0009B1A9B089B0143F0010322462946E8E75D
:10E2F000F4B14FF0FF334FF0FF32164815F076FCC3
:10E3000044F053FFCDE9026502AB049498B10122B9
:10E310008DF81420104A41F64C50CDE9002307F047
:10E32000BDFD684607F0C0FD04460A4815F022FC12
:10E33000204606B070BD8DF814001846FFF778FF30
:10E34000F2E700BF04070020E8060020A0DA05007D
:10E35000DCDA0500502B002031E2000007B55368DD
:10E3600000931368044A012142F061F96FF015002F
:10E3700003B05DF804FB00BF04DB05002DE9F341A9
:10E380001F461368DDF8208006460D46586814467F
:10E3900001A9102242F0F9FF019BC8F800001B7888
:10E3A0007BB12368586814F039FA386058B93046A0
:10E3B000144A012142F03BF96FF0120002B0BDE8AF
:10E3C000F0811148EFE7019B18780028F6D02B6800
:10E3D000022B07D830460D4A012142F028F96FF090
:10E3E0001500EBE723681022986801A942F0CDFFE1
:10E3F000C8F800002B68013B2B60236804332360BE
:10E400000020DBE71EDB050019CC05003BDB050027
:10E41000F0B5A7B005ABCDE90221009302AA04AB89
:10E4200003A90546FFF7AAFF0446F8B9039B022B90
:10E4300015D916AF039AA31C9A424FEA840618D83E
:10E44000DDE9040133463A4644F0D1FA10B31F4ADD
:10E450000121284642F0EBF86FF0040406E01C4A64
:10E460000121284642F0E3F86FF01504204627B05A
:10E47000F0BD0E2CE4D0029B33441022986800219A
:10E4800042F083FF06AB47F82400C04343F8240062
:10E490000134CFE728460F4A082142F0C8F8DDE9E9
:10E4A0000401836806AA1C683346A047324606A9C1
:10E4B000384643F059F8044628B9074A0821284647
:10E4C00042F0B5F8D2E7054AC2E700BF6ADB0500B3
:10E4D0004DDB050081DB05008CDB050097DB0500CB
:10E4E00030B58BB006ABCDE90221009302AA05AB93
:10E4F00003A90546FFF742FF044620BB039B022BFE
:10E5000013D9029B10220146986842F03EFF024652
:10E51000DDE9050144F089FA0446C8B103460F4A13
:10E520000121284642F083F80DE0DDE9050107AA44
:10E5300044F059FA034648B1094A0121284642F0FD
:10E5400076F86FF0150420460BB030BD089ADFE76F
:10E55000044A0821284642F06AF8F4E7D5DB0500B2
:10E56000ACDB0500EDDB050010B50C46002142F0E8
:10E570007AFA00B1006820600023E3606360014B19
:10E58000A36010BDA4AD05002DE9F04F87B005AB29
:10E59000CDE90221009302AA04AB03A90546FFF7C7
:10E5A000EDFE044650BB029B01461022986842F0E3
:10E5B000ECFE029B06461022D868214642F0E5FE9A
:10E5C000B6F5805F074610D8254A2346B34219D1D5
:10E5D000DFF8A090DFF888A0DFF89CB0B7B9214A37
:10E5E0000821284642F023F808E01F4A4FF48053E0
:10E5F0000121284642F01BF86FF01504204607B0B1
:10E60000BDE8F08F02F8013B0133DFE7DDE90401EB
:10E61000324644F00AFA804638B10346134A0121D3
:10E62000284642F004F84446E8E728464A460821CE
:10E6300041F0FDFFDDE904013346524644F0D7F9CD
:10E64000013F804628B10A4A0121284641F0EFFFE8
:10E65000E9E75A460821284641F0E9FFBEE700BF36
:10E66000682B002026DC0500FDDB0500D5DB05005E
:10E670006ADB05001BDC050081DB05002DE9F043AA
:10E680008BB005ABCDE90221009302AA04AB03A92C
:10E690000646FFF773FE044650BB039B022B10D9BE
:10E6A000029B01461022986842F06FFE07464FF029
:10E6B0000008B84507DB164A0821304641F0B7FF8D
:10E6C00016E00127F3E7A7EB0805102DA8BF1025DA
:10E6D000DDE90401836806AAD3F800902B46C847F9
:10E6E00050B10C4A0121304641F0A1FF6FF0040403
:10E6F00020460BB0BDE8F0832B46059906AA3046AC
:10E70000FAF7CCFD059B2B440593A844D1E700BF45
:10E71000CEBF05003EDC0500F0B54B79012B28D0BB
:10E72000032B23D110248B79032B1FD1CE790EB16B
:10E73000012E1BD10A79012A1DD0022A1FD0AAB9A5
:10E7400015460B684768B3F5164F3F686ED033D84F
:10E75000B3F5165F6DD01CD8B3F5966F6BD010D89B
:10E76000B3F5967F6AD0B3F5167F6AD06FF0850057
:10E770005BE00024D7E74FF480750E22E1E7002527
:10E78000FBE7B3F5166F5FD0B3F5965FEED1394B6B
:10E790003EE0B3F5E14F5AD007D8B3F5615F58D0EA
:10E7A000B3F5964FE2D1344B32E047F6122C634575
:10E7B000DCD14FF400032BE0B3F5613F4BD013D80D
:10E7C000B3F5963F4AD009D84DF6C02C634547D0E3
:10E7D000B3F5614FCAD14FF46B0319E0B3F5E13FD4
:10E7E000C4D14FF0EB7313E0B3F5612F3BD009D8E0
:10E7F000DFF898C0634539D0B3F5E12FB6D14FF0BB
:10E80000E86305E0DFF888C06345AFD14FF080537F
:10E81000C7F82435036903C9224335432A43043327
:10E82000C7F86C2583E803000020F0BD4FF41D03FA
:10E83000EEE7124BECE74FF49E23E9E74FF4A033E9
:10E84000E6E74FF41C33E3E74FF41D23E0E70C4BFE
:10E85000DEE70C4BDCE74FF06C73D9E70A4BD7E7E8
:10E860004FF46503D4E74FF07063D1E74FF0806356
:10E87000CEE700BF00B0130000A04E0000502700FC
:10E8800000C0750000F03A0000903A0190D00300FB
:10E8900040420F000268530910B504462AD0012BEC
:10E8A00040F2FF3318BF002302F01F02D340DB0702
:10E8B0000AD41349134840F2292240F08DFE104833
:10E8C00040F2292141F062F9236803F01F025B093D
:10E8D00022600CD0012B10D009490A4840F22E22A8
:10E8E00040F07AFE064840F22E2141F04FF94FF0F9
:10E8F000A04010BD4FF0FF33D6E70348F9E700BF53
:10E90000D5D40500A2B8050000030050F8B506698B
:10E9100005460F4647F002FE10B9204B1B7883B91D
:10E920004FF04003EFF3118483F31288BFF36F8F2E
:10E93000284644F005F928BB84F31188BFF36F8F94
:10E94000EEE76424284644F0FBF870B9012045F056
:10E95000A2F8013CF6D10021212016F025FDF0E7B8
:10E9600084F31188BFF36F8FF5E74FF04003EFF3A7
:10E97000118483F31288BFF36F8F284644F0E0F8C8
:10E980000028EDD03146012201F8147F284644F0DA
:10E9900068F984F31188BFF36F8FF8BD61680020B8
:10E9A0002DE9F743D0F804800769D8F80040002328
:10E9B000C4F8003538604568EB685A1C064613D029
:10E9C00001A80193FFF766FF019A01239340C0F865
:10E9D0000835EB68019301A8FFF75CFF019B03F585
:10E9E000E073032240F823202B69581C11D02A7FA2
:10E9F0000193002A01A814BF4FF003094FF000094A
:10EA0000FFF748FF019B03F5E0734FEA890240F8E6
:10EA100023206B69591C13D001A80193FFF73AFF1B
:10EA2000019A01239340C0F808356B69019301A84E
:10EA3000FFF730FF019B03F5E073032240F823202A
:10EA4000AB695A1C11D06A7F0193002A01A814BF38
:10EA50004FF003094FF00009FFF71CFF019B03F57E
:10EA6000E0734FEA890240F82320D5E903122B68AE
:10EA7000C3F80C15C3F81425D5E90512C3F8081519
:10EA80003169C3F8102504313046FFF745FE0546CD
:10EA9000002856D1D8F804309E0729D507F1160072
:10EAA0000EF03EF9294B98420FD029490B685807C0
:10EAB00008D0284B2848C91A8908890141F001016A
:10EAC00041F0CDF96FF004053BE0B87DC30003F1E0
:10EAD000804303F5F83304F10C0204F59071C3F898
:10EAE0001015C3F814251D4A01238340C2F80435CC
:10EAF0000823C4F8003598F808305BB9C4F8103121
:10EB0000D4F8103107F11503C4F834350123C4F8E3
:10EB100038352360D8F804309A075CBF4FF4807210
:10EB2000C4F80423DB0644BF4FF48003C4F8043365
:10EB300014370023C4F84475C4F848350123A36092
:10EB4000E360284603B0BDE8F08300BF0000AD0BD2
:10EB500040070020E806002014DD050000F0014019
:10EB60004FF04003EFF3118283F31288BFF36F8FEE
:10EB7000084B196859B10849D1F8080500211960F6
:10EB80001B68C0B282F31188BFF36F8F70476FF0BC
:10EB90000A00F7E700D1004000D00040F0B503467E
:10EBA0008478C7784FF04005EFF3118085F3128821
:10EBB000BFF36F8F1E7893F801E0A41B3C40A24284
:10EBC00088BFA2B206EB020C07EA0C0C354683F8AC
:10EBD00000C080F31188BFF36F8F0A440846824259
:10EBE00019D176450DD14FF04005EFF3118285F331
:10EBF0001288BFF36F8F1D785D7082F31188BFF3A9
:10EC00006F8F411A1B7988B2211A8B4222BF064BA3
:10EC100001221A60F0BD03EB050C01359CF805C01C
:10EC200000F801CB3D40DAE700D000402DE9F04785
:10EC300014461D4602692C4B9A420E460AD02B49B7
:10EC40002B484FF4847240F0C7FC28484FF484717D
:10EC500040F09CFFEB4313F0010506D02548224607
:10EC60003146FFF79BFFBDE8F087002C33D04FF013
:10EC70004003EFF3118883F31288BFF36F8F0D20E9
:10EC8000FBF760FC07460D20FBF748FC88F3118872
:10EC9000BFF36F8F184A15601368184B0121196074
:10ECA00017494FF40053C1F88031254691468A46F2
:10ECB0009846D9F8003083B1FFF752FF031ECAF817
:10ECC0008081F6DB013DADB27355002DF1D117B156
:10ECD0000D20FBF713FC2046C5E7BFF34F8F20BF85
:10ECE00040BF20BFE5E700BF683B002051DD0500C5
:10ECF000A2B80500983B002000D1004000D00040A1
:10ED000000E100E02DE9F8431A4B144602699A42EB
:10ED1000894608D018491948EA2240F05DFC164897
:10ED2000EA2140F033FF134E06F1450706F11808BB
:10ED300014B92046BDE8F8834FF0FF334FF0FF329F
:10ED4000304614F053FF224649463846FFF726FF67
:10ED50000546304614F00EFF3DB94FF0FF324FF03C
:10ED6000FF33404614F042FFE2E7641BA4B2A9441B
:10ED7000DEE700BF683B002051DD0500A2B80500BA
:10ED800038B51F4C0369A3420AD01E491E4840F201
:10ED9000571240F021FC1B4840F2571140F0F6FE9C
:10EDA00001221146164847F00DFC012200211748A8
:10EDB00047F008FC40F20743A4F848304FF0706376
:10EDC00023630C2384F834300025114B84F845501C
:10EDD000A4F84650D3F8042522F00102C3F8042514
:10EDE0000C4A012115601268C3F804132A46196001
:10EDF0000D20FBF7B5FB0D20FBF780FB284638BD47
:10EE0000683B002051DD0500A2B80500803B0020D2
:10EE100000D0004000D1004010B5FFF7A1FE00284F
:10EE200020DB174B93F8322093F8311093F83340DE
:10EE3000511A34EA0101C0B20DD193F8472093F87A
:10EE4000461093F84840511A34EA01010BD10D4B9A
:10EE500001221A600EE099180132224081F8350033
:10EE600083F8322010BD99180132224081F84A00FF
:10EE700083F847200448BDE8104014F07BBE00BF73
:10EE8000683B002004D00040803B0020194970B549
:10EE9000044622F07F460868C1E90023A6F5001366
:10EEA000101AB3F5400F4FF000050AD2124B196843
:10EEB0000A060B0A9219114943F10003C1E9002324
:10EEC000012516F099FDA30003F1804303F5883373
:10EED000D3F84025B2420BD11DB94FF40002C3F85C
:10EEE0004025074B4FF4803000FA04F4C3F8444344
:10EEF00070BD00BF80180020C43B002068180020AF
:10EF00000010014010B501238340114ABFF35B8F0D
:10EF1000DC4352E8001F01EA040C42E800CEBEF1D7
:10EF2000000FF6D1BFF35B8F4FF4803202FA00F08E
:10EF300002F1804202F58052C2F80803BFF35F8FEE
:10EF4000BFF36F8F0B4214BF0120002010BD00BF24
:10EF5000C03B00200123124ABFF35B8F834052E87D
:10EF6000001F194342E8001CBCF1000FF7D1BFF3AA
:10EF70005B8F0C4A4FF480338340C2F804330A4B52
:10EF8000BFF35B8F1B68BFF35B8F23FA00F0C307EF
:10EF900042BF064B4FF40032C3F80021704700BF58
:10EFA000C03B002000100140BC3B002000E100E01D
:10EFB0000D4B1B68190A1806BFF35F8F0B4BD3F874
:10EFC0000435C01841F10001B3F5801F0AD2084B87
:10EFD000D3E90023994208BF904203D210F1807018
:10EFE00041F10001704700BFC43B00200010014008
:10EFF000681800202DE9F04F85B016461F460546DB
:10F00000FFF780FF0190FFF7D3FFB94208BFB0427E
:10F010007FD2B6EB000867EB010900234FF0807246
:10F020004B4508BF4245C0F08580444B03EB0513B8
:10F03000D3E902239F4208BF964254D04FEA850984
:10F040004FF4803B09F1804905F150080BFA05F2B5
:10F0500009F588394FEA88081FFA88F80292384A79
:10F06000D9F8400526F07F4308F1804808F5883834
:10F070001C469346D2F804A5A0EB0A0020F07F407E
:10F080002AF07F410128C9F8401505D103931320C8
:10F0900047F030FB2A4A039B02990AF1020CA4EBC9
:10F0A0000C0020F07F40B0F5000F88BF64460020C0
:10F0B000C8F80000D8F80000CBF8441324F07F40D3
:10F0C000C9F84005DBF80405824506D0201A02384D
:10F0D00020F07F40B0F5000F19D8E41A24F07F44E7
:10F0E000321947F10003154C290104EB0510C0E962
:10F0F00002230E9A0F9B625043600024019B13B1C0
:10F100002846FFF727FF204605B0BDE8F08F2046D0
:10F11000B0E701230B4ABFF35B8FAB4052E8001FFF
:10F12000194342E800100028F8D1BFF35B8F324644
:10F130003B46D8E76FF01504E0E700BF70180020E9
:10F1400000100140BC3B002073B5194B194D002441
:10F150004FF0FF304FF0FF31C5F80845C3E9020119
:10F160004FF48033C5F80433134B02264FF40032BA
:10F170000121C5F804631120C3F880212246FBF762
:10F18000EFF91120FBF7BAF90C4A012313600C4A7E
:10F190002B6013600B4B0C4A009301940023204614
:10F1A000FFF728FF3046FDF7D5FD204602B070BDC1
:10F1B000701800200010014000E100E0081001403C
:10F1C000C03B00208DEE0000FFFF7F002DE9F347DC
:10F1D0002A4CD4F80433990709D5294B1A6832B15F
:10F1E00000221A60274A1B68136801331360EFF38B
:10F1F000108372B6D4F80423D2032CD5BFF35B8FEF
:10F20000214A52E8001F21F0010042E80005002DCC
:10F21000F7D1BFF35B8F1D4A09B91168D9B1002539
:10F220001560126883F31088FFF7C2FEEFF31082B7
:10F2300072B6174BD3E90289494508BF40450FD242
:10F24000294682F3108841B1CDF800A042464B46D2
:10F250000020884701E083F3108802B0BDE8F08702
:10F260004FF0FF364FF0FF37D3E9001AC3E90267CA
:10F270001D604FF48033C4F84833E2E700100140CA
:10F2800004110140C43B0020BC3B00204011014060
:10F2900070180020144B13B5B0F1FF3F08BF18469B
:10F2A000441E002C1EDD9C42A8BF1C46FFF780FEBA
:10F2B0000E4B0F49D3E90023801AB0F5000F28BF89
:10F2C00000240130044408480091844228BF0446C9
:10F2D00012194FF00000019043F10003FFF78AFE7E
:10F2E00002B010BD0024E1E7FFFF7F00801800207E
:10F2F0008DEE000008B5FFF75BFE024B1B68C01ADD
:10F3000008BD00BF8018002043682DE9F0471B6846
:10F31000D0F80890D0F8108001268E401E42044696
:10F320000D4617460AD10C490C4840F2FD2240F028
:10F3300053F9094840F2FD2140F028FCD8F800308C
:10F3400023EA0606C8F80060D9F800303A46294694
:10F350002046BDE8F047184783DD0500A2B8050048
:10F3600002F4C043B3F5C04F2DE9F041D0E9018765
:10F3700005460E46144636D12049214840F28922DE
:10F3800040F02AF940F289211C4840F0FFFB04F4C8
:10F39000C823B3F5804F0AD11849194840F2972283
:10F3A00040F01AF9154840F2972140F0EFFBD8F8E9
:10F3B00000200123B34013420AD11049104840F203
:10F3C0009D2240F009F90D4840F29D2140F0DEFBFE
:10F3D000BF6904F4C02304F4B03231462846BC4669
:10F3E000BDE8F0416047002BD1D10449044840F208
:10F3F0008D2240F0F1F840F28D21C5E783DD050054
:10F40000A2B80500012370B503FA01F543681B6833
:10F410001D42044616460AD10A490B4840F2914261
:10F4200040F0DAF8074840F2914140F0AFFB36B1C6
:10F43000A368DB6829462046BDE870401847A368EA
:10F440001B69F7E783DD0500A2B805002DE9F74F3A
:10F450000024234FDFF89890DFF89880DFF898A019
:10F46000254609EBC50357F804BB1B7901269E40CE
:10F47000DBF804301B681E420AD14146504640F278
:10F480003A4240F0A9F840F23A41404640F07EFB53
:10F49000DBF8083001A95B685846984700280AD174
:10F4A000019B1E4203D00135042DDAD113E0012364
:10F4B000AB401C43F7E7F6DA0A490C6814F007047E
:10F4C00009D0094B0948C91A8908890141F001018D
:10F4D00040F0C5FC0024204603B0BDE8F08F00BF1B
:10F4E000C83B0020FC060020E8060020ADDD05003A
:10F4F000ACAE050083DD0500A2B805002DE9F84398
:10F50000DFF86880DFF8689006460F46002426FA88
:10F5100004F227FA04F31343D9071BD508EBC403FD
:10F52000D243197959F8240002F00102FFF76AFF6B
:10F53000054678B10A490B685B0708D0094B0A48B1
:10F54000C91A8908890141F0010140F088FC284668
:10F55000BDE8F8830134042CD9D10025F7E700BFBA
:10F56000FC060020E8060020C2DD0500CCAE050048
:10F570000C3C0020F8B54FF04003EFF3118583F306
:10F580001288BFF36F8F2B4813F0EAFC40B92A4969
:10F590002A48812240F020F82748812140F0F6FADD
:10F5A0002448274E274F13F0F9FC002407EBC4032F
:10F5B00056F8040B19794FF400520134FFF7D0FECE
:10F5C000042C0FD00028F1D01F490B685B070BD02B
:10F5D0001E4B1F48C91A8908890141F0010140F0FA
:10F5E0003EFC01E00028EFD11A4B1A78C2B9012283
:10F5F0001A7019482122002314F00AFF0D4813F055
:10F60000BDFC40B90C490D48AC223FF0E5FF0A486B
:10F61000AC2140F0BBFA85F31188BFF36F8FF8BDC2
:10F620000E490648E8223FF0D7FF0C48E82140F099
:10F63000ADFAE3E71C3C0020DCB80500A2B80500E9
:10F64000C83B0020ACAE0500FC060020E806002008
:10F65000D8DD0500F959002088180020F1DD0500EB
:10F660002DE9F041FFF7F2FEBFF35B8F4F4B0446ED
:10F6700053E8002F43E800410029F9D1BFF35B8F25
:10F680004B4BDFF864811A7872BBD8F80060A64251
:10F6900012D0484B1B6866400BB1314698474FF07B
:10F6A000FF3345484FF0FF3214F00AF8434B1D6812
:10F6B0006DB9414814F0DCF8C8F80040BCB1BDE8B1
:10F6C000F0413F484FF4A472002314F0A1BE043D62
:10F6D000002DEED02F46314657F8043B2046984780
:10F6E000002FE6D06D68E3E700221A70E4E74FF0E0
:10F6F0004003EFF3118783F31288BFF36F8F314814
:10F7000013F02EFC40B93049304881223FF064FFAD
:10F710002D48812140F03AFA2A4813F03FFC2C4B47
:10F720001A78012A34D100222A4EDFF8C0801A70DC
:10F7300008EBC40356F8040B19794FF41032FFF7A5
:10F740000FFE0134042C054601D00028F0D01D48DE
:10F7500013F014FC40B91C491C48AC223FF03CFF9C
:10F760001948AC2140F012FA87F31188BFF36F8F6C
:10F77000CDB119490B685B0715D0184B1848C91A49
:10F7800089088901BDE8F04141F0010140F067BB03
:10F7900014490E48B1223FF01FFF1248B12140F03A
:10F7A000F5F90025D3E7BDE8F08100BF203C00203B
:10F7B0006A040020D83B0020DC3B0020F03B002006
:10F7C000881800201C3C0020DCB80500A2B8050009
:10F7D000F9590020C83B0020FC060020E806002064
:10F7E0002FDE0500F1DD0500043C0020ACAE050075
:10F7F000F8B51C4D1C4F0026286813F00FF847F889
:10F80000040B78B919490B685A0708D0184B1948E6
:10F81000C91A8908890141F0010140F020FB6FF00D
:10F82000120413E029794FF40072FFF76DFD0446CE
:10F8300070B10E490B685B0708D00D4B0E48C91A12
:10F840008908890141F0010140F009FB2046F8BD1B
:10F850000136042E05F10805CED1BDE8F8400F2190
:10F86000FFF74CBECCAE05000C3C0020FC0600208F
:10F87000E806002047DE05005FDE0500074BBFF30A
:10F880005B8F1B68BFF35B8F00B10360044811B14D
:10F8900002685A400A600360704700BF203C0020A5
:10F8A000083C00202DE9F84F504B18605048514D4E
:10F8B000DFF8748146F051FE47460026A9462868C5
:10F8C00012F0ACFF47F8040B78B94B490B685C07A2
:10F8D00008D04A4B4A48C91A8908890141F00101F8
:10F8E00040F0BDFA6FF0120413E029794FF48872EA
:10F8F000FFF70AFD044678B13F490B68580708D066
:10F900003E4B4048C91A8908890141F0010140F085
:10F91000A6FA2046BDE8F88F0136042E05F1080549
:10F92000CDD1DFF804A1054606464FF0010B09EBE7
:10F93000C6035AF8040B1F794FF400523946FFF7FB
:10F940000FFD044658B12C490B685A07E1D02B4BE8
:10F950002D48C91A8908890141F00101D7E701360C
:10F960000BFA07F7042E45EA0705E0D1274E284B8E
:10F97000C6E90135054658F8040B8368DB6983B195
:10F98000012231469847044670B11B490B685B075A
:10F99000BFD01A4B1F48C91A8908890141F00101DB
:10F9A000B5E76FF08504F0E70135042DE3D11A497E
:10F9B0001A4814F037FC1A4B184801221A70002319
:10F9C000002214F0BDFC21462046FFF757FFFFF749
:10F9D0003DFDBFF35B8F134B53E8002F43E800015D
:10F9E0000029F9D1BFF35B8F93E700BFD83B00201C
:10F9F000DC3B0020ACAE0500FC060020E806002041
:10FA000047DE050079DE050096DE0500F83B0020A4
:10FA100075F50000B1DE050061F6000088180020D1
:10FA2000F9590020203C0020C83B0020032810B5D5
:10FA30000FD916490B685A0708D0154B1548C91A33
:10FA40008908890141F0010140F009FA6FF01504BD
:10FA50001AE0114B03EBC003B1FA81F219790F4B95
:10FA6000520953F82000FFF7CDFC044660B1074966
:10FA70000B685B0708D0064B0948C91A8908890139
:10FA800041F0010140F0EBF9204610BDFC060020DA
:10FA9000E8060020C5DE0500CCAE05000C3C0020C9
:10FAA000C2DD050002460B46014813F009BE00BF47
:10FAB000DC070020014813F0DBBE00BFDC0700209C
:10FAC00008B5F7F747F808490B685B0708D0074BFC
:10FAD0000748C91A8908890141F0010140F0BFF9BE
:10FAE0000020FBF75DFC00BF00070020E8060020B7
:10FAF000F4DE05000E4B13B50A46196849070ED00F
:10FB00000C4C01921C1BA408F6F79AFEA40144F0C9
:10FB100001040146019A0848234640F0C6F94040D6
:10FB200080F311884FF0030002DF02B010BD00BF68
:10FB300014070020E806002011DF050037B5322346
:10FB4000ADF80430134A00230125192168468DF8C9
:10FB50000630ADF800508DF80230F3F723FF04466D
:10FB6000A0B90D482946F4F7D0FC044670B9014607
:10FB70002A460820FAF7F4FC2A4621460B20FAF719
:10FB8000EFFC2A4621462846FAF7EAFC204603B055
:10FB900030BD00BFF5FA0000243C0020014813F0FE
:10FBA000E9BF00BF9808002038B50F4D0F4C4FF04B
:10FBB000FF324FF0FF33284614F018F84FF0FF30B3
:10FBC0004FF0FF31FFF76EFF40B109482146462252
:10FBD0003FF002FD462120463FF0D8FFF4F7A2FD9A
:10FBE000FFF768FFE3E700BF9808002025DF050066
:10FBF000A2B8050030B589B00F4D1049002200238E
:10FC0000CDE9062300246FF00703CDE90334CDE9E5
:10FC100001440B4B00944FF48062284613F0FCFA29
:10FC20000849284613F052F9224604211920FAF710
:10FC300097FC204609B030BDB818002080DB0020BA
:10FC4000A9FB000052DF050010B50F4C2378D3B19B
:10FC50000E48FF2100F096FE0D4B90B90D4918702B
:10FC60000B68207003F00703022B0CD90A4B0B48DA
:10FC7000C91A89088901BDE8104041F0030140F02C
:10FC8000EEB801221A7010BDFB590020F92D0500B5
:10FC9000FC59002048070020E806002068DF050026
:10FCA00008B52EF029FDF0B90F4B1B78DBB10F4BD7
:10FCB0000F4A18701378B3B9012111700D4A0E491B
:10FCC00013700E4A13700B6803F00703022B0AD956
:10FCD0000B4B0C48C91A89088901BDE8084041F05E
:10FCE000030140F0BCB808BDFE590020FA590020BD
:10FCF000FB590020FC59002048070020FD59002036
:10FD0000E80600208ADF05002DE9F84F1C469DF823
:10FD100028300746884691466BB1661E002BDFF8F7
:10FD200038B014BF4FF0FF3A4FF0010A002524B954
:10FD30002846BDE8F88F1E46F0E719F806305A4607
:10FD4000A8EB05017819FBF7E3FA0028F1DB013C89
:10FD500005445644E4B2EAE7ACDF05002DE9F04182
:10FD60008EB0002604A98046049648F0A6FB0546FE
:10FD7000404647F0B7FF044648F02FFC334607469D
:10FD80008E4E312D00F20683DFE815F03900520067
:10FD90005A02D30104036900CC00040304030403E2
:10FDA0003A018E01CA02040304030403040304039A
:10FDB00039000102040304032A023200BA020403D8
:10FDC00004030403040304030403040304030403FB
:10FDD00004030403040304030403040304030403EB
:10FDE000040304030403040304036B022D02DA0278
:10FDF000734A136803F0070374B1022B01D801257D
:10FE00002BE0704B7048D21A9208920142F0030224
:10FE1000214640F033F8F2E7022BF0D969496B48EC
:10FE2000511A8908890141F0030140F018F8A8E04F
:10FE30006349012333700B6803F00703022B08D9D1
:10FE4000604B6348C91A8908890141F0030140F0F9
:10FE500006F800200DF00AFF0546002431E0584D59
:10FE60002B6803F00703022B08D956495948691A31
:10FE70008908890141F003013FF0F1FF2B6803F08D
:10FE80000703002C42D16FB1022B08D94D495248CB
:10FE9000691A8908890141F003013FF0E0FFFFF78B
:10FEA000FFFEACE7022B08D946494C48691A89087D
:10FEB000890141F003013FF0D2FF04200DF0D6FE8E
:10FEC00005463378CBB146490B78B3B1454B1A7828
:10FED000002A00F0708200220A7039491A700B68FB
:10FEE00003F00703022B08D9364B3F48C91A89088B
:10FEF000890141F003013FF0B2FF1CB985F0010414
:10FF0000E4B2644220460EB0BDE8F081002B3FF41D
:10FF100076AF2C4A3548AA1A9208920142F00102A3
:10FF2000214676E7264D74BB0D2221460AA8099486
:10FF300041F04CFB05A82EF057F905AA112109A89C
:10FF400042F05DFF002803DA294909A841F0B6FA1A
:10FF5000FFF77AFE2B6803F00703022B11D9194A29
:10FF600009A8AD1AF6F76CFCAD08039022F082FBED
:10FF7000AD0145F00305428803991E482B463FF02A
:10FF800094FF01259DE72B6803F0070348B1022B7E
:10FF900085D90C491848691A8908890141F003017B
:10FFA0007BE7002B3FF42BAF064A1448AA1A9208AD
:10FFB000920142F0010221462BE700BFFE590020CA
:10FFC00048070020E8060020B1DF0500F1DF05004A
:10FFD0001EE0050037E0050059E0050070E005006F
:10FFE000FB590020FC59002068DF050088E005006F
:10FFF000B7E00500BFE0050013E1050046E105009C
:020000021000EC
:10000000B04D8CBB0D2221460AA8099441F0DEFABE
:1000100005A82EF0E9F805AA112109A842F0EFFE83
:10002000002803DAA84909A841F048FA2B6803F030
:100030000703022B11D9A54A09A8AD1AF6F700FC4F
:10004000AD08039022F016FBAD0145F00305428890
:1000500003999F482B463FF028FF0FB1FFF7F4FDAF
:10006000002025F06FFECAE62B6803F0070370B18D
:10007000022B09D9954A9748AA1A9208920142F090
:10008000030221463FF0FAFEFFF70AFEE8E7022BE3
:10009000E6D98E4A9048AA1A9208920142F00302C9
:1000A00021463FF0EBFEDBE7864D64BB0D22214687
:1000B0000AA8099441F08AFA05A82EF095F805AA35
:1000C000112109A842F09BFE002803DA7E4909A805
:1000D00041F0F4F92B6803F00703022B11D97B4B95
:1000E00009A8ED1AF6F7ACFBAD08039022F0C2FAAE
:1000F000AD0145F003054288039978482B463FF04F
:10010000D4FE0220DAE62B6803F00703022B09D99C
:100110006E4A7348AA1A9208920142F003022146DD
:100120003FF0ACFE6F484222042100F0EDFB044694
:1001300027E7644A136803F00703DCB9022B0AD9E6
:10014000624B6948D21A9208049B9201197942F0D5
:1001500003023FF093FE48F040FA38B904200DF056
:1001600085FD0546002025F0EDFD76E6FFF798FDBC
:100170000125F7E7002BFBD0544B5C48D21A9208BC
:10018000920142F0010221463FF078FEF0E7049D23
:1001900009930D2200210AA841F018FA2A1D112105
:1001A00009A842F02CFE002803DA474909A841F0CB
:1001B00085F9444B1A6802F00702022A7FF61FAE47
:1001C000424C09A81C1BF6F73BFBA408A40144F011
:1001D000030401462A7B464823463FF066FE0EE6AE
:1001E0002DF0B6FE0BE6049D09930D2200210AA80E
:1001F00041F0ECF92A1D112109A842F000FE002867
:1002000003DA314909A841F059F92E4B1A6802F076
:100210000702022A7FF6F3AD2C4CA98903911C1B1F
:1002200009A8F6F70DFBA408A40144F00304AB7B76
:100230000399ADF8004002462E483FF04FFEDEE540
:10024000204A136803F00703022B7FF6D8AD1F4B3B
:100250002948D21A9208049B9201998842F003021D
:10026000D7E5049D09930D2200210AA841F0AEF9BB
:100270002A1D112109A842F0C2FD002803DA124903
:1002800009A841F01BF90F4B1A6802F00702022A75
:100290007FF6B5AD0D4C09A81C1BAB890593F6F78D
:1002A000CFFA0690AB7B0793A408A401EB7B0893DD
:1002B00044F0030411482346042205A93FF02DFE13
:1002C0009DE500BF48070020B7E00500E8060020D4
:1002D00086E10500C9E10500FAE1050035E2050007
:1002E00090E205006DDC0100BCB70500DAB705003F
:1002F000B7E20500EAE2050028E305005DE305003A
:100300004C490B6813F0060F3FF479AD4A4B4B484C
:10031000C91A8908890141F002013FF0A0FD6EE58C
:10032000444A136803F00703022B7FF668AD424B83
:100330004348D21A9208920142F00302214668E52E
:100340003C4D2B6803F00703022B08D93A493D487E
:10035000691A8908890141F003013FF080FD47F0E7
:10036000A6FA044650B1414647F025FB0421204639
:1003700047F0CAFB204625F03FFD40E52B685807B3
:100380003FF43DAD2C493048691A8908890141F094
:1003900001014AE5274B1A6802F00702022A7FF69C
:1003A0002EAD254A29489B1A9B089B0143F0030365
:1003B0002246294611E7264F3B78002B7FF49DAD5E
:1003C000244925480B7801229A40B2F5617FDCBFB1
:1003D00001330B702149C8BF4FF4617243F6FF33FC
:1003E00001FB02324FF470530021B2FBF3F200F034
:1003F0008BFA4242D8B10F4B1968490715D00E4EFF
:1004000009929E1B10460CF035FDB608144B0B9359
:10041000B60140F2B72346F001060A900C9311484A
:100420003346042209A93FF078FD00F02DFB01239B
:100430003B7062E548070020E8060020CEE3050097
:10044000E4E305000FE405003DE405007EE405005B
:10045000FA590020FD590020F92D050040420F00F7
:10046000ACE4050090B705008A4A2DE9F04F136807
:10047000894E02EB43270133082B28BF00230437A2
:10048000136085B04FF4007204460021384641F0F5
:100490009DF81B21204647F09FFB8046204647F0F1
:1004A00073FA8346204647F065FA7C4BD3F80090F8
:1004B00009F101021A608246794A4B4640F2FF1167
:1004C0003846FAF725FF00280FDA33685B0708D0B3
:1004D00074497548711A8908890141F001013FF09A
:1004E000BEFC002005B0BDE8F08F07F2FF143D18F8
:1004F000A5420AD333685A07F3D06A496B48711A88
:100500008908890141F00101E9E798F80030C0F558
:10051000FF710131032B00F2A180DFE803F00279C3
:100520008C90B8F80130624A2846FAF7F1FE0028AC
:10053000CBDB0544A542DDD2B8F8112098F80B308A
:100540000292B8F80F20019298F80C200092611BDB
:10055000584A2846FAF7DCFE0028B6DB0544A542D7
:10056000C8D298F8172098F81430039298F81520FC
:10057000029298F81320019298F816200092611BBD
:100580004D4A2846FAF7C4FE00289EDB0544A542E2
:10059000B0D298F81830611B002B61D0B8F8193030
:1005A000464A2846FAF7B4FE00288EDB0544A542E9
:1005B000A0D2434A611B2846FAF7AAFE002884DB32
:1005C0000544A54296D2611B4FF00008CDF800808B
:1005D0005FFA8BF3524689B22846FFF795FB002855
:1005E000FFF673AF0544A54284D2364A4B46611BE1
:1005F0002846FAF78DFE0028FFF667AF33682A1801
:10060000A24203F0070330D3002B3FF46AAF74E734
:1006100008F1010289B2284642F0F1FB0028FFF6FA
:1006200054AF0544A542BFF465AF274A611B284675
:10063000FAF76EFE7BE7D8F80130244A74E708F138
:10064000010289B2284642F0DAFB0028FFF63DAFEE
:100650000544A542BFF44EAF1D4AE7E71D4AE6E751
:100660001D4A2846FAF754FE9EE7022B05F8008043
:100670007FF637AF0B4C3846341BF6F7E1F8A40889
:10068000A40144F003040146224614483FF0F6FB5F
:1006900027E700BF483C00204C0700204C4C0020BE
:1006A00003E50500E806002028E505006EE50500E5
:1006B000A0E50500DCE5050015E605005CE60500A3
:1006C00080E605008BE60500AEE50500B9E505000E
:1006D000CAE50500D1E505006FE6050018C1050073
:1006E00008B547F090FF50B109490A4840F251124D
:1006F0003EF072FF064840F251113FF047FA064BB8
:1007000001221A7001F01CF947F065FFFCE700BFF9
:10071000A1E60500A2B80500005A0020F0B5444B40
:10072000BFF35B8F87B0002053E8002F43E8000140
:100730000029F9D1BFF35B8F3E4D04466946284638
:1007400012F07EFF002871D19DF80030072B0BD8E6
:10075000DFE803F004141C4A515559619DF80C1050
:1007600001982CF09BFE044614F11D0F5BD0002273
:1007700000236946284612F0CFFEDFE7BDF80E20C1
:100780009DF80C1002982CF0A3FEECE745F0B0FFAA
:100790004FF47A740B46DDE90467A0FB040104FB07
:1007A0000311C20B42EA4142CB0B964277EB0303A3
:1007B00018DB45F09DFF0B46A0FB040104FB031171
:1007C000C20B42EA4142B21A43F6FF3604FB026210
:1007D0004FF47056B2FBF6F29DF80C1001982DF014
:1007E0003BF8C0E70122F7E79DF80C1001980022C2
:1007F0002DF04EF8B7E7019847F06BF8B3E7019892
:1008000047F079F8AFE7BDF80C20BDF80E1002985C
:1008100047F084F8A7E7BDF80C20BDF80E10029849
:1008200047F092F89FE7044813F08CFC07B0F0BD46
:10083000504C00204C080020544C0020024B1868FB
:10084000003818BF01207047644C0020014B186825
:1008500014F05EBB644C0020014B186814F076B9AC
:10086000644C0020014B1878704700BF005A0020EC
:1008700013B50F490F4813F0F3FB0F4B00241C7006
:100880000E4B1C600E4B1C7047F075FC28F08AFA6A
:10089000684600F04FFE68462DF090FC20462DF093
:1008A000BDFC4FF4803043F0B4F9204602B010BDD7
:1008B0003D0B0100544C00207A0400200859002010
:1008C0008DB0002030B587B005460C4618220021B7
:1008D000684640F07BFE0195ADF80C4008480022C8
:1008E0000023694612F08AFD044628B9054813F032
:1008F00029FC204607B030BD6FF01C04F9E700BFAB
:100900004C080020544C002070B586B006460D46B9
:10091000144600211822684640F058FE02238DF844
:1009200000300196ADF80C5045F0E2FE4FF47053E4
:1009300003FB04F24FF47A730D46A0FB0301B2FBF4
:10094000F3F403FB0511C20B42EA414212194FEACC
:10095000D13343F10003CDE90423084800220023EA
:10096000694612F04BFD044628B9054813F0EAFB2E
:10097000204606B070BD6FF01C04F9E74C0800205B
:10098000544C002030B587B005460C461822002193
:10099000684640F01BFE03238DF800300195ADF84A
:1009A0000C40084800220023694612F027FD044647
:1009B00028B9054813F0C6FB204607B030BD6FF0DC
:1009C0001C04F9E74C080020544C002010B586B0F8
:1009D000044618220021684640F0F8FD04238DF8F3
:1009E00000300194084800220023694612F006FDF9
:1009F000044628B9054813F0A5FB204606B010BDF3
:100A00006FF01C04F9E700BF4C080020544C002094
:100A100070B586B006460C46154600211822684679
:100A200040F0D4FD06238DF800300296ADF80C504E
:100A3000ADF80E40084800220023694612F0DEFCA3
:100A4000044628B9054813F07DFB204606B070BD6A
:100A50006FF01C04F9E700BF4C080020544C002044
:100A600008B5084B1A785AB901221A7042F0B8FA40
:100A700042F0B3FA00F086FEBDE8084042F0AEBA9C
:100A800008BD00BFFF5900200A4908B50B685B0785
:100A900008D0094B0948C91A8908890141F00101A8
:100AA0003FF0DDF9F6F756F842F09DFA0120F5F730
:100AB00077FD00BF44070020E8060020D6E60500C9
:100AC00008B5EFF3058353B10749084840F22E22D9
:100AD0003EF082FD044840F22E213FF057F80448D2
:100AE000BDE8084012F0C4BEA1E60500A2B80500AA
:100AF0000408002010B5EFF3058353B109490A48F3
:100B000040F235223EF068FD064840F235213FF0C4
:100B10003DF80648BDE810404FF0FF324FF0FF337C
:100B200012F0CEBDA1E60500A2B805000408002021
:100B30000146014815F04ABCD002002010B586B02D
:100B40001148694612F07CFDB0B9BFF35B8F0F4BC3
:100B5000012153E8002F43E800100028F9D1BFF32A
:100B60005B8F8A4208D00A4C002120462CF096FC6C
:100B700020B90320FFF7DCFF06B010BD00214FF4C1
:100B8000004014F011FCEFE74C080020504C00200E
:100B90001D07010073B500230546009345F0A8FD2D
:100BA00004461248124A4FF4004600210023E6FB97
:100BB0000501EFF7C3FE02460B4601210D4815F073
:100BC0002FFB0D4801AA694645F035FE009B13B185
:100BD000094845F02DFE45F08BFD054A001BA0FBA2
:100BE0000223D00B40EA434002B070BD3F420F00E9
:100BF00040420F00BC020020D002002010B588B097
:100C00000D4C0E4900220023CDE9062300230322C8
:100C1000CDE90323CDE9013300934FF40062084B83
:100C2000204612F0F9FA074B18600749204608B031
:100C3000BDE8104012F04AB9B019002000E00020D1
:100C4000E1060100644C0020F1E6050008B51349F7
:100C50000120F9F737FA60B111490B685A0708D03B
:100C6000104B1148C91A8908890141F001013FF070
:100C7000F6F80E490220F9F725FA70B108490B6819
:100C80005B070AD0074B0A48C91A89088901BDE8E1
:100C9000084041F001013FF0E2B808BD684C002077
:100CA00044070020E806002002E705006C4C002005
:100CB00024E70500012870B51DD85E18B6F5005F61
:100CC0001CD8F2B103B301EB40311148006840F089
:100CD0004BFA90B10F4A13685B0709D00E4BD21A3A
:100CE00092089201014642F001020C483FF0C6F81A
:100CF0004FF0FF3001E06FF0380070BD6FF016006C
:100D0000FBE76FF00B00F8E76FF00C00F5E700BFB2
:100D1000684C002044070020E806002049E7050051
:100D2000012870B51C4622D85E18B6F5005F21D8A0
:100D30001AB30BB9002070BDA40821D001EB4031DB
:100D40001148006840F02CFA01460028F2D00F4A02
:100D500013685B0708D00E4B0E48D21A9208920116
:100D600042F001023FF08AF84FF0FF30E3E76FF006
:100D70003800E0E76FF01600DDE76FF00B00DAE710
:100D80006FF00C00D7E700BF684C0020440700203C
:100D9000E806002058E70500012838B5044605D9C3
:100DA0000025204628F0DEFF284638BD0C4B4103C5
:100DB0004FF40052186840F021FA01460028EFD0A5
:100DC000084A13685B0708D0074B0848D21A9208F4
:100DD000920142F001023FF051F84FF0FF35E0E799
:100DE000684C002044070020E806002068E7050062
:100DF00013B50D4B0D480024CDE9003404230068E1
:100E00000DEB0302214640F0AFF950B904226946C8
:100E10000DEB020040F0A8FBB0FA80F0400902B0F0
:100E200010BD2046FBE700BFE737DDF66C4C002025
:100E300002460C4808B500680B46042140F094F9BE
:100E400078B1094A13685B0709D0084BD21A920897
:100E50009201014642F0010205483FF00FF84FF0C1
:100E6000FF3008BD6C4C002044070020E80600203D
:100E700078E7050008B50B46114602460B480431D9
:100E8000006840F071F978B1094A13685B0709D02E
:100E9000084BD21A92089201014642F0010206481C
:100EA0003EF0ECFF4FF0FF3008BD00BF6C4C00205F
:100EB00044070020E806002098E7050010B5104C14
:100EC000BFF35B8F04F12003002153E8002F43E8B8
:100ED00000100028F9D1BFF35B8F012A0ED12068E2
:100EE00083685B6898472068217F83684268527AEC
:100EF0008A4203D9BDE810401B69184710BD00BFE6
:100F0000704C00202DE9F0412A4CBFF35B8F04F1B7
:100F10002003012153E8002F43E800100028F9D1F5
:100F2000BFF35B8F002A42D1637F83BB224811F05D
:100F300075FC206040B92149214854223EF04CFB09
:100F40001E4854213EF022FE0025257725612068A9
:100F500042F038F84FF4F0511A4A0023A0FB010187
:100F6000EFF7ECFC0646A0608846206842F02AF8BD
:100F7000144B0246A6FB030103FB08112B46EFF7B7
:100F8000DDFC114B6360C4E905050123637720682C
:100F900083681B6898472068217F83684268527A7B
:100FA0008A4204D9BDE8F041DB68084A1847BDE829
:100FB000F08100BF704C0020B6D30500B1E70500FA
:100FC000A2B8050040420F00D10F0100744C002070
:100FD00010B5124CB1B9BFF35B8F04F1200353E895
:100FE000002F43E800100028F9D1BFF35B8F012ADE
:100FF00008D1D4E905231344B3F5705FA36101D28E
:10100000FFF780FFA369B3F5705F06D3A3F57053B4
:10101000A361BDE810402CF073B810BD704C0020E7
:10102000044BBFF35B8F186ABFF35B8F003818BFA8
:1010300001207047704C002008B5044845F0ADFA17
:101040000220FFF775FD002008BD00BFC84C00203E
:1010500047F6FF73994218BF01EB8101054B15BF9D
:101060002F390122C9B21A7618BF83F8201001481F
:1010700012F080BD984C002013B50023ADF8063067
:10108000064BADF804001B6805481C69006801ABFD
:1010900002220121A04702B010BD00BFC04C0020B9
:1010A000C44C002013B5064B01901B6805481C6911
:1010B000006801AB00220121A04702B010BD00BFB3
:1010C000C04C0020C44C002013B50023ADF80630FE
:1010D000064BADF804001B6805481C690068012236
:1010E00001AB1146A04702B010BD00BFC04C0020AC
:1010F000C44C0020F8B5114C002323764FF47053F4
:1011000058434FF47A73B0FBF3F0E0614FF0FF32D5
:101110004FF0FF33204612F069FD094D094F0A4E8A
:10112000E1693B682868DB6A324689B2984700B9B2
:10113000F8BD4FF4FA7014F067F9F1E7984C00200D
:10114000C44C0020C04C0020511001002DE9F0419A
:10115000134C144E144F05464FF0FF3310484FF018
:10116000FF3212F043FD237E3BB994F820302B7000
:101170000B48BDE8F04112F0FDBC0023DFF82C80E5
:101180002376E1693B683068DB6A424689B298475A
:101190000028E1D04FF4FA7014F036F9F1E700BFFF
:1011A000984C0020C44C0020C04C0020511001007D
:1011B000034B044A1B680146DB681068184700BFF0
:1011C000C04C0020C44C0020054B064A1B6810B5DB
:1011D0005B690446014610689847034B1C7010BDBC
:1011E000C04C0020C44C00206B04002038B5094CD2
:1011F00094F900208032054608D107490748CD22DE
:101200003EF0EAF90448CD213EF0C0FC23782B7073
:1012100038BD00BF6B040020E3E70500A2B805005D
:101220001FB50023CDE901330393064B8DF804006D
:101230001B6805485B6A006801AA0221984705B04F
:101240005DF804FBC04C0020C44C00201FB50021F9
:101250000123CDE901118DF80530064B8DF804000E
:101260001B6805485B6A039101AA0068984705B0AE
:101270005DF804FBC04C0020C44C002008B5054BB1
:10128000054A1B681068DB699847044B02225A70B4
:1012900008BD00BFC04C0020C44C00206B040020DF
:1012A00008B5054B054A1B6810681B6A9847044B34
:1012B00000225A7008BD00BFC04C0020C44C002062
:1012C0006B040020024B5878831E584258417047E7
:1012D0006B040020024B5878003818BF012070477B
:1012E0006B0400202DE9F047137886B08846023B56
:1012F000511C9BB203910591054600260020002158
:10130000CDE90166ADF81030ADF81230FAF786FF7E
:101310000446002841D03B4F022D3E602ED0032DC5
:101320004FD0012D58D1DFF8E880374B374E0322DC
:101330005A70D8F8003030685B689847D8F80030A9
:1013400010F0080FD3F81880306801AB22460CBFAC
:1013500029460221C0470546204640F08EFD2A4B13
:10136000022215F1230F5A703AD0002D45D138686A
:1013700027F012FF0120FFF7DBFB3CE0DFF890A035
:10138000224EDAF8003030685B68984710F48075B8
:1013900006D1204640F071FD284606B0BDE8F08732
:1013A000194B30684FF47A71A8FB018903215970F9
:1013B000C4E90C89DAF8003022469D6901ABA847E0
:1013C000C9E7114B5D70124B02461B680F489D69BF
:1013D000006801AB3146F2E740F04FFD3046DCE7F4
:1013E000042027F005FF0020FFF7A2FB40F2F220C7
:1013F000002113F0D9FF0120CFE7012027F0F8FEEC
:101400000020B8E7944C00206B040020C44C00205E
:10141000C04C00201FB50023CDE902330A4B0190D8
:101420001B680A488DF8082081F001018DF8091029
:101430005B6A006801AA01219847B0FA80F0400970
:1014400005B05DF804FB00BFC04C0020C44C002078
:1014500030B50C4D0C4C85B00023CDE9013303931E
:101460008DF808302B6820685B6A01AA0121984733
:101470002B6820685B6A01218DF8081001AA984743
:1014800005B030BDC04C0020C44C0020024B186891
:10149000003818BF01207047C84C0020F7B505463A
:1014A00010B9002003B0F0BD20480022002312F044
:1014B00007FB04460028F4D0836800268BBB314626
:1014C000284646F0A9FA0190204640F02CFD32460D
:1014D0000199174E204640F0A1FD284646F05BFAE0
:1014E00094F85D3000F8023C94F85C3000F8013C60
:1014F000236A042128465E434FF47A77A36AB3FB3C
:10150000F7F746F069FB3E44066094F85E10284603
:10151000C1F3400146F044FE204640F0AEFC0120FD
:10152000C0E79A891B681644C8E700BFC84C002072
:1015300040420F0070B5214D2B68044653B9204935
:10154000204840F20E223EF047F81D4840F20E219E
:101550003EF01CFB2B681B681B7D082B0AD018492A
:10156000184840F20F223EF037F8154840F20F219C
:101570003EF00CFB2B681B681D691E7DA54212D234
:10158000AB199C420AD210490E4840F217223EF095
:1015900023F80D4840F217213EF0F8FA731E1D445F
:1015A000013C26B970BDEED0A3199D42EAE715F8BB
:1015B000013904F8013F013EF3E700BFBC4C0020B5
:1015C000E3E70500A2B805004FD5050070B5044655
:1015D00050B92149214840F219223DF0FDFF1E4833
:1015E00040F219213EF0D2FA1D4B1E4D1C602368BB
:1015F0001B682B6053B91849184840F21D223DF072
:10160000EBFF154840F21D213EF0C0FA2B68164E44
:101610009A68326052B9104910484FF408723DF090
:10162000DBFF0D484FF408713EF0B0FA0120FFF7E0
:101630000DFEFFF71DF90D4844F0A2FF01221146EF
:101640000B4844F0BFFF336828681B6A9847204660
:10165000BDE87040FAF7CCBCE3E70500A2B805008E
:10166000BC4C0020C44C0020C04C0020C84C0020C2
:10167000984C002070B50C46896800220B463BB997
:10168000052A14D0294A1368580705D1012070BDD6
:1016900098891B680244F2E7254B26492648D21A4E
:1016A0009208920142F001023EF0E8FBEEE78B68FF
:1016B0001B7803F00703022B0CD01C4A1368590750
:1016C000E4D01B4B1B491D48D21A9208920142F0EC
:1016D0000102E9E71A4E326862B1144B1A685207E8
:1016E00008D0134917485B1A9B089B0143F001017E
:1016F0003EF0B5FB144D2946052201F8012B20468A
:1017000040F08CFC00280DDA08490B685B07BDD05F
:10171000074B0E48C91A8908890141F001013EF0C2
:101720009EFBB3E735600020B1E700BF440700200F
:10173000E806002086E805001BE8050030E8050003
:10174000944C00204BE80500015A00206CE805008D
:1017500007B50023019304210DEB010040F044FF85
:1017600040B10649064862223DF036FF0348622137
:101770003EF00CFA019803B05DF804FBA2E8050006
:10178000A2B8050008B5094B0948186044F07FFE6F
:1017900050B9084908486A223DF01EFFBDE80840DC
:1017A00004486A213EF0F2B908BD00BFE44C0020B5
:1017B00050A20500A2E80500A2B805002DE9F041FD
:1017C000804690B00F4616460AB101B158B930496B
:1017D000304871223DF000FF2D4871213EF0D6F9CE
:1017E00010B0BDE8F0812C4D2B6843B92849294839
:1017F00025223DF0F1FE264825213EF0C7F908AC30
:101800001C22002120463FF0E1FE244B28680F9364
:101810000023CDE90633102382680593CDE9033612
:10182000012300935668CDF8288002970B908DF81D
:1018300020301A462146B04770B115491548362266
:101840003DF0CAFE362112483EF0A0F928688368B0
:1018500021469B689847C3E79DF82030012B08D0AC
:101860000F490C48D1223DF0B7FE0D48D1213EF082
:101870008DF9099B079402A9204698470028E5D0D6
:10188000034904483D223DF0A7FE3D21DBE700BFB0
:10189000A2E80500A2B80500E44C002010003200C8
:1018A000D5E8050070B550B3154B164A1978164C9B
:1018B000117000251D700123BFF35B8F54E8002FCA
:1018C00044E800310029F9D1BFF35B8F4FF47A76F9
:1018D0007043FFF75FF9BFF35B8F4FF4705300F570
:1018E0006F503F30B0FBF3F05843B0FBF6F054E8D4
:1018F000003F44E80052002AF9D1BFF35B8F70BD6E
:101900007A04002079040020E84C0020024B1A7869
:10191000024B1A70704700BF790400207A0400203F
:1019200010B5034C20463EF0A4F80028FAD010BDB4
:10193000E0020020014B1878704700BF075A0020D2
:1019400010B50EF04FF9436873B91D490B6858077D
:1019500035D01C4B1C48C91A8908890141F0010186
:10196000BDE810403EF07BBA184C402020700DF0CE
:101970009BFC78B9124A1368590720D0114B217883
:101980001348D21A92089201BDE8104042F00102B9
:101990003EF074BAD0F803305BB109490B685B07BD
:1019A0000DD0084B0B48C91A8908890141F0010183
:1019B000D6E720780DF078FC074BC0F8033010BD57
:1019C00050070020E806002000E90500075A002023
:1019D0003BE905005FE90500F5190100014B1870AE
:1019E000704700BF085A0020014B1878704700BFAD
:1019F000085A002070B50546FEF736FD064E002455
:101A000056F8043B28469847012803D00134042C9B
:101A1000F6D1002070BD00BFECAE050073B51646D0
:101A20000D461A46044600285DD0002B5BD0312EAF
:101A30001CD8072E1ED9A6F10803292B1AD8DFE8D7
:101A400003F02A311936191919191C1919191919FC
:101A500019192A311936191919192A31193619196A
:101A600019192D331939191919192A31422E24D06F
:101A7000F02E32D01D4A334606E011781C4B1D4A29
:101A8000002908BF13461C4A2946204602B0BDE87B
:101A90007040F9F73DBC1378184AF5E792F9003029
:101AA000174AF1E71388F7E7B2F90030F8E713684F
:101AB000144AE9E71368144AE6E71978481C854296
:101AC00011DB00238B4203DB0023635402B070BDA3
:101AD00012F8015FE5540133F4E701230093082372
:101AE000FEF712F9F2E74FF0FF30EFE7C2E9050029
:101AF000AFE90500B4E9050018C10500BAE9050021
:101B0000BEE90500A4B7050022DF05002DE9F04F6E
:101B10004FF0010B0BEB42089A4608F1070383B024
:101B200003F4FF6302AFADEB030D02AE044689463A
:101B300015460021424630463FF048FD2B464A46B6
:101B40004146CDF800A03046FEF7DEF80028BBBFC6
:101B5000064B074A064A5946A4BF33460821204689
:101B60003EF065FD0437BD46BDE8F08FDEE90500B7
:101B700018C1050037B50E4A0821044600253EF07D
:101B800056FD0B23CDE9003520460A4A03230821E0
:101B90003EF04DFD084B094A204608213EF047FD26
:101BA0002046074A08213EF042FD284603B030BDDA
:101BB000F6E9050011EA050024EA05002BEA050014
:101BC00040FA050010B504460020FFF707FF204645
:101BD000054A08213EF02BFD2046044A08213EF02C
:101BE00026FD002010BD00BF46EA050040FA0500B2
:101BF00010B50446FFF7F8FE0849094B094A0028CA
:101C000018BF0B46204608213EF011FD2046064A2B
